:020000040800F2
:10000000D8530020F50100088D7F00080545000841
:10001000917E0008EF0A000811FA000800000000B5
:10002000000000000000000000000000CDD4000827
:10003000B70C0008000000001B950008C5DF000891
:100040000F0200080F020008F9E100080F02000883
:100050000F0200080F020008B90E0008BF0E0008CA
:100060000F0200080F0200080F0200080F0200082C
:100070000F0200080F0200080F020008FD0B000825
:100080000F0200080F0200080F0200080F0200080C
:10009000000000000F020008C50E00080F02000853
:1000A0000F0200080F0200080F02000801E200081A
:1000B0000F0200080F0200080F0200080F020008DC
:1000C0000F0200080F0200080F0200080F020008CC
:1000D0000F02000849F100080F0200080F02000893
:1000E0000F0200080F020008719D00080F020008AF
:1000F0000F02000800000000000000000F020008CE
:100100000F0200080F020008D1CA00080F02000801
:100110000F0200080F0200080F0200080F0200087B
:100120000F0200080F0200080F0200080F0200086B
:100130000F0200080F02000800F002F800F04AF871
:100140000AA090E8000C82448344AAF10107DA4532
:1001500001D100F03FF8AFF2090EBAE80F0013F03A
:10016000010F18BFFB1A43F001031847580403009E
:10017000780403000A4410F8014B14F00F0508BF7F
:1001800010F8015B240908BF10F8014B6D1E05D063
:1001900010F8013B6D1E01F8013BF9D1641E03D03C
:1001A000641E01F8015BFBD19142E4D3704700006B
:1001B0000023002400250026103A28BF78C1FBD870
:1001C000520728BF30C148BF0B6070471FB51FBD25
:1001D00010B510BD00F0A4F91146FFF7F7FF11F0BC
:1001E0002DF800F0C2F903B4FFF7F2FF03BC00F0F2
:1001F000C5F900000948804709480047FEE7FEE7C7
:10020000FEE7FEE7FEE7FEE7FEE7FEE7FEE7FEE7C6
:1002100004480549054A064B70470000F5E100080F
:1002200039010008D84D0020D8530020D84F0020B5
:10023000D84F002053EA020C00F069802DE9F04B02
:100240004FF00006002B1FBFB3FA83F503FA05F445
:1002500024FA05F65E4012BF1643B2FA82F502FA9E
:1002600005F4C5F120051EBF22FA05FC44EA0C0482
:10027000203556EA044C4FEA144418BF641C4FF072
:1002800000084FF00009904271EB030C39D30029AC
:1002900019BFB1FA81F701FA07F6B0FA80F700FA50
:1002A00007F6C7F120071EBF20FA07FC46EA0C0636
:1002B0002037B6FBF4FCA7EB0507103F07F01F0B38
:1002C000CBF120062CFA06F60CFA0BFB44BFB34622
:1002D0000026202FA4BF5E464FF0000B5BEA060C01
:1002E00008BF4FF0010B19EB0B0948EB0608ABFBFD
:1002F000027C06FB02CC0BFB03CCC01B71EB0C0198
:10030000C1E70B46024641464846BDE8F08B13B5AF
:10031000084318BF4FF0FF300146AFF30080BDE83F
:100320001C40704710B5431C02E010F8011B71B16E
:100330008107FAD14FF0013202C88C1A8C4314EABB
:10034000C211F9D0C01A0A0603D0C01E10BDC01ACF
:1003500010BD0A0401D0801E10BD0902FCD0401E51
:1003600010BD032A40F2308010F0030C00F015801D
:1003700011F8013BBCF1020F624498BF11F801CBA8
:1003800000F8013B38BF11F8013BA2F1040298BF0D
:1003900000F801CB38BF00F8013B11F0030300F077
:1003A0002580083AC0F0088051F8043B083A51F81B
:1003B00004CBA0E80810F5E7121D5CBF51F8043B20
:1003C00040F8043BAFF30080D20724BF11F8013B93
:1003D00011F801CB48BF11F8012B24BF00F8013BF5
:1003E00000F801CB48BF00F8012B704710B5203A48
:1003F000C0F00B80B1E81850A0E81850B1E81850D0
:10040000A0E81850203ABFF4F5AF5FEA027C24BFA1
:10041000B1E81850A0E8185044BF18C918C0BDE88A
:1004200010405FEA827C24BF51F8043B40F8043B53
:1004300008BF7047D20728BF31F8023B48BF11F808
:10044000012B28BF20F8023B48BF00F8012B704762
:1004500002F0FF0343EA032242EA024200F024B81A
:100460004FF000020429C0F0128010F0030C00F0DD
:100470001B80CCF1040CBCF1020F18BF00F8012B5B
:10048000A8BF20F8022BA1EB0C0100F00DB85FEA29
:10049000C17C24BF00F8012B00F8012B48BF00F8F5
:1004A000012B70474FF0000200B513469446964664
:1004B000203922BFA0E80C50A0E80C50B1F1200177
:1004C000BFF4F7AF090728BFA0E80C5048BF0CC025
:1004D0005DF804EB890028BF40F8042B08BF704783
:1004E00048BF20F8022B11F0804F18BF00F8012BF5
:1004F000704770477047704710B500F009F8006802
:1005000010BD10B5044600F003F8046010BD0000F3
:1005100000487047500100200048704750010020FB
:100520007546FFF7F9FFAE4605006946534620F0D1
:100530000700854618B020B5FFF76AFEBDE82040E9
:100540004FF000064FF000074FF000084FF0000B8F
:10055000AC46ACE8C009ACE8C009ACE8C009ACE8FE
:10056000C00921F007018D46704710B50446AFF36E
:1005700000802046BDE81040FFF735BE0149182035
:10058000ABBEFEE72600020070470000B0B504468F
:1005900000688168490701D40020B0BD81688907DF
:1005A00004D48168464A11401031816001F06CFE2C
:1005B0000546206880684007EED501F065FE401BC7
:1005C0000328F6D3206880684007F2D5714607F00B
:1005D0000EFD8E46B0BD00BFB0B501680446886808
:1005E0008A6880074FF0000020D412F001021DD06D
:1005F000886800F00500012816D18868304A10404C
:10060000023088600320086001F03EFE0546206845
:100610008068C0070BD001F037FE401B0328F6D3DB
:1006200020688068C007F2D007F0E1FCB0BD002070
:10063000B0BD00BF7CB504460020019021688A68E7
:10064000D20707D11E4E886806F12F02104202D051
:1006500007F0CDFC7CBD8868304040F00100886028
:1006600018480068000204D4607E01280ED10020E2
:100670007CBD154815490068B0FBF1F001300190D0
:1006800001980028F0D001980138F8E701F0FCFD4E
:10069000054620680168C907E9D18168C90704D106
:1006A0008168314041F00101816001F0EDFD401BA6
:1006B0000328EED320680068C007EAD1C8E700BF6E
:1006C000E8FFFF7F0827014044010020400D0300A0
:1006D000BFB5002504460395CDE9015507F0F2F9B1
:1006E000144800F061FE08B100F00AFC11480395BF
:1006F000CDE9014501A900F0DFFE08B100F000FCE2
:100700000C4801F075F908B100F0FAFB094C4FF004
:10071000FF31204601F014F9204601F091F92046FE
:1007200000F0DCFF0546204600F092FF284604B0AA
:10073000B0BD00BF78490020BCB56B4C00204FF421
:100740007A750DF10602A62101238DF807008DF8B8
:1007500006000095204601F099FE642001F045FB5B
:100760000DF107022046A6210123009501F034FE79
:100770009DF80700BCBD00BFF8B50246002001216E
:100780000DF10F038DF80F006420CDE90031A62193
:1007900001230290544801F0D5FE9DF80F0004B0EB
:1007A00080BD00BF70B586B014460D460646642075
:1007B00006210DF112020123CDE9002102904A48E1
:1007C000A621322201F0BEFEBDF812003080BDF835
:1007D00014002880BDF81600208006B070BD00BF50
:1007E000BCB5FFF7A9FFE52803D0284B009007F020
:1007F0003AFD002000F04EF8082000F04BF80820E9
:1008000000F04CF80F4C2E200021A0472720FF219C
:10081000A0470D4D24202978A0472F20E721A0478D
:1008200069782520A047A9782620A0472E203821C6
:10083000A0472D203821A0473020BDE8BC40FFF75D
:100840009BBF00BFC5080008420000201CB5FFF791
:1008500073FFE52803D00D4B009007F004FD2E2018
:10086000002100F02FF80A4C0320A0470020A047E9
:100870000820A0470D2000F011F82E20C72100F01D
:1008800021F80120BDE81C4000F00CB8B785010834
:10089000950800080146312000F014B801462C20CC
:1008A00000F010B810B504462D20FFF765FF00F0EA
:1008B000F70040EAC400C1B22D20BDE8104000F0AE
:1008C00001B80000F8B502468DF80F104FF47A70A9
:1008D00001210DF10F03CDE9003102900248A6215C
:1008E000012301F0A3FE8FBD3C4A0020F0B589B082
:1008F00005AE0C46054600211022304610F0C1FC22
:1009000030463146224610F0BFFA9DF9140000210E
:10091000B0F1FF3F06DD0F290CD007F0F3FBFAE73B
:1009200007F0F0FB0F29FBD19DF82300872181EA16
:10093000400002E09DF8230040008DF82300D4F829
:10094000140110280AD104F201100021102936D018
:10095000425C735C5A4042540131F7E79DF9141030
:100960000022B1F1FF3F06DD0F2A0CD007F05EFD3B
:10097000FAE707F05BFD0F2AFBD19DF823108722D1
:1009800082EA410102E09DF8231049008DF823100E
:100990008021204480F801110021D4F81401013095
:1009A0001028C4F81401F4D304F201100021102916
:1009B00005D0425C735C5A4042540131F7E7002095
:1009C000102803D0211807F028FCF9E701AE04F144
:1009D000F1011022304610F040FC304629462246F4
:1009E00010F052FA05A80021102210F04AFC09B0BC
:1009F000F0BDB0B50446F13000211022002510F002
:100A000040FCC4F8145120460021F022BDE8B0405B
:100A100010F037BC02460846102110F091BB2DE9BA
:100A2000F04385B00E46D0F814111446804699B3B1
:100A300008EB0100C1F1100527463146A54238BF39
:100A40002F4600F20110BAB210F007FCD8F81401DA
:100A5000A5423844C8F8140146D2102844D30020D7
:100A6000102804D008EB000107F0D7FBF8E708F1E5
:100A7000F1050DF1040910224846294610F0EDFB5E
:100A800048464946424610F0FFF92846494610229A
:100A900010F0E3FBE41B3E4408F1F10701AD112C1B
:100AA0001AD30020102805D0395C325C51403954EB
:100AB0000130F7E728463946102210F0CEFB2846D1
:100AC0002946424610F0E0F938462946102210F037
:100AD000C4FB103C1036E2E708F20110A2B2314626
:100AE00010F0BBFBC8F8144105B0BDE8F083FEE789
:100AF0002DE9F041CCB051B3DDF84881B8F1000FD9
:100B000025D0074602A81C4615460E46FFF771FF82
:100B100001A9204600F08CFB0446C8B90198411C8D
:100B200002A8FFF777FF27B102A839461022FFF786
:100B300076FF02AF31462A463846FFF770FF48A8D5
:100B40003946FFF7D3FE4898C8F8000000E00224B9
:100B500020464CB0BDE8F081B8B170B50C4C4FF0F8
:100B6000FF3200238B420ED0C55C6A400025082D61
:100B700007D202F0010601357642264086EA52028B
:100B8000F5E70133EEE7D04370BD0020704700BFAA
:100B90002083B8EDB0B586B000F062FF00F06AFFC8
:100BA00000F062FF032001210490002002910390D5
:100BB000059003F08FFE03F08DFE4FF480500E4C35
:100BC000019001AD2046294601F08CFA4FF4005007
:100BD00029460190204601F085FA20464FF48051C5
:100BE000002201F04BFB20464FF40051002201F09F
:100BF00045FB06B0B0BD00BF00040048014801F04D
:100C000001B800BFDC49002010B51049436C104CFE
:100C100001F1640223F00303C2640268A24238BFF8
:100C200004F57E711944142381646FF00701A24218
:100C300051FA82F1B1FBF3F128BF0731012201F033
:100C40001F0102FA01F1016510BD00BF1C0802403E
:100C50000804024010B5436807490124543003F0EA
:100C60007F0301F14002013B01EB830103F0030329
:100C700004FA03F30EC010BD00090240F0B500F104
:100C80004C0670CE656016B1D0E916456560046803
:100C90008568D0E91060012700F01C00102D07FACC
:100CA00000F070600846636008BF1046A06008BF8F
:100CB0000A46E260F0BD70471FB504460020022CD2
:100CC000CDE90200CDE9000003D0032C22D102209F
:100CD00000E001208DF80000180A8DF804208DF83E
:100CE00001108DF807308DF80800100C8DF8060003
:100CF000100A22468DF80500080C8DF80300080A3A
:100D000001218DF8020068460CF0A4FD002818BFF0
:100D10000F2000E00B2004B010BD00002DE9F04FC3
:100D20008DB052484FF00008DFF83891DFF838A155
:100D30004F4FDFF840B14FF40071CDE90588CDE9A0
:100D40000388CDE90188C0F800804B48C9F80080CD
:100D5000CAF80080C7F80080CBF80080C0F8008097
:100D600007A810F017F810B144A307F078FC4B4D1A
:100D7000494907A800232A460FF0EAFF484C07F02C
:100D8000FBFC484D0426C4F80080B6F5806F0BD0FC
:100D9000A05911F0B1F807F018FE07F093FD10F01C
:100DA000E9FDA0510436F0E73D4806AA03AB07F081
:100DB00049FD0398394D3C490023002638600698C8
:100DC0002A46C9F8000007A80FF0C2FF374C07F009
:100DD000D3FC344D26600426B6F5806F0BD0A059A5
:100DE00011F08AF807F0F1FD07F06CFD10F0C2FD7C
:100DF000A0510436F0E72D4805AA02AB07F022FD0A
:100E00000298264D2A4900230026CBF800000598B9
:100E10002A46CAF8000007A80FF09AFF254C07F0F1
:100E2000ABFC204D26600426B6F5806F0BD0A05990
:100E300011F062F807F0C9FD07F044FD10F09AFDCB
:100E4000A0510436F0E71B4804AA01AB07F0FAFCF6
:100E50000198094908600498044908600DB0BDE88C
:100E6000F08F00BFD4010020D0010020CC01002071
:100E70006C31002070310020743100200941524D46
:100E800020207266667420696E6974204641494C60
:100E900045440D0A000000006C190020D00A002013
:100EA000783100200000703F6C210020783900204C
:100EB0006C29002078410020012001F009B90220AE
:100EC00001F006B9402001F003B90020704700008E
:100ED000B0B50649094D064A064B074CC0E900511A
:100EE000C0E9022403610020B0BD00BF00009041B2
:100EF00000004842AB0305000D093E0000007A44A3
:100F0000EFF3108072B6FEE7F8B5CDE902010220DA
:100F1000019001A812B100F0C5FF02E0694600F09F
:100F20006BFF6FF00101022808BF0121002808BFF4
:100F30000146084604B080BD2DE9F84F07466FF022
:100F4000040000297DD0894642EA0701904611F04D
:100F5000070176D1414843490068096800296ED4E9
:100F60003F496FF000629A46464601EA802007EB4F
:100F700008011144B1FBF0F202FB1011CB0A07F19A
:100F80007841B1FBF0F2009302FB10104FEAD02B36
:100F900038466FF3DF209B4518BFC0F50066009808
:100FA000834550D8002338463146FA18540706D0F6
:100FB0001278FF2A16D1013301390130F5E7CB0849
:100FC0003BB1D2E900452C4001340BD1013B083242
:100FD000F6E721F0070291422DD0835CFF2B01D16F
:100FE0000132F8E7BAF1000F30D04FF000604FF453
:100FF000006200EBCB24504621460EF069FB3846D8
:10100000B2B249466FF3DF2050440EF061FB584600
:1010100001210022FFF778FFE0B9204651464FF446
:10102000006200F039F8A8EB0600B14437440BF138
:10103000010B0646B3E7384649463246F1E76FF002
:101040000300BDE8F88F0020BDE8F88F6FF00400C2
:10105000BDE8F88F6FF00100BDE8F88FE075FF1F65
:1010600000FCFF0314400058F8B5384F1C461546E5
:101070000646D6E9000161406840084309D0386857
:101080000003FCD4012031462A46234600F048FFE5
:10109000EFE70020F8BD00BFFEB50C460546D708B7
:1010A0006E468FB13046214608220EF011FBDDE975
:1010B000002302EA0300013002D02846FFF7D4FFE4
:1010C000013F08350834ECE7FEBD0000B0B51F4A0B
:1010D000536843F480235360EFF31083EFF31084DD
:1010E00072B6402420C9013C20C02506FAD1106800
:1010F000C003FCD483F31088B0BD00BF70B5134E9D
:10110000044601F0C1F805463068C00306D501F079
:10111000BBF8401BA042F7D3032070BD3068C10765
:1011200001D0012131604CF2FA31084009D0084960
:1011300048603060012070BD01F0A6F8401BA0425D
:10114000EAD230684003F7D4002070BD1040005848
:10115000BC4B002080B50CF0BBF940F6E44188425E
:1011600001D9FE200DE0B0F5E16F01D2002008E0CA
:101170000549C0EBC01001EB400040F2DC51B0FB70
:10118000F1F0C0B280BD00BF1006F9FF10B5854870
:101190000068411C00D010BD01F080F8044601F049
:1011A00083F8444001F086F8604010BD008871B9B2
:1011B00049F6B02142F210738A4238BF4FF47A7375
:1011C000B2F5616F38BF6423834228BF18460028F8
:1011D00008BF01207047000070B50B4A92F820301C
:1011E0007BB1002402F11C059C420AD20E78864293
:1011F00008D00E1DA94208BF02F10C063146013489
:10120000F2E70021084670BDA80A002010B5074A81
:101210000223043A3BB112F8044F013B8442F9D156
:1012200000200A6010BD0C2010BD00BFA8000020E7
:1012300010B5084A0023126803F11104BB2C06D034
:1012400013441B7C83422346F6D106F0EFBF0320F4
:1012500010BD00BFE818002061B1013803280BD889
:10126000DFE800F0020C12190E48006802690A60FB
:1012700001690EE00A2070470520704709480068A0
:1012800042690A60416904E00648006882690A60B0
:101290008169016203E003480068C06908600020BA
:1012A000704700BFCC0A0020E0B50B498DF8010063
:1012B00091F8742091F8400091F880108DF8022088
:1012C0000E220029694608BF0D228DF800200AF081
:1012D0003BFFC0B28CBD00BF28870020FEB568462A
:1012E000FFF7F6FD019810F0C1FF06B080BD0000C9
:1012F000F0B585B0064613480D461349845730466D
:101300000AF0ECFC014611480023EAB2476A0120CA
:10131000072E0BD10525CDE90053CDE902204FF46E
:101320007A70002304FB00F2002007E00825CDE9D5
:101330000053CDE90220012022460123B84705B021
:10134000F0BD00BF54280108342801084C290108C9
:101350000348016802689142FBD1C843704700BF4F
:1013600008280040B0B504460E4801684A1C08D061
:1013700009BA61604168E1704268100E110C120AEE
:101380000CE000F08BFF054600F094FF054400F0F0
:101390008BFF010E6560020CE170010A6170A270A2
:1013A0002070B0BD8075FF1FF8B504460020009086
:1013B00094F85400012801D1022544E0012084F86A
:1013C00054002046FFF708F9054620688268A16DA1
:1013D000D20728D121F4817148F203030231A165BB
:1013E000C168C2689A4301EA030732490023C26018
:1013F0000022082B29D086680E4006F10046866040
:101400008668B6F1FF3F07DC009E01360096009E1D
:10141000B6F52E3FF4D30CE0D0F8B460013306F0FB
:101420007F063244E5E741F01000002184F85410B3
:1014300008E00020012584F85400A06D40F0100061
:1014400020F00200A0652846F8BD83680B4043F0F9
:1014500001038360D0F8B43023F07F0343EAD20263
:10146000C0F8B4208268114041F00201816000F0B0
:101470000BFF064620688168C90712D000F004FF00
:10148000801B0328F6D320688068C007F2D0A06DC7
:10149000012540F01000A065E06D40F00100E0651E
:1014A000D1E7C1683943C1600121A06D61F301003A
:1014B000BBE700BFE8FFFF7FF8B50022009290F87D
:1014C0005420012A01D10221B3E0012280F85420E6
:1014D000026893685B0711D403694C6843F0040306
:1014E000022C11D1544CA34219D10B68574CD9434B
:1014F00061EA0401946A2140916211E0816D41F03A
:1015000020018165012191E04B4DAB421AD1144677
:1015100054F8285F0B681E466FF39F4635E00B6852
:10152000B3F1FF3F00F38180F349464C0A68A342C0
:101530006BD0454CA3426BD0414CA34275D102F015
:10154000A07267E00B689D0393FAA3F5B5FA85F6E0
:1015500004F01F0508BFC3F3846606FA05FC076E96
:10156000D0F81CE00F26AE40B74347EA0C07BEEBAD
:10157000940F07660BD99C0EF64304F00F0404FA8F
:1015800005F5144654F8287F3E40354325605469DC
:1015900089682A4D01EA032124EA032429402143D2
:1015A000B3F1FF3F516140DCD34A254915688B42B6
:1015B00008BF15F4000105F0E07411D021498B42F9
:1015C00008BF15F080712BD01F4E0021B34208BF19
:1015D00015F480032AD107F0FCF941F4800123E0DF
:1015E00007F0F7F941F400011160BF49BF4A0968EB
:1015F000B1FBF2F10C2201EB410102EB8101009100
:10160000009991B100990139F9E702F4400201E033
:1016100002F0C0720B6823F0E0731A440A6004E021
:1016200007F0D7F941F0807111600021002280F8A5
:1016300054200846F8BD00BF0400008000FFFF03EF
:10164000001000B0004000B8002000B4FFFF03000D
:1016500070B558B10446806D40F00200A065204688
:10166000FEF794FF20B1054620680CE0012530E02C
:1016700007F06FF9054608B90120A0652068994A6E
:10168000816811408160416840F29F320026914399
:1016900041600260104AC1681140C160016921F0D7
:1016A00040410161416921F007014161016A01F096
:1016B000F0210162816A86628F48016821F0FE7123
:1016C0000160204600F01AF9E665266684F8546049
:1016D000A665284670BD00BF00023E830068006C0E
:1016E000704700002DE9FC4104460020019044B3FE
:1016F000254655F8580F30B9204600F00BF9002068
:1017000084F85400E06521688868C00013D48868B4
:10171000744A1040754A00F1805088607248006831
:10172000B0FBF2F0022202EB40000190019810B1F0
:1017300001980138F9E78868C00005D406F057FC25
:1017400003E00120BDE8FC8100208A682B68C2F319
:10175000800203F01003D2182A6803D042F010016F
:101760000120BBE022F4817202322A608A68D2072B
:101770002CD104F10808237E98E8C00146EA83339F
:10178000667E43EAC633A67E43EA46333B43276B75
:10179000002F28F0004718BF43F48053B8F1FF3FF3
:1017A000C8BF4FF400173B4394F82C7043EA47033B
:1017B00094F82070012F0ED15EB1A66D46F0200680
:1017C000A665E66D46F00106E66504E0D4F81080F3
:1017D0002CE043F48033666A26B106F4E0763343A6
:1017E000A66A3343CE68424F3E403343CB606368C2
:1017F000E66C03F040473E4394F83C70012F0AD159
:1018000004F1400E9EE880503E4346EA0C0646EA4C
:101810000E0646F001060F69364A3A403243B3F1EC
:10182000004F0A6118BFB3F1404F1ED1D4E90D3209
:101830004E6926F007061E434E61B8F1000F4E694F
:1018400026F0700646EA02124A611AD0B8F5001F67
:101850002CD1226E0026202E19D022FA06F707F08E
:101860000F070F2F0BD00436F5E7B3F1804FDDD013
:101870009A0C214B1E6862F395461E60D6E7042E33
:1018800005D10A4652F8286F66F00F060DE0E669AA
:101890001C2707EB86066FF00F0706F01C0607FAF9
:1018A00006F616430A4652F8287F1660496901F089
:1018B0000701994206D100210122E165A16D62F381
:1018C00001010BE0A06D40F0100020F00200A065C7
:1018D00054F85C0F40F00101012025462960BDE865
:1018E000FC8100BFE8FFFF6F44010020400D0300B2
:1018F0000102FEFF02FCFF1F0827014000680E499D
:10190000884200D070470D48016821F400710160E1
:10191000704700BF81B000680749884209D1074875
:10192000016841F400710160006800F400700090EB
:10193000009801B0704700BF0024014060000058CB
:101940002DE9F041044640690D46082801D10827D9
:1019500004E02068C068C00733D1042700F094FC7D
:1019600080466E1C2068016839420FD1002EF9D0E4
:1019700000F08AFCA0EB0800A84201D8002DF1D1AC
:10198000206800683842EDD106F01FBDA16D41F41A
:101990000071A165C16811F4406F21D1A17EF9B930
:1019A000016809071CD58168490711D4416840F2D4
:1019B000011221F00C014160A16D91430131A1653B
:1019C0000EE0A06D40F02000A0650120BDE8F08190
:1019D000A16D41F02001A165E16D41F00101E165DA
:1019E000217E09B90C2101600020BDE8F0810000D2
:1019F00010B5044600688068400703D494F854008A
:101A0000012801D1022010BD06F0BCFE08B106F08D
:101A10005DBF2168A06D40F60172084B90431C2207
:101A200000F58070A0650020E0650A6084F854002D
:101A30008A681A4004328A6010BD00BFE8FFFF7F49
:101A400010B506F011FE01D1022010BD06F098FB82
:101A500020B906F07EFF08B906F0F8FE06F036BFA2
:101A6000064806F07CBD00BF0448016821F004016F
:101A700001607047014806F0F2BA00BF042004E09C
:101A800050B3B0B590F82510022927D1016800F1B4
:101A900040041CCC0D6803F01C0325F00E050D60FE
:101AA000256825F4807525600C6824F001040C601D
:101AB000012101FA03F35360D0E913235360426D0F
:101AC00032B1136823F480731360D0E91623536096
:101AD00080F82510002104E0012107E00421C16302
:101AE0000121002280F82420BDE8B040084670475C
:101AF000B0B590F8251002292BD10168D0E9103239
:101B0000846C0D6825F00E050D600D6825F001054B
:101B10000D60216821F48071216002F01C01012216
:101B200002FA01F15960D0E913134B60416D31B1F4
:101B30000B6823F480730B60D0E916134B6000210F
:101B400080F8241080F82520826B2AB1904700216C
:101B500002E00421C16301210846B0BDF8B54FF091
:101B6000010C002846D00368254A7E4F04461968B8
:101B700002F5806521F00101196020490E1DB34274
:101B80003CBF0025C4F2020538BF07F580671F443B
:101B90001420B7FBF0F08700C4E910570025B342CA
:101BA0001D6038BF111D1C2202EA80000CFA00F0F3
:101BB00008602046FFF728F8606804F148030ECB60
:101BC000013803280D60536007D82046FFF742F81C
:101BD00004F1540207CA05604A60E563C4E915557B
:101BE000E565C4E90B55C4E90D5584F8245084F823
:101BF000255000E001252846F8BD00BF040402403E
:101C000000000240F0B5D0E910230168042403F07D
:101C10001C0316680D689C40344201D06F071BD42A
:101C200002249C40344201D0AF071FD426FA03F4AB
:101C3000240735D52C0733D50C6824F00E040C602E
:101C4000012101FA03F353600022C16380F82420CC
:101C500080F82510416B1FE00B689B0603D40B68CE
:101C600023F004030B605460016B15E00A689206D0
:101C700006D40A6822F00A020A60012280F82520B0
:101C8000002280F82420074A02F17C03994288BF91
:101C900002F580621460C16A11B1BDE8F0400847E6
:101CA000F0BD00BF04000240B8B3F8B504460220FE
:101CB0002B4984F8250004F10806206801F1080288
:101CC00068CE9042274A38BFA1F5806138BF02F53F
:101CD000806214270244B2FBF7F29200C4E91012AA
:101CE00047F6F07201689143016045EA03016269B9
:101CF00031431143A2691143E2691143226A11433E
:101D00000268114301602046FEF77EFFA068B0F52F
:101D1000804F04D10020606002E0012070476068BD
:101D200004F1480300F07F0501380ECB03280D6055
:101D3000536009D82046FEF78DFF04F154020023BA
:101D400007CA03604A6003E00020C4E91500E065AB
:101D500000200121E06384F8240084F82510F8BDF8
:101D600000040240F8FBFDBFB0B5044690F8240023
:101D7000012801D10220B0BD06F065F913D102207F
:101D800084F825000020E0632068056825F001053F
:101D900005602046FEF772FF2068226B01684AB199
:101DA00041F00E010CE0002084F824008020E06364
:101DB0000120B0BD21F004010160016841F00A0179
:101DC0000160A16C0A68D20303D50A6842F48072EC
:101DD0000A60616D19B10A6842F480720A60016894
:101DE00041F0010101600020B0BD81B00090009879
:101DF00001B00CF035BA00002DE9F84FDFF88CA1E6
:101E000005469AF80000012802D10220BDE8F88FAB
:101E10000120002489468AF800004FF47A70CAF83D
:101E20000440FFF76BF9C8BB2868594B354A0428B2
:101E30009B4607D11968901C0843186006F0FFF80C
:101E40005B4627E04FF0FF302F49C9F80000686873
:101E50008846C4000646A968084486420FD218681E
:101E6000174600EA080020431043186006F0E7F820
:101E700038B96868083401363A465B46EBE700201B
:101E800002E05B46C9F80060196840F2FA320024AB
:101E90009143196053F8141C53F8141C8AF800403D
:101EA000BDE8F88F70B5394D04462878012801D176
:101EB000022070BD01200026287020686E60A86096
:101EC00006F0BDF808B12E7070BD31490D4A0868A2
:101ED00040F0407008602068042806D100200232DB
:101EE00028610B681A430A6070BDD4E90103064CEF
:101EF000C5E904030B68234043EAC00010430860AF
:101F0000002070BD0200010005FCFEFF20480168B2
:101F100041F0004101600068C043C00F704700BF3E
:101F20002DE9F843194F04463878012802D10220E0
:101F3000BDE8F88301204FF00009984616460D468B
:101F400038704FF47A70C7F80490FFF7D7F8C8B923
:101F50000F49012C0AD1086840F0010008602E608A
:101F6000BFF36F8FC5F804800D4604E028460D4688
:101F70003146FFF7ABF84FF47A70FFF7BFF82968E6
:101F8000A143296087F80090BDE8F883BC4B00208E
:101F9000144000580648C168B1F1FF3F01DD002040
:101FA00070470449016004490160C068C00F704770
:101FB0000840005823016745AB89EFCD2DE9FC4F60
:101FC000A64A4FF0000890424FF0070208BF0222D5
:101FD000002500230092019131FA03F608BFBDE805
:101FE000FC8F012202FA03F616EA010C56D00722F2
:101FF00008F00C094FEA930E02FA09F4994AB0F17D
:10200000904F52F82E7007EA040A07D0964ADDF87E
:1020100000B0904208BF4FF0010B01E04FF0000B01
:102020000BFA09F7BA451AD18D49D1F8807027EA21
:102030000C07C1F88070D1F8847027EA0C07C1F84A
:1020400084700F6827EA0C070F604F6827EA0C07B7
:102050004F60844951F82E70A74341F82E70032138
:102060002C4601FA05F705680F213D43056008F08D
:102070001C0501FA05F56FF0030101EA5302024461
:10208000116AA943254611628168B943816041689C
:10209000B1434160C168B943C160019908F10408C6
:1020A0000235013398E700BF012818BF704780B59B
:1020B000064801210170102000210DF099FB02203B
:1020C0000021BDE880400DF093BB00BFB84B00205D
:1020D00003490A68024208BF70470860FFF7E4BF7F
:1020E0000C0800582DE9F84F5C4A5E4F4FF000098C
:1020F0004FF0010B4FF0000890424FF0070208BF6D
:102100000222002300920C6834FA03F208BFBDE8F3
:10211000F88F0BFA03F214EA020A00F098804E6876
:1021200006F0030CACF10104012C19D803248568D6
:1021300004FA08F425EA040ECD6805FA08F545EA24
:102140000E058560C6F3001505FA03FE456825EA0D
:10215000020242EA0E026FEA040E42605A000CE0EC
:10216000032202FA08F2BCF1030F6FEA020E4246A4
:1021700003D142464FF0030C1FE0C4688D6804EAA7
:102180000E0495402C43BCF1020FC46015D109F038
:102190001C040F2505FA04FC6FF0030505EA53063D
:1021A0000644356A25EA0C0C0D6905FA04F444EA84
:1021B0000C0434624E6806F0030C04680CFA02F258
:1021C00004EA0E04224316F4403F02603FD009F0B7
:1021D0000C06072202FA06F49A0857F82250A54383
:1021E000B0F1904F05D0204CA042009C08BF0124C4
:1021F00000E00024B440BC462C4347F82240184A73
:10220000174612684D6842EA0A04EE0258BF22EAF5
:102210000A043C60AE027A6842EA0A0458BF22EA25
:102220000A047C60EE03D7F8802042EA0A0458BF13
:1022300022EA0A04C7F88040AD03D7F8842042EAB6
:102240000A0458BF22EA0A04C7F88440674609F125
:10225000040908F10208013355E700BF00080048EF
:10226000000800580800014000040048426902EAE2
:102270000103914341EA0341816170471823002A19
:1022800008BF2823C150704703480078012808BFC1
:102290000CF016B800207047E418002001480068D0
:1022A000704700BF9075FF1F01480068704700BF6E
:1022B0009475FF1F01480068704700BF9875FF1FA5
:1022C00090F84120202A03D190F84020012A01D122
:1022D000022111E0242280F841200268136823F0D3
:1022E00001031360136823F48053136013681943C8
:1022F000734605F0F4FE9E460846704790F841206C
:10230000202A03D190F84020012A01D1022110E0B7
:10231000242280F841200268136823F0010313602F
:10232000136823F4706343EA0121734605F0D7FE76
:102330009E460846704790F84100704700B3B0B51C
:10234000044690F8410018B906F03AFB00F0E4F9B1
:10235000242084F84100D4E90003D4E9021205687E
:1023600023F07063012A25F001050560036183688D
:1023700023F40043836005D141F40041816009E00A
:102380000120704741F40441022A816004BF4FF4E8
:102390000061416041680F4A04F11005114341603A
:1023A000C16821F40041C1602ECD114341EA0321EF
:1023B000C160216A29430160016841F001010160A7
:1023C00000202021606484F84110206384F84200DA
:1023D000B0BD00BF008000022DE9F84305F018FFF2
:1023E00002D106F0ECF902D1022706F09EBA06F0FF
:1023F00089F98146009006F002FB0028F5D12220E1
:1024000006F00FF98848618DB1F5807F02D306F0A0
:10241000DFF801E006F0EEF82046414602F07CF9D4
:10242000089F0025FF26608D10B3204639464A4696
:1024300002F0BAF908BB05F064FFF4D10028F2D02D
:102440002046802100223B46CDF8009002F07AF928
:1024500098B906F08AF905D306F0A6FA009502F0BD
:102460005BF9E0E706F0E6F9009502F055F9DAE7E6
:102470002046394606F010FA08B10127B5E7206872
:102480002021A44B06F00EF8AFE700BF2DE9F8437A
:1024900005F0BEFE02D106F092F902D1022706F045
:1024A00044BA06F02FF98146009006F0A8FA0028F9
:1024B000F5D1212006F0B5F82148618DB1F5807F76
:1024C00002D306F085F801E006F094F82046414674
:1024D00002F022F9089F0025FF26608D10B32046E8
:1024E00039464A4602F0BDF908BB05F02CFFF4D18D
:1024F0000028F2D02046802100223B46CDF80090F3
:1025000002F020F998B906F030F905D306F04CFA3C
:10251000009502F001F9E0E706F08CF9009502F071
:10252000FBF8DAE72046394606F0B6F908B101278C
:10253000B5E720682021774B05F0B4FFAFE700BF77
:10254000002000802DE9FE4F05F062FE0CD1DDF881
:1025500030B0BBF1000F09D0DDF83480B8F1000FC6
:1025600004D006F02CF907D1022502E006F0D6F9D6
:1025700001252846BDE8FE8F06F0DAF88146009076
:1025800006F03DFA0028F4D122200E9905F09AFEBB
:10259000CDE900192046514602F072F810B184F8D6
:1025A0004050E5E7618D2048B1F5807F02D306F009
:1025B0000FF801E006F01EF82046514602F0ACF894
:1025C0000027FF262046042100224346CDF8009034
:1025D00002F0B8F80028CBD105F093FE14D198B1E1
:1025E0002046802100224346CDF8009002F0AAF850
:1025F0000028BDD106F0B9F802D306F00DF901E0CC
:1026000006F0F3F802F088F8608D0028DAD1204651
:10261000414606F041F90028AAD1206820213D4B0F
:1026200005F065FFA5E700BF002400802DE9FE4FFF
:1026300005F0EEFD0CD1DDF830B0BBF1000F09D094
:10264000DDF83480B8F1000F04D006F0B8F807D1F7
:10265000022502E006F062F901252846BDE8FE8F5A
:1026600006F066F88146009006F0C9F90028F4D11A
:1026700021200E9905F026FECDE90019204651468D
:1026800002F022F810B184F84050E5E706F06DF84A
:1026900005D3FF20514606F00EF9204608E0608D74
:1026A00000214FF0007320850091C2B220465146B0
:1026B00002F032F80027FF26204641464A4602F043
:1026C000D0F80028C8D105F03EFE14D198B12046BC
:1026D000802100224346CDF8009002F033F8002814
:1026E000BAD106F042F802D306F096F801E006F0FF
:1026F0007CF802F011F8608D0028DDD120464146BB
:1027000006F0CAF80028A7D120682021014B05F067
:10271000EEFEA2E700E800FEF0B593B004460EA876
:102720001421FDF7BFFE68463821FDF7BBFE206887
:10273000324988422AD0324988425DD14FF4403034
:10274000402605906846009600F028F908B1FEF78B
:10275000D7FB022002F0CCF8022002F0C9F80420D6
:10276000002501271224129011951097CDE90E64CF
:10277000244E0EA93046FFF7B5FC80201195CDE917
:102780000F471E241F254FF400171BE04FF4402075
:10279000069080200090684600F000F908B1FEF72E
:1027A000AFFB0120012402F0A3F8002021254FF403
:1027B00080074FF09046CDE91040122020240F9062
:1027C0004FF4C0500E90042012900EA93046FFF72F
:1027D00089FC384602F0A6F828460121002200F0C4
:1027E00049F8284600F038F820460221002200F07F
:1027F00041F8204600F030F813B0F0BD005800401A
:10280000005400400004004880B5032000F04EF85A
:1028100000F04CFA3A4908600F2000F007F808B1C0
:10282000012080BD00F004F8002080BD002070472A
:102830007047000000280CD400F01F01012240095D
:1028400002FA01F1034A42F82010BFF34F8FBFF3A1
:102850006F8F704780E100E0002808D400F01F016E
:102860000122400902FA01F1014A42F820107047A2
:1028700000E100E070B5134B4FF0FF351B68C3F368
:102880000223DC1E83F0070338BF002405FA04F698
:10289000B243042B28BF042305FA03F39943A14054
:1028A0001143BDE870400DF0CDB800BF05494FF6AB
:1028B000FF030A681A4060F30A22034810430860C5
:1028C000704700BF0CED00E00000FA0521483222FD
:1028D000016821F480410160F24909685143094AC5
:1028E000B1FBF2F14A1E43698A4203D213F400712C
:1028F0001146F7D140690321800501EAE070704775
:102900004401002040420F001248016841F4804118
:10291000016070470F49022301280A6863F302022D
:102920000A601D490A6842F004020A600FBF30BF06
:1029300040BF20BF20BF05F08DBB00BF0548006829
:1029400000F4C060704700BF0248016841F4807124
:10295000016070470004005810B50C460D49096825
:1029600001F4007118B139B9FFF7CEFF04E019B1D5
:10297000FFF7ACFF00B110BD0748012C016821F042
:102980000401016004BF30BF10BD40BF20BF20BFA5
:1029900010BD00BF1404005810ED00E0F8B5044667
:1029A0008078544EC00742D0FFF7CEFFFFF76CFC93
:1029B0000546D6F8F403C00506D4FFF765FC401BB6
:1029C0000228F6D9032533E0606BD6F8841001F4B1
:1029D0004071814224D0D6F88410D6F8842042F485
:1029E0008032C6F88420D6F8842022F48032C6F8DB
:1029F000842021F4407289070146C6F884200FD54F
:102A0000FFF742FC054641F28837D6F8840080077C
:102A100005D4FFF739FC401BB842F6D9D2E7616B09
:102A2000D6F8840020F440700843C6F884000025DE
:102A30002068C10702D0616805F01EFE810702D53B
:102A4000A16805F019FE810605D52169F26F22F40F
:102A500040621143F167810502D5216A05F0E5FA6C
:102A6000410502D5616A05F0E0FA010502D5A16AC7
:102A700005F0DBFA410603D5606901F061FF2068CB
:102A8000010603D5A06901F05BFF2068C10503D5ED
:102A9000E06901F055FF2068C1060CD5E168F26FCE
:102AA00022F440720A43B1F5807FF26703D13168A6
:102AB00041F08071316001040AD5216BF26F22F080
:102AC00040420A43F26719B9316841F080713160C0
:102AD00040040CD5E06AF16F21F040510143B0F1A0
:102AE000005FF16703D1306840F4803030602846E1
:102AF000F8BD00BF0C0000582DE9F843002800F095
:102B00009F80674F05460C46386800F007008842F2
:102B100011D2386820F00700204305F0AAFD0646D0
:102B2000386800F00700A04205D0FFF7ADFB801B1E
:102B30000228F5D956E02868B946704F810711D5AB
:102B4000A868396821F0F001084305F092FD0646B7
:102B50003868C00305D4FFF797FB801B0228F7D91C
:102B600040E02868410616D56869D7F8001121F0C1
:102B70000F0141EA1010C7F80001FFF785FB064678
:102B8000D7F80001C00305D4FFF77EFB801B0228A5
:102B9000F6D927E02868410711D5E868396821F49B
:102BA000E061084305F065FD06463868800305D4FA
:102BB000FFF76AFB801B0228F7D913E0286801079A
:102BC00014D52869396821F4605141EAC00005F044
:102BD00050FD06463868400307D4FFF755FB801BBD
:102BE0000228F7D90320BDE8F8832868C0071CD164
:102BF000D9F8000000F00700A04224D9D9F800005D
:102C000020F007002043C9F80000FFF73DFB054610
:102C10004846D9F8000000F00700A04213D0FFF7A3
:102C200033FB05F098FCF3D930E068684FF0B04111
:102C300098B103282CD002282ED1096889030FD41B
:102C40000120BDE8F88300F031F816490860164805
:102C50000068BDE8F843FFF7E9BD09688907EFD5CB
:102C6000396821F00301084305F003FD064641F2EF
:102C700088386868396801F00C01B1EB800FB7D073
:102C8000FFF702FB811B03204145F2D9BDE8F88321
:102C900009688901D4D5E3E709684905D0D5DFE79C
:102CA00000400058440100204C00002080B500F096
:102CB00029F812493C22096802EA9101024A515856
:102CC000B0FBF1F080BD00BFD027010880B5FFF751
:102CD000EDFF0A490A4A0968C1F3022152F821109E
:102CE000C84080BD80B5FFF7E1FF0449044A096888
:102CF000C1F3C22152F82110C84080BD080000581D
:102D00001028010810B5364951F8042C086812F053
:102D10000C0205D00C2A15D100F00300012811D1B6
:102D20004FF0B0400368006800F008001B0705D4AE
:102D3000B8B9D1F88800C0F303201CE0B0B9D1F8CD
:102D4000880011E02748042A1ED0082A1BD14FF022
:102D5000B0421268D2025CBF44F60000C0F2E81034
:102D600012E04FF0B0400068002004E04FF0B040A7
:102D70000068C0F303101C4B002A53F8203018469B
:102D800018BF002001E00020002351F8042C02F0BD
:102D90000C020C2A22D1086800F003021148022A12
:102DA0000CD0032A09D14FF0B0421268D2025CBFA6
:102DB00044F60000C0F2E81000E018460A680B680C
:102DC00009680124C2F3062204EB51715043C3F396
:102DD00002120132B0FBF2F0B0FBF1F010BD00BF07
:102DE0000C0000580024F4000C2901082DE9F047DC
:102DF000002800F05981DE4C8246606800F00C0823
:102E0000A06800F003099AF80000800627D49AF819
:102E10000000C00770D0B8F1080F63D0B8F10C0FF4
:102E200008BFB9F1030F5DD04FF0B041DAE90102FC
:102E30000B6823F480131A43B0F5803F0A6009D071
:102E4000B0F5041F40F096814FF0B040026842F4A4
:102E500000120260086840F48030086097E1B8F121
:102E6000000F1DD0B8F10C0F08BFB9F1010F17D03A
:102E70004FF0B0463068DAF82010002900F03481B5
:102E800040F0010005F082F905463068800700F146
:102E90003A81FFF7F9F905F05EFBF6D9BDE8F08756
:102EA0004FF0B0410868800704D5DAF82000002808
:102EB00000F0FA80DAF828000968090747BF4FF0E8
:102EC000B0410968D4F89010090901F0F001884276
:102ED00040F2D48006F0E2FE002840F0E58005F0E4
:102EE00090F8E4E04FF0B0400068800304D5DAF8D1
:102EF0000400002800F0D8809AF80000800730D540
:102F0000B8F1040F1BD0B8F10C0F08BFB9F1020FD4
:102F100015D04FF0B0463068DAF81010002900F0F4
:102F2000468140F4807005F031F90546306840056F
:102F30000FD4FFF7A9F905F00EFBF7D9AEE74FF074
:102F4000B0400068400504D5DAF81000002800F011
:102F5000AB80DAF81400216821F0FE4141EA0060FC
:102F600020609AF8000000072CD49AF8000040076F
:102F70004FD4DAF82C0010B3B8F10C0F40F0C68033
:102F8000012800F09180DAF83010A06800F0030208
:102F90008A4240F08980DAF8341000F070028A42E8
:102FA00040F08280DAF8381000F4FE42B2EB012FD4
:102FB0007AD1DAF8441000F06040884274D10020E1
:102FC000BDE8F087D4F89010DAF8180000287AD01D
:102FD000DAF81C0001F01002904200F08D8101F03F
:102FE0000302022A60D0C90700F07F81D4F8900064
:102FF00020F0010005F0CCFB0546D4F890008007D6
:1030000040F17181FFF740F9411B03201129F4D9E8
:1030100044E7D4F8FC03C0050ED4FFF795FCFFF796
:1030200033F90546D4F8FC03C00505D4FFF72CF9A5
:1030300005F091FAF6D931E7DAF80C00002800F033
:10304000C580852801D0052805D1D4F88C0040F032
:103050000400C4F88C00FFF717F905F0C0F940F040
:103060000100C4F88C00D4F88C00800764D4FFF70A
:103070000BF9411B0320B142F5D90FE74FF0B041E6
:103080000A6842F008020A600A6822F0F00202436D
:103090000A60DAF82410226822F47F4242EA012111
:1030A000216006F0FBFD10B10120BDE8F087FFF7BD
:1030B000FDFD9B4908609B480068FFF7B7FB0028AF
:1030C0007FF4ECAEA3E621F0010005F061FB0546BC
:1030D000D4F8900080077FF548AFFFF7D5F8411B83
:1030E00003201129F4D9D9E620F0010005F04EF8AB
:1030F0000546306880077FF58AAEFFF7C5F805F012
:103100002AFAF6D9CAE604F07CFF80E64FF0B04612
:103110000228316821F08071316071D1FFF7B4F875
:1031200005463068800140F18180FFF7ADF8411B12
:1031300003200A29F5D9B1E6DAF80C0040F00400C2
:10314000852840F09980FFF79FF805F048F940F096
:103150008000C4F88C00D4F88C0000053FF509AF5E
:10316000FFF792F8411B0320B142F4D996E600BF65
:10317000040000584FF0B0460028316821F4803137
:103180003160316821F40011316000F09E80FFF75A
:103190007BF805464FF0B046306880033FF5ACAE93
:1031A000FFF772F8411B03206429F5D976E620F475
:1031B000807004F0EBFF0546306840057FF5D1AE26
:1031C000FFF762F805F0C7F9F6D967E6FFF75CF894
:1031D0000646D4F88C0041F2883920F08000C4F80B
:1031E0008C00D4F88C0027460405FFF74DF80546FF
:1031F000002C55D5A91B03203C464945F1D94DE685
:10320000A068494920F00300A060A0680840A060C1
:10321000FFF73AF80446306880017FF5D0AEFFF73B
:1032200033F8011B03200A29F5D937E6A0683F4986
:103230000AF130070840EECF0843104340EA03206C
:1032400028434FF0B04530433843A060286840F031
:1032500080702860A06840F08050A060FFF714F8EC
:103260000446286880013FF5AAAEFFF70DF8011B60
:1032700003200A29F5D911E6FFF706F805F0AFF8A3
:1032800020F08000C4F88C00D4F88C0000057FF595
:1032900070AEFEF7F9FF411B0320B142F4D9FDE502
:1032A000D7F88C003C4641F2883620F00100C7F880
:1032B0008C00D4F88C0080077FF55BAEFEF7E4FF4E
:1032C000411B0320B142F4D9E8E5FEF7DDFF0546D6
:1032D000306880037FF510AEFEF7D6FF411B032058
:1032E0006429F5D9DAE5DAF81C00D4F8901021F059
:1032F00010010843C4F89000D4F8900040F0010099
:1033000005F046FA0546D4F8900080073FF52DAE4B
:10331000FEF7BAFF401B1128F5D90320BDE8F0875E
:10332000440100204C000020FFFFFEEE8C80C11104
:1033300070470000034850F821007047014840F8EA
:103340002120704700B1004090F82C200221012A72
:103350000DD080F82D10C049734604F08CFF9E46B6
:1033600042F020020A60734604F090FE9E46084632
:10337000704700BF80B50AF049FF0130BDE88040CA
:103380000AF050BF10B5044621480168490604D52B
:10339000402181602046FFF7EDFF012084F82D00D9
:1033A00010BD00BF90F82C200221012A12D080F815
:1033B0002D10A949734604F05EFF9E4642F080023C
:1033C0000A60A74A136843F480231360734604F02D
:1033D0005DFE9E46084670470CF052BA70B50C4D23
:1033E00004462868216B01EA0006F00704D001209A
:1033F000A8602046FFF7F0FFB00704D50220A860C0
:103400002046FFF795FF012084F82D0070BD00BF16
:1034100054280040B0B590F82C300222012B2ED059
:103420008D4BCA2480F82D20DC605324DC606FF4BF
:103430000854B1F5807F08BF6FF488541D682C4094
:103440001C603424B1F5807F08BF2C24E55825F09A
:103450000045E55008BF01225A64FF22DA600022CD
:10346000012380F82C2080F82D306FF00203B1F595
:10347000807F08BF6FF00103016B194001631046A4
:10348000B0BD00BF70B590B3044690F82D0028B9C8
:10349000002084F82C00204600F03EF802207C4DED
:1034A00084F82D00CA20A8615320A861204606F0A8
:1034B00077FCC8B9E8681749261D0840E8604ECE79
:1034C000A06931430843E9680843E86043EA0240E1
:1034D0006860D4E909012A6822F4F85210430843CD
:1034E000286004F0C5FE20B1FF21A96170BD012054
:1034F00070BD6069D4E90712EB6823F060431A439A
:1035000011430843E860FF20A861012084F82D00E2
:10351000002070BDBFFF8FFB10B590B0044601A81E
:103520003821FCF7BFFF20681749884229D14FF4A2
:1035300080700E904FF48030019001A8FFF72EFAB2
:1035400008B1FDF7DDFC11480022816B41F4004118
:103550008163016841F4806101600021006800F42A
:1035600080600F900F980220FFF784F90220FFF788
:1035700073F92A2000210022FFF77CF92A20FFF7A7
:103580006BF910B010BD00BF002800405800005873
:103590002DE9F84F04F0FDFD5CD084F82D000120EA
:1035A0002D4F05F0F9F801D1002029E072B16869CA
:1035B000B0F1803F07D0B0F5000F04D0396849065C
:1035C00001D40021E97004F04FFD19E0386840068D
:1035D00002D40026EE7001E0E87886052878DFF84E
:1035E0007CB0D5F814A0D84780466878D84705F055
:1035F000F5F905F033F9296A41EA080141EA00606A
:1036000005F041F80ED105F0A7F919BFB862A86915
:10361000D5E906010843F86268680121B8654FF4EE
:1036200088500DE005F056F919BF3863A869D5E94F
:1036300006010843786368680221F8654FF4085072
:103640003A68104338600648026842F4003202606B
:1036500004F0D0FEBDE8F88F182800407D9D0008DA
:1036600080080058B0B50A4D286820F02000286076
:10367000FEF70AFE04462868800607D4FEF704FE1B
:10368000001BB0F57A7FF6D90320B0BD0020B0BD95
:103690000C280040014804F0A8BE00BF10E000E084
:1036A000012904D041B9CF48816880200847CD481E
:1036B00081684FF480700847704700BFC94881682F
:1036C000402008472DE9F04105F00CF902D160795E
:1036D000012802D10220BDE8F08104F0E0FCED49B0
:1036E00005F042F9394609F0A5F9204600210027E6
:1036F00009F0A0F9AF4204D205F0B7F8013701365E
:10370000F8E704F0C9FF724604F080FE964618BF41
:103710000120BDE8F08100BF2DE9F04105F0E2F89D
:1037200002D16079012802D10220BDE8F081012593
:1037300020461E4617468846657109F0A9F948F0EB
:1037400010004146942818BF00252571D14D2868E6
:1037500020F400402860204609F06CF936B117F8D3
:10376000011B204609F066F9013EF7E72868B8F129
:10377000840F40F40040286002D0204609F0ACF9E4
:10378000724604F043FE964618BF0120BDE8F08162
:103790009448816820200847924881681020084793
:1037A0007CB5044600200DF1060212210223ADF87B
:1037B00006002046FFF786FF9DF807609DF806503B
:1037C000F00702D0204600F009F9B00702D52046E4
:1037D00000F0F6F8700702D5204600F091F83007A7
:1037E00002D5204600F0F6F8F00602D52046FFF795
:1037F000D3FFB00602D52046FFF7CAFF700602D5F8
:103800002046FFF75BFF300604D505F00101204696
:10381000FFF746FFA80702D5204600F0D5F80DF1C6
:103820000602204602210223FFF776FF7CBD00003E
:10383000BCB510B30446807920B9002060712046E1
:1038400000F046F802201E4A6423A0711D488158EA
:1038500021F4004181501C490968C1EBC101C1F349
:103860004C4159430191019949B1019B013B01939D
:1038700083585B04F7D4002503E001251DE00125F2
:10388000A560D0F8882042F40042C0F888200F4A92
:10389000136843F480531360026842F400620260CC
:1038A0004FF40062026131B1206809F083F8002012
:1038B000A060012020710120A0712846BCBD00BF7E
:1038C0008CFCFFFF080400584401002090080058B9
:1038D000E0B50A480022016841F0010101600021C1
:1038E000006800F00100019001983220FEF7C2FF4D
:1038F0003220BDE88C40FEF7AFBF00BF6400005827
:1039000038488168042008472DE9F84304F0EAFFAD
:1039100002D16079012802D10220BDE8F88304F0C9
:10392000BEFB5C49DFF8708104F01EFE1E21C0471B
:1039300020463946C047204600210027C047AF42F5
:1039400004D204F092FF01370136F8E704F028FCB6
:10395000724604F05BFD964618BF0120BDE8F8836F
:103960002DE9F84304F0BEFF02D16079012802D1AD
:103970000220BDE8F88304F092FB4649DFF8188185
:1039800004F0F2FD1D21C047390A2046C047F9B2B4
:103990002046C047204600210027C047AF4204D23E
:1039A00004F063FF01370136F8E704F0F9FB7246D3
:1039B00004F02CFD964618BF0120BDE8F88300BF37
:1039C0000848816802200847064881684FF4007063
:1039D000084700BF034881680820084701488168FC
:1039E00001200847780200202DE9F04104F07AFF19
:1039F00002D16079012802D10220BDE8F08104F0F3
:103A00004EFB244904F0B0FF0E2109F013F82046C4
:103A1000394609F00FF81DB104F0E6FF013DFAE761
:103A200004F03AFE724604F0F1FC964618BF0120FD
:103A3000BDE8F0812DE9F84304F054FF1ED10F4694
:103A400061790220012922D0A07101201D4616466D
:103A50006071204609F01CF80E49DFF83C8004F044
:103A600083FD0D21C047390A2046C047F9B22046E0
:103A7000C04735B104F0B8FF013DFAE70220BDE8C8
:103A8000F88304F08DFB04F0C1FC18BF0120BDE8F1
:103A9000F88300BF9004005835CA0008014804F0BC
:103AA000DEBA00BF10E000E07047704770470000CA
:103AB00070B590F83C300222012B23D080F83D20D5
:103AC0000122334C80F83C20026855689368A2427A
:103AD00003D14E6825F4700535430E6825F0700556
:103AE0003543A242556002D0B2F1804F04D18968BB
:103AF00023F08003194391600022012180F83C20CB
:103B000080F83D10104670BD58B110B504F079FE34
:103B100003D104F0FBFC00F006F804F02CFF04F0E5
:103B200048BB0120704780B50068B0F1804F18BFD6
:103B300080BD012000F0F6FE1B2003210022FEF7CD
:103B400099FE1B20BDE88040FEF786BE90F83D1030
:103B5000012918D1022180F83D100168C86840F0A1
:103B60000100C8600A48814202D0B1F1804F0CD1F7
:103B70008868084A734604F0F4FD9E4602D0B2F508
:103B8000803F02D170470120704704F04DBE00BF56
:103B9000002C014007000100016841F21113CA68BE
:103BA00022F00102CA600A6A1A4208D10A6A40F287
:103BB00044431A4203D10A6822F001020A6004F069
:103BC00075BE000010B504F0C6FD4ED084F83D006F
:103BD0000120274B84F83C00206882681A408260EC
:103BE0000A68C2B1102A16D0202A14D0302A12D066
:103BF000402A17D0502A1DD0602A23D0B2F5005F8A
:103C00002BD0B2F5805F2DD0702A2FD104F05AFC52
:103C100041F0770125E08168164B1940114341F0CE
:103C200007011EE004F084FE2068124A81681140FA
:103C3000473116E004F07CFE20680E4A816811408E
:103C400057310EE04B68CA6819460AF0E4FB206859
:103C5000084A81681140673103E004F033FC41F405
:103C600080418160002004F01AFE10BD0120FAE7B7
:103C70008800CEFF88FFCFFF704710B5044600686C
:103C80000169890714D5C168890711D56FF0020150
:103C90000161012121778069800702D004F0F6FDDF
:103CA00003E004F03FFE04F0F4FD002020772068DC
:103CB0000169490715D5C168490712D56FF004019C
:103CC000016102212177806910F4407F02D004F065
:103CD000DDFD03E004F026FE04F0DBFD002020778C
:103CE00020680169090714D5C168090711D56FF06B
:103CF0000801016104212177C069800702D004F026
:103D0000C5FD03E004F00EFE04F0C3FD00202077A3
:103D100020680169C90615D5C168C90612D56FF0BA
:103D20001001016108212177C06910F4407F02D0A1
:103D300004F0ACFD03E004F0F5FD04F0AAFD002062
:103D4000207720680169C90709D0C168C90706D072
:103D50006FF001010161204600F03AF82068016926
:103D6000090609D5C168090606D56FF08001016111
:103D70002046FFF79AFE20680169C90509D5C16888
:103D8000090606D56FF4807101612046FFF78CFEAD
:103D900020680169490609D5C168490606D56FF052
:103DA00040010161204600F019F820680169890688
:103DB00002D5C168890600D410BD6FF020010161F1
:103DC0002046BDE81040FFF771BE70477047000005
:103DD000014801210180704748190020704710B543
:103DE00004F0CDFB01D1022010BD2420C4F88400D2
:103DF00020680168026822F0010241F0005102606F
:103E0000012284F880204FF0005262660160204653
:103E10000AF0F8FC0020202184F88000C4F8841007
:103E200010BD90F88010012901D102210FE001217D
:103E300080F88010016851E8001F026841F002011B
:103E400042E80013002BF5D1002180F880100846CD
:103E5000704770477047B0B504F091FB01D1022064
:103E6000B0BD04F02EF922F0606204F028FC04F0EA
:103E7000C6B9B0B504F083FB01D10220B0BD04F097
:103E800020F922F0604204F01AFC04F0B8B9BCB585
:103E900004F075FB01D10220BCBD2420C4F88400CD
:103EA0002068036823F001030360012384F8803055
:103EB000836823F440130B43836059B9436891B27C
:103EC00023F0100319434160C2F30741426861F3D4
:103ED0001F624260016841F001010160FEF7D4F900
:103EE00003466FF07E404FF48001002200250090D1
:103EF00020460BF0C3F808B1032003E02020C4F8EB
:103F00008400002084F88050BCBD70477047704723
:103F100070B50446006840F60F05C2690168836801
:103F20002A426BD0A54D01EA0506A54D1D40761924
:103F30006ED0D60709D0CE0507D501260662D4F883
:103F40008C6046F00106C4F88C60960709D5DE0740
:103F500007D002260662D4F88C6046F00406C4F846
:103F60008C60560709D5DE0707D004260662D4F810
:103F70008C6046F00206C4F88C6016070BD501F081
:103F80002006354307D008250562D4F88C5045F04B
:103F90000805C4F88C5015050AD54D0108D54FF415
:103FA00000650562D4F88C5045F02005C4F88C50AB
:103FB000D4F88C50002D6ED092060AD501F0200165
:103FC00003F08052891804D0216F11B12046884730
:103FD0002068D4F88C10806801F0280100F04000BF
:103FE000401852D020460AF007FD20688168490633
:103FF0005DD504F012FA4FD02068FAE7950607D590
:1040000001F0200503F08056AD1901D0216F13E0B7
:10401000E56E012D03D1D50601D5CD064CD4D502D0
:1040200001D55D0229D415060BD501F0800503F4F6
:1040300000035B1905D0616F69B32046BDE870408D
:104040000847530601D54B060DD4100201D5480090
:1040500057D4D0011FD5B1F1FF3F1CDC2046BDE88D
:104060007040FFF7F7BE50E8000F216820F04000D5
:1040700004F0A1FB3BD02068F5E74FF4801101620A
:104080002046BDE87040FFF741BF2046FFF73FFFE5
:104090000020C4F88C0070BDE06F40B149498163D5
:1040A000FDF726FD0028F6D0E06F816BC6E72046BD
:1040B000BDE87040FFF72BBF1021016281684906FF
:1040C00024D4B4F85E10B4F85C20B4F85E30002B51
:1040D000E1D0511A0A04DED050E8000F226820F423
:1040E000907042E80003002B48D02068F4E70020DD
:1040F00060672020C4F884002046BDE8704000F0CE
:104100008BB92046BDE87040FFF7FFBEE16F0A683B
:1041100053689DB2002DBED0B4F85C108D42BAD267
:10412000A4F85E301268920623D450E8000F21688C
:1041300020F4807004F03FFB01D02068F5E7206890
:1041400050E8020F216820F0010004F014FAF6D1C3
:10415000206804F062F9FBD12020C4F88800002018
:10416000E06603F0A4FFFCD1E06FFDF789FCB4F832
:104170005C10B4F85E00081A81B21AE01248226896
:1041800052E8022F2368024043E80225002DF6D1B1
:104190002020C4F8880000202067E066206850E8EE
:1041A000000F226820F0100042E80003002BF5D138
:1041B00089B22046BDE87040FFF74BBE20010004E5
:1041C0000100001055E90008FEFFFFEF10B548B1EF
:1041D0000446D0F8840008B904F00BFC04F004F89D
:1041E000012801D1012010BDA06A08B104F016FA1F
:1041F00004F0F9F921F02A01816004F052F8BDE8D9
:1042000010400AF075BB000010B5044600688749ED
:10421000884218BF10BD0948016821F400310160CF
:104220004FF090400C21FDF7C9FEA06FFDF796FC02
:104230002520BDE81040FEF7FDBA00BF5800005829
:1042400070B594B004460EA81421FCF72BF968460B
:104250003821FCF727F920687449884248D125485D
:104260000225009502906846FEF798FB08B1FCF71E
:1042700047FE21480026C16841F40031C160C16891
:1042800001F4003113911399016841F001010160BB
:10429000006800F001001390072012900320119095
:1042A0000C20CDE90F560E9013980EA94FF09040B8
:1042B000FDF718FF114D124B142280201021C5E983
:1042C0000032C5E90216C5E904062846C5E90666B6
:1042D0002E62FDF7E9FC08B1FCF712FE2520022151
:1042E0000022AC62A567FEF7C5FA2520FEF7B4FAF6
:1042F00014B070BD04000C004C000058DC490020D4
:1043000058000240B0B5D0F88830202B05D131B12B
:104310002AB190F88030012B03D10220B0BD0120DA
:10432000B0BD0023074C04F0F9F802D05C68240209
:1043300003D40AF023FE0020B0BD04F013F8F8D037
:104340000368FAE70080004010B50446006837496A
:10435000884218BF10BD0848436833B1D4F88C00B8
:1043600018B9054801210022984703492046012237
:10437000BDE81040FFF7C6BFB0010020F8B5044605
:10438000D0F88400202806D161B3134652B394F8C4
:104390008000012801D10220F8BD00250120A4F8E9
:1043A0005630C4F88C5084F880002120A4F8543092
:1043B0002165C4F88400A06FB0B1144A144E154FA3
:1043C000C0E90B76C0E90D2522682832FDF7CCFC48
:1043D00050B11020C4F88C00002084F88000202008
:1043E000C4F884000120F8BD2068402184F8805082
:1043F000016250E8020F216840F0800004F0BBF831
:1044000001D02068F5E70020F8BD00BF65E900088D
:10441000F3E90008BBE9000800680449884218BFB6
:104420007047034801680020084700BF004400406F
:104430005019002070470000F8B52F4F05460C4674
:1044400097F80401022802D02C48C06A804700F087
:10445000E5FF064628B1022000F0F5FF002000F03D
:10446000D6FF97F80401012813D100F0DDFF30B129
:10447000002000F0EBFF002000F0E0FF012600F03C
:10448000D1FF30B1002000F0DFFF002000F0D2FFAC
:1044900028E03EBB1A4E96F8841496F8140451B1E5
:1044A00008B186F83944204601F084F997F80401F0
:1044B000022811D116E008B186F83954284601F0D7
:1044C00079F9F86A0BF0CCF9D6F8B413884209D31D
:1044D00006F566700BF068FA96F8850440F0200047
:1044E00086F8850497F804010549022818BF0620BC
:1044F00081F88404F8BD00BF288700204C290108FA
:10450000D0120020FEE700688169890701D50021EB
:1045100081628169C90703D1816941F0010181612B
:10452000704700002DE9F047044600688A460027DE
:104530008169C90601D4002146E0102190460AF1A4
:1045400001064FF020090025C161816901F02001B9
:10455000294334D10025002EF7D0FDF795FEA0EBBE
:1045600008012068514503D80025BAF1000FECD1AD
:10457000436894F8421082695B0409D412F4004243
:1045800006D0202904D004F0DFF9FDF77DFE804637
:104590000025206881698906D7D4FDF775FEA0EB58
:1045A00008001A28F5D3606C012540F020006064F3
:1045B00084F8419084F8407084F84270E9E70DB9BE
:1045C0002021C161012104278269D30505D54FF45B
:1045D000807147F00107C1610121530505D492059F
:1045E00009D469B90020BDE8F0874FF4806108372D
:1045F000C161910504D54FF4007147F00207C16114
:1046000004F021F82068884A416811404160606CDC
:104610003843714603F0BEFE8E460120BDE8F087A8
:1046200010B586B00446642006210DF11202012364
:10463000CDE9002102900E48A6213222FDF782FF2B
:10464000BDF812000DF04EFE0A4941F82400BDF8F5
:1046500014000DF047FE084941F82400BDF816008B
:104660000DF040FE054941F8240006B010BD00BF22
:104670003C4A00206C1900206C2100206C2900208D
:104680002DE9FC410446234815461E46DAB20023B4
:10469000009003F052FEDDE9088704F08CF910B1B8
:1046A0000120BDE8FC81012E03D004F033F800287E
:1046B000F6D104F042F94021009700F043F80028B9
:1046C00018BF0120BDE8FC812DE9FC4104461148DA
:1046D00015461E46DAB24FF08073009003F02DFEAF
:1046E000DDE9088704F067F910B10120BDE8FC811D
:1046F000012E03D004F00EF80028F6D104F01DF9C5
:104700008021009700F01EF8002818BF0120BDE8A6
:10471000FC8100BF0020008070B500686FF39F210E
:10472000049D074E1943446841EA0241294324EAA3
:10473000555421F0004134402143416070BD00BF19
:10474000009C00FC2DE9F843DDF820801D4616464C
:104750000F4681465C1CD9F8000080693840C01BB8
:10476000B0FA80F04009B0421AD1002CF3D0FDF726
:104770008BFDA0EB0800A84201D8002DEBD1D9F8A1
:10478000440040F02000C9F84400202089F841008E
:10479000002089F8400089F842000120BDE8F88334
:1047A0000020BDE8F883000070B515460E460446AB
:1047B0002068806940071DD403F0C2FF90BB2068C9
:1047C0008169890611D4FDF75FFD401BB04201D815
:1047D000002EEDD1606C40F020006064002084F871
:1047E0004000202084F841001CE08169490703D57E
:1047F000218D09B1002070BD81690022C9064FF0EA
:10480000000102D51022C261042262642022064DFA
:10481000C26143682B40436084F8412084F8401013
:1048200084F84210012070BD00E800FE70B5154606
:104830000E46044620688069800610D403F080FF8D
:1048400058B9FDF721FD401BB04201D8002EF1D12F
:10485000606C40F0200003F09DFD012070BD002041
:1048600070BDF8B515460E4604464F1C2068806999
:10487000800712D403F064FF68B9002FF6D0FDF76B
:1048800003FD401BB04201D8002EEFD1606C40F018
:10489000200003F07FFD0120F8BD0020F8BD0000DE
:1048A00081B005490A6802430A600968084000901F
:1048B000009801B0704700BF4800005881B0184907
:1048C0000A6802430A60096808400090009801B035
:1048D000704700BF81B01248016841F002010160D9
:1048E000006800F002000090009801B0704700BF1F
:1048F00081B00B490A6802430A60096808400090C9
:10490000009801B0704700BF81B005490A680243B2
:104910000A60096808400090009801B0704700BF25
:104920004C00005881B005490A6802430A600968D2
:1049300008400090009801B0704700BF5800005830
:10494000064A6FF47F2161EA101100F47F4013687A
:10495000194041EA00101060704700BF88000058FD
:104960002DE9F04190B0724D0146142205F130005E
:104970000AF0AEFE03F098F895F830204068D04079
:10498000C00708D005F10C0005F11C0101F032FA56
:1049900040B1FF26C8E0734B0020002101220AF03D
:1049A000C9FDFEE726208DF81C0007A801F018FEBF
:1049B000F0B127208DF81C006868006940B107A895
:1049C00001F058FD68684FF4E56102690898904766
:1049D00026208DF81C0007A801F002FE58B901201E
:1049E0008DF81C0007A801F045FD9DF8200010B1CE
:1049F0000120287001E0287800B36868C16909B116
:104A00000020884706208DF81C0007AC03F060FEEC
:104A100048480899016326208DF81C0003F058FED1
:104A2000089890F8401090F8042190F8060185F855
:104A3000301085F8312085F8320014E0002008900D
:104A400005208DF81C0007AC204601F0C9FD686800
:104A5000C068804737490890086306208DF81C001D
:104A6000204601F0BDFD02208DF81C0007AC03F0CC
:104A70002FFE304E0899082206F11C000CF0EDFBC9
:104A800003208DF81C0003F023FE089906F1240092
:104A900008220CF0E2FB08F025FF96F8300096F8AB
:104AA000311096F8322096F833300026CDE90032E6
:104AB000CDE9021020A30220002100220AF03AFDD5
:104AC0000120924F4FF00F088DF8200020468DF8FE
:104AD0001C80B84710208DF820608DF81C002046FF
:104AE000B84704208DF81C0095F832008DF820009E
:104AF0002046B84737208DF81C00286C08902046C7
:104B0000B84795F830008DF8148005A907F01CFB14
:104B1000002818BF012085F83600142000F06EFA36
:104B200095F8360002F088FE70B210B0BDE8F08152
:104B3000F0020020500000202323232323232044BD
:104B40006576416464723A20202020202530325856
:104B50003A253032583A253032583A253032580DFD
:104B60000A00000074860108FEB50A208DF80400D2
:104B700001A801F055FFE649059A00288A6018BF90
:104B80004FF0FF3006B080BD10B58AB038B1044692
:104B900000208DF8040001A801F06CFC08B1FF2092
:104BA00003E09DF808002070002040B20AB010BD5C
:104BB000D7488068704700BF10B58AB038B1044646
:104BC0001F208DF8040001A801F054FC08B1FF205B
:104BD00006E09DF80800CE49207081F834000020DE
:104BE00040B20AB010BD00BF21B1012804D028B9DD
:104BF000474802E0FF2002E002480860002040B27F
:104C0000704700BF0300010180B501F065F800287E
:104C100018BF6FF0010080BD80B5F7490D4A836968
:104C20008A610D4A4860CB624A610C4A0A610C4AAB
:104C3000CA600C4A8A6282684A62D0E90020C1E9EF
:104C400007200949002000F0ADF8002818BF4FF0F8
:104C5000FF3080BD217F0008957E0008097E000896
:104C6000D17D0008917F00083401002070B58EB01E
:104C7000E14D012302288DF8243095F834208DF879
:104C800029200BD1DB48C171022181718DF82810D8
:104C900002F0B8FD09A801F0C3FE35E0D5488DF853
:104CA0002830C1714FF480710271A0F80510287886
:104CB000C0B91E206C46154E8DF804208DF80000FA
:104CC0002046B0471F208DF8000095F834008DF87D
:104CD00004002046B0470E48019028208DF80000BF
:104CE0002046B04702F08EFD01208DF804008DF8BB
:104CF0000000684601F074FC6868416ABD48884756
:104D000095F8310000F0BEF80EB070BDE165000806
:104D10000003000180B58AB001208DF8040001A8CD
:104D200001F0A8FB9DF80810B0FA80F0002918BF28
:104D30000121400908400AB080BD0000B0B58AB02A
:104D4000FFF762FF044650BB03F028F9811C15D021
:104D500090B9A94C6068406970B126208DF80400B4
:104D600001A801F087FB60684FF4E5614269029891
:104D700090470025002403E0FF2400E0F8240125EB
:104D800003F01AF9002818BF4FF0FF343DB930B9CD
:104D900099484068C16909B101208847002460B280
:104DA0000AB0B0BDB0B508B1FF2018E00C4605460A
:104DB00000F084FA0028F7D08F490B4B01EB8502F5
:104DC0000A4D5064074AC0E90A53496843680263C0
:104DD000F22289694161064920469847002040B285
:104DE000B0BD00BF694B0008154F00086D4C0008AE
:104DF000BA0800202DE9F0417F4F8846054600267D
:104E0000052E08BFBDE8F08107EB8604606CE0B1B9
:104E1000032D1AD8DFE805F002041315816911E0AB
:104E2000C16991B198F80320007890420BD066B91F
:104E3000786CC068804740B1606CC16903E0016A6A
:104E400000E0416A09B1404688470136D8E700BF13
:104E500070B501F08BFF684D0024052C08BF70BDB4
:104E600005EB8406706C50B1042C08D8016931B18F
:104E7000806820B1804710B1706C006980470134B0
:104E8000EBE700BF10B58AB0044601F043F908B162
:104E9000FE240DE0FFF73EFF012808D100208DF829
:104EA000040001A801F0E6FA28B1FF2400E0FD2487
:104EB00060B20AB010BD9DF80800A04226D0022CB6
:104EC00014D0012CF1D00CBB00240028F0D08DF8B8
:104ED000084001A801F084FB0028E6D1464840685C
:104EE000016B99B1002000248847E1E70028DCD15C
:104EF00002208DF8080001A801F072FB0028D4D12F
:104F00003D484068016B09B1022088470024CFE783
:104F1000F00200202DE9F04186B014460E46054609
:104F200001F0F8F808B1FE2160E0FFF7F3FE012878
:104F300025D1DFF8C480D8F84400C068804738B174
:104F4000D8F8441028780978884218BF002846D13C
:104F5000284F002E694687F83C6018BF012698F854
:104F600034008DF804608DF81200687802F054FB6C
:104F700058B10020F92603908DF804000CE01D497B
:104F80008879C979FFF772FE25E0297868780026CC
:104F90008DF8081069680391D5E90012ADF810008A
:104FA000C7E9111298F8341087F83E1001A821467D
:104FB00001F0BCF805991128C8F8081015D8FE2191
:104FC000DFE800F00B141313131313091313130F5B
:104FD000131314141411FD2108E0314606E0FC21DE
:104FE00004E0FA2102E0FB2100E0FF2148B206B014
:104FF000BDE8F08150000020F002002080B58AB0AA
:10500000029022208DF8040001A801F0E9FA00289E
:1050100018BF4FF0FF300AB080BD80B500F03EFEF3
:10502000002818BF6FF0010080BD000010B50029F6
:105030000B46044618BF0123002818BF0124234053
:10504000012B04D1BC4CC4E90801227302E0BA4828
:1050500000210162B848037010BD00BFB648007857
:10506000704700BFB44801780079084000F00100A3
:10507000704700BFB0490A78012A0AD10A79012A8B
:1050800007D10278012A04D1007910B1888B013050
:1050900088837047B0B58AB0A74C2178012940F0C9
:1050A000F780417B002900F0F3802179012932D17A
:1050B000817B11B9A18B0131A183C178E02940F036
:1050C000E78081680A780A2AA27100F2E180DFE8AD
:1050D00002F00666696C718486A5B0B4BE0004F166
:1050E00028000AF061FC00202071A08304208DF8C4
:1050F0000400206A00788DF8080001A801F070FA19
:10510000206A407802F098FB206A8068002800F04E
:10511000BF808047BCE0C178E02940F0B980017BC6
:10512000042940F0B58080680178012940F0B08002
:105130004178012940F0AC808178012940F0A880B5
:10514000C078012840F0A48002200025A07301202F
:10515000A5832572257625752574A07120718DF89B
:10516000080004208DF8040001A801F039FA00209D
:1051700002F062FB206A406800B180472834454B4A
:105180004FF0FF310022009520460AF045FB2046F3
:1051900041F288310AF0BAFB00F094F878E002207E
:1051A000A07375E00120A07102E00120A071002031
:1051B00020726DE0037B616A0422A3730A70227B74
:1051C000934238BF1A460123DCB2A24260DD8568F3
:1051D00001332D5D01350D55F6E704202AE004F179
:1051E00028000AF0E1FB00202071A08304208DF844
:1051F0000400206A00788DF8080001A801F0F0F999
:10520000206A407802F018FB206A806800B180476D
:105210004A480121826A0220904739E0007B072832
:105220001FD003282FD105208DF8040002F063FF62
:1052300029E00A208DF804000FE000208DF804001A
:1052400048788DF8080001A801F0CAF920E00D2087
:105250008DF8040048788DF8080001A801F0E0FB03
:1052600016E002F048FF0A79C8784B79120242EA48
:105270000040642218445043039006208DF8040037
:1052800088798DF8100001A801F0CAFB0120A071F7
:105290000AB0B0BD3D8B000827490A78012A0BD11E
:1052A0000A79012A08D10278042A05D101220A7458
:1052B000027A407A0A750876704700BF1F48704727
:1052C000704700001CB51C4C2078012832D1207991
:1052D00001282FD1207C01280BD103200521A073A8
:1052E00000202074606A0170217D4170217E8170F0
:1052F00004E0A079012804D0042809D10120A0717C
:1053000006E0A18B0220A073606A09BA090C018033
:10531000E0208DF80000A07B8DF80100606A01900C
:1053200004F128000AF00AFB0448217A0122C36A2A
:10533000684698471CBD00BF18020020FC000020F2
:105340002DE9F04F85B00446807808B1002658E07A
:10535000A06894F8118094F910701D4691468A4611
:1053600018606079002843D00220A17C8DF80C00E1
:10537000E07C8DF80E1003A906F0E6FE4FFA80FBE4
:10538000BB45A8BF5F4636DAA089A16800268142E6
:1053900028BF0126E289104481422ED308208DF8CF
:1053A0000C00E07C03A906F0CFFE8046E089A168EE
:1053B000B1FBF0F202FB101001281ED12220A17CCB
:1053C0008DF80D708DF80C00E07C8DF80E1003A99F
:1053D00006F0BAFE074640B258450ED1207940B1DA
:1053E000022069468DF80800E07C06F0B7FE00E078
:1053F000FFB2002601E000262E608AF8007089F8CE
:105400000080304605B0BDE8F08F0020704770473F
:105410007047704770477047002070470020704702
:105420000020704700207047002070470020704720
:1054300002207047704700207047704770477047E0
:10544000704700207047704770477047704770473B
:10545000022070472DE9F843002942D0814F914640
:105460008046002207F1080007EB0215002605F12F
:105470000803102E0CD0845D0136002CF9D0741E68
:105480000F2C05D8103001320F2AEDD1022629E069
:10549000386800B93B60786800B10360002605F108
:1054A0000D001FFA89F27B60C5F8109085F80C801A
:1054B0001E600BF0D2FEA8F10500C1B200F03F0063
:1054C00006294FF0000138BF0121392222FA00F0ED
:1054D00008402875D7F8F80048440130C7F8F800AC
:1054E00000E001263046BDE8F88300BF811E0020A1
:1054F000112913D8DFE801F013090B090D0F0B0B6D
:105500000912120F12120D09111105207047022005
:105510007047012070470620704704207047032021
:105520007047000028B14F49D1F8F8100160002001
:1055300070470120704700BFB0B54A4C0021FC22E3
:10554000002520460BF09DFE0020C4E90055B0BDAB
:1055500050B180B543490B68834207D043B11A4626
:105560001B688342FAD104E00120704702680A6098
:1055700000224B68834208BF4A600AB10368136087
:10558000836800220260D1F8F820DB431A44C1F896
:10559000F820002110220BF074FE002080BD00BF17
:1055A00010B5304804683CB120462468017B0029CE
:1055B000F9D1FFF7CDFFF6E7002010BDB0B52948BF
:1055C0000124056865B128462D6801790A29F9D8B2
:1055D00004FA01F111F4E46FF4D0FFF7B9FFF1E739
:1055E0000020B0BD2DE9F04142B3884631B31D4DD6
:1055F0000746164600202D68B5B1AB68C1B27A1ACD
:1056000001339A4210D32A79441C56FA84F072541A
:10561000691D2A890BF021FE287A2044EBE72C68CB
:105620002846FFF795FF2546002DF8D10D48D0F804
:10563000F800C8F800000020BDE8F0810120BDE8B6
:10564000F08100BF58B1002101700649096821B1FD
:105650000A7B002AFAD00121017000207047012046
:10566000704700BFAC09002010B55F4A92F82010C7
:10567000042911D8038894682380231DC078E07022
:105680000020A070481C82F8200002F11C00844217
:1056900008BF02F10C0393600020052938BF0120E8
:1056A00010BD00BF504890F82000704780B54E49AB
:1056B00091F820202AB14968FBF78EFD08B14078A7
:1056C00080BD012080BD00BF2DE9F843DFF81891AF
:1056D00004460025E84699F82070BD4228BFBDE881
:1056E000F883D9F8040086780178427821706270D6
:1056F0002EB1D9F8000081682046884706E0C078BE
:105700008DF801208DF800108DF8030000F02CF8C2
:1057100016B94046FFF7A8FF0135DEE710B5324C59
:105720000021142284F8201004F10C01C4E90001C6
:10573000A1600846FF210BF0A4FD012084F82100A0
:1057400010BD00BF80B528494968FBF745FD00281A
:1057500018BF012080BD00BF234890F82010002012
:10576000042988BF0120704710B51F4991F8200017
:1057700058B14B68421E81F8202001F11C021C1D0B
:10578000934208BF01F10C044C60002818BF0120AF
:1057900010BD00BF10B50446134890F8202042B158
:1057A000426808461146FBF717FD10B1012144700D
:1057B000817010BD70B50C4991F8202081F821004E
:1057C00082B1D1E90152012301F11C04EE78687025
:1057D00006B9AB702E1DA54208BF01F10C06354677
:1057E0009642F3D170BD00BFA80A002004280FD153
:1057F000F8B5002004217F22CDE90200CDE90000A8
:10580000684608F027F8002818BF0F2004B080BDB4
:105810000B20704709B10B207047F8B50021012813
:10582000CDE90211CDE9001102D120208DF8000050
:1058300068460021042208F00DF8002818BF0F2048
:1058400004B080BD7CB50C460021019133B101A9A3
:105850001E461546FBF700FD10B17CBD0A207CBD3D
:105860000198411C0CD081B2691A012901DB0D1885
:1058700006E0B1B100F580314FF6FF7291430D445F
:10588000AE4935600968897839B90021281A61F173
:105890000001001B71F1000001DA00207CBD08202E
:1058A0007CBD306007207CBD30B1A4490968C9685F
:1058B00001310160002070470A2070472DE9F04354
:1058C0008DB002B30E46F1B104AC07462121154656
:1058D0002046FAF7E7FDDFF8C09300202B680DF1B2
:1058E0000F018DF80F00D9F80000B0F80480287976
:1058F000CDE90004029138463146424608F08CF862
:1059000028B10F2000E00A200DB0BDE8F0832A790D
:10591000286804A90BF0A1FC284601F0DAF908B1C7
:105920001020F1E7287AE98841EA0046D9F800001A
:1059300081688E4201D10320E6E786609DF80F0062
:105940000021FFF767FF0028DED10420FFF74EFF9C
:105950000028D9D1E87AB5F80910434641EA004554
:10596000032031462A46FBF7A7F90028CCD10220B4
:1059700031462A464346FBF79FF90028C4D1D9F89F
:1059800000109DF80F3000204FF0FF328B70C1E9FE
:105990000302C1E90522B7E7B0B580B1BE4D0021D1
:1059A0002822002428600BF06CFC28680549FF229F
:1059B0000160C46010301421FAF74AFD00E00924A8
:1059C0002046B0BD0001010190B11CB50446002085
:1059D000019001A808F05EF8AF48BDF80410006817
:1059E000E1828180204601F0DAFE18B111201CBD51
:1059F0000A20704720461322012350F8181B0090FC
:105A0000002007F021FF08B10F201CBD204601F047
:105A1000C6FE002818BF11201CBD00BFF0B587B01E
:105A20004BB39D4E04463068C068A04201D90620A1
:105A300022E01D460FD2AB6895F82810686A95F8E9
:105A400020700022CDE900240322002F08BF02228B
:105A500003F002FD80B9284601F03AFE08B111209A
:105A60000AE0296839B12879043882B2B2F5807F1A
:105A700004D90E2000E00A2007B0F0BD0023AF6873
:105A800005F12C0C8DF816408DF81B008DF81A309E
:105A90008DF81130CDF80D304923CDF800C08DF8C8
:105AA0000C30230E8DF812708DF81930230C8DF800
:105AB0001830230A8DF817303B0E8DF815303B0C4B
:105AC0008DF814303B0A8DF8133003A8022307F039
:105AD000BBFE08B10F20CFE7284601F0F9FD0028F2
:105AE000BDD13068C4600020C6E700BF10B50446D1
:105AF00007F0F8FF08B10F2010BD0CB1002010BD59
:105B00006548002100688078FFF784FE0028F2D104
:105B10000420FFF76BFE0028EDD1EFE75E4909682E
:105B200008600020704700BF28B15B4909681C313C
:105B30000162002070470A20704700BFCC0A002095
:105B40002DE9F04FCBB0549F7FB3064600200DF1F6
:105B50001C088B461C461546079010464146FBF72D
:105B60007BFB08B1062021E00798A04201D3013059
:105B7000F8D1384601F052F808B1102016E006A915
:105B80003046FBF743FB88B9B868584511D1D7F8C0
:105B900000A0BAF1000F08D03879061F1FFA86F965
:105BA000B9F5807F07D90E2000E00A204BB0BDE890
:105BB000F08F0220FAE7039006984FF4887241783C
:105BC00080780291F96A05904046049100210BF01B
:105BD00058FB012000214A468DF826408DF822B05E
:105BE0008DF82B608DF8210049208DF82A10CDF812
:105BF0001D1051468DF81C00200E8DF82900200C38
:105C00008DF82800200A8DF827004FEA1B608DF8D8
:105C100025004FEA1B408DF824004FEA1B208DF829
:105C2000230008F110000BF018FB0398DDE90423B2
:105C300000F10C01404607F089FF0146012818BF1A
:105C40000F200029B2D197F82020012397F82810BF
:105C5000786ACDE900345B46002A029A08BF022226
:105C600003F0FAFB0028A1D1681E032812D8DFE850
:105C700000F002060A0E0848006804610AE00648BF
:105C80000068446106E004480068846102E002485C
:105C90000068C461002089E7CC0A0020B0B501F09B
:105CA000B7FD08B10120B0BD514C1D4D04F55A702F
:105CB000A84704F56070A84704F56670A84704F586
:105CC0007E70A847FFF7A6FB06F09AFA1548C06A4F
:105CD00080470020B0BD00BFB0B5454C104D04F565
:105CE0005A70A84704F56070A84704F56670A84785
:105CF00004F57E70A847FFF78DFB0A48C06A80470D
:105D00000020C4F8400300F011F80748F2494FF4AE
:105D1000E5620BF0A2FA0120C4F840030020B0BDF8
:105D2000A9F900084C2901080080002070B5EB4E4D
:105D3000D6F8400300B170BDE74D24212846FAF79C
:105D40000BFF696A884201D1002401E001246862E6
:105D500005F1280002F020FEE96B88421CBFE863D1
:105D6000023405F14000DC21FAF7F6FED5F81C11EB
:105D700088421CBFC5F81C01043405F59070BC2195
:105D8000FAF7EAFED5F8DC1188421CBFC5F8DC0141
:105D9000083405F5F0709021FAF7DEFED5F87012A0
:105DA00088421CBFC5F87002103405F51D704FF411
:105DB0009361FAF7D1FED5F80C1788421CBFC5F8DD
:105DC0000C07203405F5E26002F0E6FDD5F8241753
:105DD00088421CBFC5F824074034D6F84803002881
:105DE000A9D0C1680029A6D02046BDE87040084768
:105DF000D01200202DE9F04F89B0002800F04A8130
:105E00000D46002900F0468104460068002800F095
:105E100041816068002800F03D81A068002800F002
:105E20003981E068002800F035811046174606F0F9
:105E30009AF9002800F033812046FFF76FFCA64E48
:105E400000214FF4E5624FF0000A30460BF019FADA
:105E5000DFF8BC8D002140F20C5240460BF011FAE5
:105E600040F201100DF11C09DFF878B286F804A1A8
:105E700086F8407086F880A0A8F811049848494632
:105E8000C6F814010F208DF81C003846D8470028AA
:105E900018BF012086F8080149460A208DF81C0029
:105EA00002F053F986F8CC00062049468DF81C0014
:105EB00002F04BF986F8CD00102049468DF81C0001
:105EC00002F043F9C6F8900096F8400011274946C1
:105ED0008DF81C70D847C6F89400122049468DF8FA
:105EE0001C0002F032F9C6F89800132049468DF8DC
:105EF0001C0002F02AF9C6F89C00142049468DF8CF
:105F00001C0002F022F9C6F8A000172049468DF8BF
:105F10001C0002F01AF986F8A500182049468DF8F1
:105F20001C0002F012F9C6F8B000C6F8A80019204B
:105F300049468DF81C0002F008F986F8B40086F88E
:105F4000AC001E2049468DF81C0002F0FEF886F8D1
:105F5000B8001F2049468DF81C0002F0F6F886F8BC
:105F6000B900202049468DF81C0002F0EEF8C6F872
:105F7000BC00212049468DF81C0002F0E6F8C6F866
:105F8000C0000B2049468DF81C0002F0DEF8A8F88E
:105F9000F4030C2049468DF81C0002F0D6F84FF0AF
:105FA00001090621A8F8F6030A2006F1900C06F173
:105FB0004C0E8DF818A086F8A49086F88C10C6F8C0
:105FC000880086F84810706486F860909CE80F108E
:105FD0008EE80F1006F51D70059006F5F070049020
:105FE00096F8400004A906F0B9F8C8F8485306F03E
:105FF00007F988F885A4C8E9D0943B4B3B4C08F5D9
:106000005A704FF0FF31002286F80591C6E90BAABD
:10601000CDF800A0A047364B08F560704FF0FF3177
:106020000022CDF800A0A047324B08F566704FF073
:10603000FF310022CDF800A0A0472F4B08F57E705D
:106040004FF0FF310022CDF800A0A04702A808F0D1
:1060500009F8DDE902012B4A2C4C2B4BC6E9430120
:10606000C8E9D32426492A4C2448C8E9D513216815
:10607000C8F85C0308F553708847A96806F5907066
:1060800007F01EFC38B9F94D2846FFF785FC40B1F2
:10609000112700E00327384609B0BDE8F08F092733
:1060A000F9E7FFF749FA08B11327F4E705F1D8003B
:1060B000FFF73AFD0028EBD16069E66AA46D8047DE
:1060C0000BF070F995F80501A047B04701200027B3
:1060D00088F88604DFE700BF28870020D012002060
:1060E0000003000149C10008E592000819F8000802
:1060F000F58F00082D900008158A0008ED8C000827
:10610000918C00084D8D0008098D0008A18D0008B4
:106110004C290108D448D0F8401390F8860480F048
:106120000100084318BF0120704700BF2DE9F04F60
:1061300091B0002800F01581DFF8D4BA0446012799
:10614000DBF84003002840F07F819BF8860401289B
:1061500040F07A8188460BF58760002114224FF0C9
:1061600000090BF08EF801218BF812148BF839140A
:10617000207803280FD0012818D070BB012004F12B
:106180000C0104F108024FF040098BF8110404F1EE
:106190000E00237919E08BF81114002304F10A0092
:1061A00004F10801221D4FF0E0090EE0E07B04F14C
:1061B0000C0104F108024FF08009082828BF0820CC
:1061C0008BF81104237904F10E000493067810680B
:1061D000012505900888039005E000200026002591
:1061E000049000200590DFF82CAA02278DF81C707F
:1061F0009AF874109AF840008DF81E1007A905F05F
:10620000A3FF40B271B28842B8BF0846002D00F02B
:1062100018819AF8061111B19AF8392012E09AF80B
:1062200074108DF818009AF8400005228DF81A10A5
:1062300006A905F0DEFF002800F093809DF81820E5
:106240008AF839209AF81811DAF828009AF83830C4
:1062500000290E9000F087809AF80711CDF8008091
:1062600011B90021CAF830100B9001209AF84010A3
:1062700002938DF835309AF8043116468DF83420A3
:106280009AF874208DF82800DAF814018DF8371088
:106290009AF806118DF83620012B0AF13802099080
:1062A000DBF8F4034FEAC1180AF139010C909AF8AF
:1062B0003A0008BF08F11008002818BF08F12008AC
:1062C0005FFA88F0C0098DF8290009A80EABFFF726
:1062D00037F8059901900020039F0BF59C758BF80A
:1062E0001404ABF80000CDE90F002846002908BFD0
:1062F0000F46BAB20AF0B1FF39468BF8377202275F
:106300008BF80290B7EB591F09D04FEA59100728B4
:106310002BD0042840F0818001208BF814040198D0
:106320008BF80D918BF83011CBF82C5160F3861857
:1063300004988BF814818BF82801FF208BF80C014E
:1063400004208BF804010BF10200CBF80801DAF805
:10635000D400CBF8100110A8FFF7A6FAB0B11227AD
:106360005BE0032770E007275CE0059800284FD02A
:1063700008064DD0CAB205990BF103000AF06DFF73
:106380009BF837020130ABF8000041E01098ABF801
:106390001601CBF844040020ABF83C040FA8FFF72B
:1063A000C1F808B1132738E00F9888B39AF939007B
:1063B000FAF77AFF9BF837720F9D9FB10F2D11D816
:1063C0000BF58C720FA90F20FFF70CF90028E9D10B
:1063D0009DF83C1008F0F00001F00F0108448BF824
:1063E000140115E00BF28C480FA94246FFF7FAF8AA
:1063F00027B1102D02D30028D4D109E00028D1D133
:106400000020CBF82C818BF828010F988BF83001F5
:10641000009807F081F80746D0B102988AF83960F1
:106420008AF838001FB100208BF8140409E02078A6
:1064300000278BF838049BF8850440F001008BF8A6
:106440008504DBF888042061384611B0BDE8F08F80
:106450000E9800278AF83A70CAF82800FFF7A0F8CB
:106460000028DFD01327DDE7D01200202887002086
:10647000022070471CB5002826D004460078372833
:1064800000F23A80DFE800F01C2226292C30343854
:10649000383838383838383C4044464A4E525759D4
:1064A00063676A6D7073767A7E8286898E9195971E
:1064B000389938383838383838383838383838A192
:1064C000454890F804016BE003201CBD424890F859
:1064D000180165E007F0DAF97AE007F0DBF977E018
:1064E0003D4890F806015BE03B48D0F8D0006FE0F3
:1064F0003948D0F8D4006BE02046FEF799FF1CBD68
:10650000354890F805014BE0334890F8800047E0AB
:106510001D2013E03048D0E919100AE02E48D0E9D8
:106520002A1006E02C48D0E91B1002E02A48D0E9E6
:106530002C10616047E01A2000E01B208DF800005D
:106540002548694690F8400005F0FEFD40E02248ED
:1065500090F8600024E02048C06C39E01E48006DCF
:1065600036E01D48406D33E01B48806D30E01A482E
:10657000C06D2DE0184890F8CD0011E0164890F855
:1065800039000DE0144890F8380009E0124890F8FE
:10659000CC0005E01048406C1AE00F4890F8480025
:1065A000207116E00C48C06F12E00B48D0F8C00014
:1065B0000EE009480CE009480AE00748D0F8140149
:1065C000606005F0C7FDA06003E00348D0F88400D8
:1065D000606000201CBD00BF2887002000800020D4
:1065E000FEB5002800F0AF81DFF824760446D7F826
:1065F0004003810700F108822178372900F25B818E
:10660000DFE811F038003C00450049005100570018
:106610005D00630045014A016F0075007B00810049
:1066200087008D00540159015E019700AB0079018C
:10663000CE00D000E000E900ED008B018F01F100F9
:10664000F50005011B0193012A01A301AA013001F4
:10665000AF01590135015901590159015901590138
:10666000590159015901590159015901590159015A
:1066700059014001207907F041FC1FE120790228EF
:1066800000F06181DFF8881F81F8180167E1606818
:1066900007F00EFA02E0606807F016FA04460028D8
:1066A00018BF0324B1E12079DFF8641F81F80601E7
:1066B00055E16068DFF8581FC1F8D0004FE160680D
:1066C000DFF84C1FC1F8D40049E16168002900F0EF
:1066D0003A8100200024FFF709FA002840F0E48006
:1066E00093E16168002900F02E810320D8E0616801
:1066F000002900F028817F20D2E06168002900F0A5
:1067000022818020CCE06168002900F01C8181207A
:10671000C6E06168002900F016818220C0E020797F
:10672000BC4981F80501BD49CC6A896D8847A047FD
:1067300015E1B84D01F028FF8DF8000095F84000F4
:106740008DF80110694605F054FD002800F0FB802B
:10675000D4E90101C5E92A0101E1AE4D01F014FFC0
:106760008DF8000095F840008DF80110694605F09D
:1067700040FD002800F0E780D4E90101C5E91B01D4
:1067800095F80401022840F0EA8095F818010028E5
:1067900000F0E580A148C06A804702F0FDFDDEE020
:1067A000002000E001208DF8080060680190994801
:1067B00090F8400001A905F064F90324002818BFEF
:1067C000002422E12079411E0E2900F2BC8091496B
:1067D00081F86000C3E060688E49C864BFE060680B
:1067E0008C490865BBE060688A49C865B7E02079D4
:1067F000884C694606228DF8000001F065FF0028EC
:1068000000F0A1809DF8000084F8CD00A7E0207979
:10681000804C052294F874108DF8000094F8400024
:106820008DF80210694605F0E4FC002800F08B802A
:106830009DF8000084F8390091E02079F54C694614
:1068400009228DF8000001F03FFF00287BD09DF861
:10685000000084F8380082E06068EE494864C1F8BE
:1068600088007CE06068EB49C1F8C00077E0A0795F
:10687000012868D86068E749C1F814016068FFF72B
:106880004DF90FE06068E349C1F8840067E0616892
:10689000002958D0012003E06168002953D002206C
:1068A000FFF724F900285AD01124AEE02079D94905
:1068B00081F8800053E02046FFF7DAFD0446A4E0AB
:1068C000D44D01F061FE8DF8000095F840008DF880
:1068D0000110694605F08DFCA8B360686946002286
:1068E000009095F8400005F084FC60B3D4E9010104
:1068F000C5E9190133E0C74D01F046FE8DF80000EF
:1069000095F840008DF80110694605F072FCD0B191
:10691000D4E90101C5E92C0121E06068BD49486561
:106920001DE06068BB49886519E02079B94C69466B
:106930000A228DF8000001F0C7FE20B19DF800008A
:1069400084F8CC000BE003245FE02079B14981F8A2
:10695000480081F88C0002E06068AE49C8670024F6
:1069600053E0012850D12C4C24212046FAF7F4F8AA
:10697000616A88424BD104F1280002F00DF8E16B06
:10698000884244D104F14000DC21FAF7E5F8D4F85C
:106990001C1188423BD104F59070BC21FAF7DCF859
:1069A000D4F8DC11884232D104F5F0709021FAF766
:1069B000D3F8D4F87012884229D104F5E26001F0CE
:1069C000EBFFD4F82417884221D1924D124E4FF498
:1069D000E562284631460AF040FC304600214FF47B
:1069E000E56200240AF04DFC40F20120A7F8F20312
:1069F00097F8150487F8E003E86EC7F8E40395F804
:106A0000750087F8F00300E001242046FEBD17243E
:106A1000FBE700BF28870020008000204C290108E8
:106A20002DE9F04186B004460020ADF802006CB1BB
:106A3000774F0125D7F8400348B997F88604012815
:106A400005D1FEF789FE30B1012500E00325284677
:106A500006B0BDE8F081FEF725FE28B907F24C40EC
:106A6000002114220AF00DFC97F88504002102256C
:106A70008DF8071040F0040087F88504012087F89E
:106A80004D048DF8050020788DF8040001380D289C
:106A900000F29980DFE800F0079797484C669797D7
:106AA00097759779878D97F840038006CCD405F0C9
:106AB000A7FBDFF8A48D94F905100022002598F8B3
:106AC000400004F0CAFF88F8390007208DF805005F
:106AD000002007F013FAFF2087F80451A7F80C01F3
:106AE000B81CC7F8080106F0D5FE014607F5877007
:106AF00008220AF0B2FB06F0C9FE014607F58B70CA
:106B000008220AF0AAFB002006F006FD00285AD051
:106B1000064694F9051098F84000012204F09DFF04
:106B200088F8390035464EE00DF10201022043E0BD
:106B3000384A97F81504A18892F838308DF8080083
:106B400092F8395092F84000ADF814108DF80A30E0
:106B5000D2E91E328DF809500393049202A905F080
:106B600035FB06E02C4B94F90C10A068A288DB6B77
:106B70009847D7F84003002540F00200C7F84003CB
:106B800021E00DF102010D2016E001258DF80750DE
:106B9000FEF742FCB8B900200025FEF754FC0020A7
:106BA000FEF735FC0FE01B4890F8040118B30225EE
:106BB00009E00DF1020112200022FEF74BFC054610
:106BC000002818BF1325D7F88804206175B1FEF797
:106BD00069FD00287FF43BAF002087F8140497F884
:106BE000850400F0FB0087F8850430E701A8FEF774
:106BF0003BFD00252BE7257905F00700FEF725FC76
:106C00008DF802500DF1020110200122D5E700BFDE
:106C1000D0120020288700204C290108B0B5002898
:106C200055D001680446002951D008786071487831
:106C3000A0608A7840EA0220A060CA7840EA024058
:106C4000A0600A7940EA0260A0604A79227302F0EB
:106C50000F028879E081CB79083140EA0320E08196
:106C600004F110000AF0F9FA0020217984F82800D4
:106C700084F82000207B00F00F0202F10803C81AFC
:106C800005280EDB25680932606A891AEB5C84F8F6
:106C900020300B1FA918DAB284F828300AF0DDFA88
:106CA00021792068084410F8041CE16210F8032CD4
:106CB00041EA0221E16210F8022C41EA0241E1625C
:106CC00010F8010C41EA0060E0620020B0BD022033
:106CD000B0BD10B578B30168044661B311F8010B7B
:106CE00003226071A01D0AF0B8FA216804F10900BE
:106CF000032204310AF0B1FA2168C879E0600A7A07
:106D000040EA0220E0604A7A40EA0240E0608A7A83
:106D100040EA0260E060C87A2074087B60742079E1
:106D200021280AD104F112000D3110220AF095FA3F
:106D300021681D2006E0022010BD112801D9012084
:106D400010BD0D200A5C0B1840F0020062625B78F7
:106D500042EA032262620B5C084442EA0342626236
:106D6000407842EA00606062002010BD2DE9F04FDB
:106D700097B0DFF89868EFF31080EFF3108172B6E8
:106D80000023F178B6F8012096F80090336080F384
:106D9000108842EA014049EA0020002800F085817D
:106DA0005FEAC9605ED5DFF8B07A97F8040102287F
:106DB00003D0DFF86008C06A8047DFF8785A05F52D
:106DC0006074D5F8B01301F066FA01F01FFE05F506
:106DD0006674D5F8B41301F05EFA01F017FE97F867
:106DE0000401022802D095F8140480B116208DF811
:106DF000180097F8400006A905F0A6F9D5F8B413D5
:106E000005F57E74014401F046FA01F0FFFD70685B
:106E1000F862099095F815048DF8200004A807F091
:106E200021F9D7E94330DDE90412009014A807F0F6
:106E300045F9DDE91401CDE90B01D5F8180497F8FF
:106E400018110A9097F84000002918BF01218DF809
:106E5000211008A905F0B5F995F8140410B900201F
:106E600085F839045FEA097040F1E780DFF8C4A9CA
:106E7000002096F814B0778AF568348ADFF8D8696C
:106E80000490CAF824048AF83C04CAF82C048AF84E
:106E90002104AAF81E048AF81C048AF83404CAF8EB
:106EA0003004CAF82704DFF86C079AF88414D6F87F
:106EB000D4808AF882B4AAF88074C06A8AF88314ED
:106EC00080470AF5667008F06FFD28462146FEF7F8
:106ED000B8FA20B18AF878B4AAF87674ADE096F8DA
:106EE0000401012816D1FEF79FFA38B10020FEF701
:106EF000ADFA0020FEF7A2FA042009E0FEF792FAAC
:106F000040B10020FEF7A0FA0020FEF793FA05201A
:106F10008AF883042F784FF0FF3000EB57100628D3
:106F200021D8DFE800F00420292026205D00102C65
:106F300050D996F818018DF824400895002849D1B9
:106F400006F0A8FC08AD0146FF202A46FEF7B6FC75
:106F5000002800F0E6810120FEF7F4FB002800F095
:106F60001B82072015E201208AF81D0402F0D6FAE0
:106F70004BE001208AF81C0496F8751096F88020E2
:106F800096F840008DF852109AF820148DF85110A0
:106F90000E21002A08BF0D218DF8501014A905F00C
:106FA000D3F8A4F10D0100B209B221EAE1718142E6
:106FB00010DC0B2C0ED9FF208DF8244008958DF89D
:106FC00048000AF50E70119008A8FFF727FE002868
:106FD00000F0978101208AF81D0402F09FFA2CE04E
:106FE0000AF50E78013C691CA2B240460AF035F958
:106FF00003208AF82844CAF82484AAF81C049AF8C2
:10700000850440F002008AF885049AF814040028E8
:1070100000F0DE809AF83C0410B1002001F0FAFC88
:107020009AF8850440F020008AF8850496F8040157
:10703000022818BF06208AF884045FEA497026D522
:10704000DFF81458022495F8040102284FF00200DA
:1070500008D0DFF8C005C06A804795F8040102280F
:1070600018BF0620DFF8CC5785F88404022085F885
:107070003944FEF79FFB95F8140410B1012085F800
:10708000130495F8850440F0200085F885045FEA34
:10709000897003D505200621FDF7CEF95FEAC97096
:1070A00003D003200421FDF7C7F9FEF7C8F9DFF884
:1070B000844794F88514880640F1FA80002084F80B
:1070C0008604D4F84003020644BF20F08200C4F8CE
:1070D000400311F0050F0AD00C20FEF733FB94F8A3
:1070E000851420B111F0010001D1480736D44807BA
:1070F00015D50120FEF726FB38B10120FEF7D6FAA0
:1071000058B9002084F8100407E00520FEF71AFBA8
:1071100018B90620FEF716FB08B101F0F1FB94F850
:107120008504C10700F0828094F83814032903D045
:10713000012916D000296FD1DFF81C1794F81034FC
:1071400091F8602093423AD2820765D591F80411F4
:10715000A9B394F8831400295ED130E001F0D0FB8C
:1071600068E094F81314002960D094F8112494F87E
:107170001214914204D2820730D594F83C246AB3A9
:10718000DFF8D40690F81621CAB994F83C24A2B9C5
:1071900002218DF8281000F51D71099100F5F0719C
:1071A00090F84000089108A904F0D8FF94F8121450
:1071B000002084F83C0484F8140484F83D1404F599
:1071C0005A7008F0F1FB01F054FB06F04FFE2DE081
:1071D00096F8040102283FF420AF21E7DFF8785643
:1071E00095F81621C2B9013184F81214C90713D0D9
:1071F000222095F8391095F874208DF8200095F824
:1072000040008DF822208DF8211008A904F09CFF81
:1072100085F8390094F8850400F0DF00002184F837
:107220008504002084F8131402F05CF894F88514A7
:10723000D4F84003A8BB01F0010001F004052A18AE
:1072400004D085F0FE02114084F88514012184F8F1
:10725000861428B1D4F84403016804F58760884790
:1072600065B104F24C40FEF72FFAFEF71BFA28B185
:1072700094F8850440F0040084F88504FEF7E0F8F3
:1072800094F8850400F0DF01D4F8400384F88514F5
:1072900038B900208DF8200008A8FEF7D3F994F83B
:1072A000851441F04001012084F8860484F8851497
:1072B000080709D501F0F70000F0F9FFC26804F5EE
:1072C0008C60904794F88514880707D501F0FD007D
:1072D00000F0EDFF426804F21C40904794F88404EB
:1072E000022808BF02F058F894F88504410605D535
:1072F00000F0BF0084F88504FEF718FD17B0BDE864
:10730000F08F9DF82CC00A9D5FEA0C71CAF83054CA
:1073100047D09DF8401000294FD0CDF80C800020B8
:1073200055E00021BDF829200B9886F816119DF82C
:107330002B1042EA0141C6E934109DF8300000F0FC
:107340000F01C0F3021086F861009DF8310086F845
:10735000701086F868104FF47A71002808BF012079
:1073600010FB01124843C6E91402A4F111008DF884
:10737000540005F11200149096F8400014A904F08E
:1073800073FB022086F818010120FEF7DBF918B123
:1073900000200121FEF7FEF99AF8850440F008006C
:1073A00031E69DF84810CDF80C8079B19DF8401079
:1073B0000320002908BF022009E09DF848100120A1
:1073C00000297FF408AECDF80C8000E001200023F6
:1073D0004FEA571E01242C2104935FEAC47837D06A
:1073E0001A46BA4B002402FB01360123D6F8DC70A2
:1073F000AF42F2D196F8DA6001230024002EECD0DF
:10740000B24B2C2102FB0131D1F8F82091F8DB407E
:1074100093F8041112680229049202D103218AF818
:1074200083141CF0600F08BF03287FF4D3ADCDE9AF
:1074300001E015208DF85000A44890F8400014A9F0
:1074400004F082FE002C00F08680012C0DD03CE080
:10745000CDE901E015208DF850009C4890F84000DF
:1074600014A904F071FE039D0024FB494FF48032FF
:1074700091F81611B2EB014F06D10299022621B103
:10748000032918BF012600E0032627460124BDF882
:107490002E2081B204AB3046FEF7D4F9B8B10828EB
:1074A00023D0072811D10820EB4A8AF81D0401983F
:1074B00005281DD192F81601D0B9506B1399884256
:1074C00016D1012082F83A0012E001200EE0049B60
:1074D000039708AF2046294632460097FEF730FB57
:1074E00060B1022835D10B2075E50A208AF81D0409
:1074F0000498CAF86404CAF82C046EE503980022C4
:107500008AF81D248AF82824CAF824248AF8392401
:107510008AF81E040498CAF86404CAF82C049DF87A
:107520002C00C0F300118AF82114C0F340118AF82E
:107530003C148AF82A149AF8831401299CBFC64B7C
:107540009A62DDE90125B8F1000F07D0C24E022290
:1075500014E00C203FE50426012798E7BE4E052ADB
:1075600009D196F81631012286F83A2033B9139AD8
:107570007263012202E0002286F83A2001298AF88B
:107580001C2407D89AF83814012901D1800601D5A6
:10759000FEF714F8DFE805F002171E2A9DF82C10FC
:1075A00007F110004FFA8BF201F00F0102F078F8AA
:1075B00001208AF829049DF840008AF81F041198D8
:1075C000CAF824041CE09DF82C1007F1100001F00B
:1075D0000F0102E09DF8481011984FFA8BF202F06B
:1075E0005FF89DF840008AF81F0408E59DF8400008
:1075F0008AF81F041198CAF8240401208AF8290483
:107600009DF848008AF82804F9E400BF60020020D1
:10761000288700204C290108B0B588B005468E485F
:107620000C4690F8CD20816A8DF8072090F8CC2088
:1076300002918DF806200022009284B30591D0F8C3
:1076400014118DF8102090F8392090F840300391F3
:1076500090F806118DF81C208DF81F300DF10602F0
:107660008DF811107349D1F8F413069190F8381081
:1076700090F874008DF81D108DF81E0003A80DF110
:10768000070102ABFDF75CFE9DF90700F9F70CFE60
:1076900060706846FDF746FF18B1132013E0032021
:1076A00011E000980F2802D86178884203D90020A1
:1076B0002070082007E00A1A28442270002288421D
:1076C00088BF0122D00008B0B0BD00BF28870020CD
:1076D000B0B598B10446006880B1227B94F8283098
:1076E0000925217902F00F02002B08BF08252A4442
:1076F0001A4404328A4203D90220B0BD0120B0BD31
:10770000617901702068A1684170A1682068090A48
:10771000817020686189C1702068E17A01712068F8
:10772000217B41712068A17B81712068E17BC1715F
:1077300004F11001227B2068083002F00F0209F0EA
:107740008CFD207B94F8281000F00F0000F1080554
:1077500039B1206894F820104155013594F828205B
:1077600000E000222068616A284409F076FD94F860
:1077700028002168E26A28440A542168E26A014428
:10778000120A4A702168E28D01448A70216894F8D7
:107790002F2001440430CA7020710020B0BD10B504
:1077A00038B10446006820B12179172903D202209C
:1077B00010BD012010BD617908220170A11D206853
:1077C000013009F053FD206804F10E010822093050
:1077D00009F04CFD2068A17D41742068E17D817431
:1077E0002068A169C174A1692068090A017520682F
:1077F000618B41752068E17E817517202071002022
:1078000010BD00000B480021C0F840130020704755
:107810000848D0F8401341B990F88624012A04D1D1
:107820000121C0F8401300207047481E18BF0120F6
:10783000704700BFD0120020BCB5074D04468DF83C
:1078400004000F2295F8400001A904F0D2FC08B111
:1078500085F80841BCBD00BF288700202DE9F0470E
:107860008AB04FF0000917225A23012503240E2065
:107870000A215E4FCDE90045CDE90259CDE9043238
:10788000594BCDE9061000F077FCCDF82490022486
:10789000B847574B00F070FCCDE90054CDF8089084
:1078A000B8470420534B00210022CDE900400220BC
:1078B000CDF80890B84750A300F05EFCCDE9005425
:1078C000CDF80890B84709AD00202946FDF78CF99E
:1078D000099852A3C0F30721C0F30742000ECDE977
:1078E00000020291022000210022B847012029460F
:1078F000FDF77AF90998C1B2C0F30722C0F3074334
:10790000000ECDE90003CDE902214DA302200021A4
:107910000022B847DFF84CA1534BDFF850814FF4F9
:10792000FA710022CDF800900AF10800C047504BD0
:107930000AF120004FF4FA710022CDF80090C04700
:107940000AF138054B4B4FF4FA710122CDF8009043
:107950002846C047484B0AF150004FF4FA61002214
:10796000CDF80090C047454A454E01200021B04760
:10797000444A02200021B047434A04200021B04776
:10798000424A08200021B04700F090F840484FF0EC
:107990008171FDF741F93F4F07F10C00FCF7E0FF63
:1079A000284607F0CBFF9AF80200002818BF0124F0
:1079B00020460021FDF75AF9374C3968374B002231
:1079C000CDF800902046C047204607F0B7FF344A64
:1079D00010200021B047334A20200021B04704F096
:1079E000ADFE0AB0BDE8F0870083010835F5000858
:1079F00031840108108401084D575F524144494FBA
:107A00005F56455253494F4E3A2020202056255864
:107A10002E25582E25580D0A000000004C325F53C9
:107A20005045435F56455253494F4E3A202020203F
:107A3000205625582E25582E25580D0A00000000E6
:107A400052505F535045435F56455253494F4E3A4B
:107A500020202020205625582D25582E25582E250B
:107A6000580D0A00480300208993000819F80008FF
:107A7000E58F0008318C000871900008514E000815
:107A8000F9F600087DDB0008A5DE000885DD0008AA
:107A9000B000002000000020541900206593000869
:107AA000D9C600081DC800080548704704480021D1
:107AB00001220323C0E90032C0E90211704700BF70
:107AC000A84B002010B51348002107224FF4805323
:107AD000114CC16480F83C10C0E90C328263012271
:107AE00080F82C10C0E909114FF0004380F82010F5
:107AF00081760183C2610422C0E90043C0E902111A
:107B0000C0E90412F9F7EEFD18B1BDE81040F9F72D
:107B1000F7B910BD784900200024014080B5042049
:107B2000FCF7BEFE0120FCF7BBFE0F200221002265
:107B3000FAF7A0FE0F20BDE88040FAF78DBE0000E6
:107B40002DE9F04385B02A4C4FF0000902204FF098
:107B50000208CDF81090A0470420A047012001267C
:107B6000A047244C4FF43A4100222046FAF786FB06
:107B70006D464FF40A40204FCDF80C80CDE90169E5
:107B8000009020462946B8474FF404100296294633
:107B9000CDE900804FF09040B8470320294603907C
:107BA0004FF44050CDE9016900902046B8474FF4AA
:107BB0008810CDF808802946CDE900604FF090404C
:107BC000B8470E4C062000210022A0470C4D06208D
:107BD000A847072000210022A0470720A847162019
:107BE00000210022A0471620A84705B0BDE8F08379
:107BF000BD48000800040048E5200008752800087A
:107C00005928000810B50F4C0F4A104B01200021D5
:107C1000C4E90032C4E9021004F110001421F8F79D
:107C200041FC2046FAF78AFB50B906480021FAF7D2
:107C300047FB28B903480021FAF760FB00B910BDE3
:107C4000F9F75EF93C4A00201A0910200054004060
:107C500080B506F05FFABDE88040FFF7FFBD4FF04A
:107C6000FF3007F059BD000080B58CB001A82C2171
:107C7000F8F718FC174800224FF480714FF080434A
:107C8000C0E90422C0E90623C0E908211F21816060
:107C900011490160FBF7F6FB08B1F9F731F90D481E
:107CA000FBF780FB08B1F9F72BF94FF48070002245
:107CB0000B904FF000500790002006900290089023
:107CC000044801A9FBF764FC08B1F9F719F90CB0F5
:107CD00080BD00BF884A00200028004080B50548CC
:107CE00008210160FBF7A4FD18B1BDE88040F9F759
:107CF00007B980BDC04A0020B0B588B0184C194DF6
:107D0000164800224FF0804140F2E7330792CDE958
:107D10000522CDE90322CDE9012224688261B4FB6A
:107D2000F5F4013CC0E90014C0E902230261FBF74D
:107D3000EBFE88B94FF480500490084804A9FBF783
:107D400041FF48B9002003900190044801A9FBF7C6
:107D5000AFFE08B908B0B0BDF9F7D2F8CC4A0020A0
:107D60004401002040420F0010B5174C174B4FF450
:107D7000E1320C200021C4E90032C4E90211C4E957
:107D8000041004F118001421F8F78CFB2046FCF7CE
:107D90001DFA08B1F9F7B4F80B480021FCF769F8AF
:107DA00008B1F9F7ADF808480021FCF754F808B11C
:107DB000F9F7A6F80448FCF712F818B1BDE810402E
:107DC000F9F79EB810BD00BF184B002000440040DA
:107DD000B0B504466B480121A278E378257900F814
:107DE000341F61788272037645724170E168C16028
:107DF0002169417664494968896A8847002021469B
:107E0000BDE8B040FCF7F6BFB0B586B004465D48AB
:107E1000012200238DF80F30027262784272A2BBF9
:107E20002379E27803748DF810200B788D78C97867
:107E3000857443740176544D21694161217B8DF82D
:107E40001110A16805916968CA6A00F1080104A8C7
:107E500090476868806B10B1217E01B18047012096
:107E60002146FCF7C7FF0DF10F00FCF78DFE60798E
:107E700001280AD19DF80F0038B900200021012205
:107E8000CDE900006846FDF745F806B0B0BD00BF7B
:107E9000FEE7000070B58AB03A4D044600213A4E24
:107EA000284600F8341F617841707168896A8847F4
:107EB00002202146FCF79EFF20780C2813D00428CE
:107EC00018D0012829D106208DF8040001A8FEF75A
:107ED000D1FA02982863281DFCF76EFE607870B115
:107EE000FF20687111E06078B8B10AB0BDE8704059
:107EF000FCF73ABE01206876208968830DE00020F7
:107F0000687196F83100FCF7BDFF7068416A1D4842
:107F10008847607808B905F071FD0AB070BD00BFF0
:107F2000BCB50446174800226378A578027222780F
:107F3000437205740B788D78C97801766168437453
:107F40008574416142F004010F2906D00E49496849
:107F5000CA6A00F108010020904703202146FCF77F
:107F600049FF207807280CD10020CDE90000064801
:107F7000406CC068804720B9684600210122FCF7A8
:107F8000C9FFBCBD50000020F0020020FEE7000049
:107F90000D490A8810430880704700BF80B50A4821
:107FA000008830B1FFF734FC002818BF6FF00200E2
:107FB00080BD6FF0010080BD80B5034800210180C5
:107FC000FFF720FC002080BDDC1700208202810D1D
:107FD000002310464FF47A72F8F72CB900210022E2
:107FE00007F0A8BA01200021012207F0A3BAA06D72
:107FF00040F01000A065E06D40F00100E065012058
:1080000070474FF0B040016841F008010160DAE9C3
:108010000912036823F0F0031A430260206820F479
:108020007F4040EA0120206070474FF6FF72F36FF7
:1080300062EA01021A4042EA0141F16770474FF4D7
:108040007A70F9F75BB8012084F8240094F82500D1
:1080500001287047086820F0040008607047016834
:1080600021F002010160704729786A78AB78EE78D8
:1080700040EA0140296A40EA0220184340EA86505B
:10808000084395F8241040EA01607047FF22CA6057
:108090000021012280F82C1080F82D20704701204B
:1080A0001D4616460F466071204604F0F1BC20685C
:1080B00050E8000F216820F0100041E80002002A7B
:1080C00070472420C4F8840020680568026822F004
:1080D00001020260012284F88020826870471160EA
:1080E000116841F0010111600021202280F8401048
:1080F00080F841207047B1F8010000BA000CADF8DB
:108100000800704772185278D30943EA400070544F
:1081100001311046704702200021002240470846E6
:1081200011461A462346704702EB420200EB8200DA
:10813000407A00EB400001EBC00090F9021070475C
:1081400002200021012207F0F5B996F840005847B7
:10815000012304F063BF4FF0FF307047022000217D
:10816000012207F0E7B9014620460AF0A3BA2046EB
:108170004FF48071FBF74EB90220002100227047B6
:10818000012084F854002046F8F700BA3060FAF76E
:108190007BB80D4690F82C10044602200129704748
:1081A000D9F8000040F40040C9F80000204604F06F
:1081B00093BC012084F8480084F83E0084F83F0016
:1081C00084F8400084F8410084F8420084F84300B9
:1081D00084F8440084F8450084F8460084F8470099
:1081E00084F83D00002010BD2420C4F884002068DD
:1081F000016821F001010160204606F0CFBD206832
:1082000020210560002084F88000C4F88410B0BDEF
:10821000044690F8410020287047013091F8F12081
:1082200091F801315A4081F8F12070471019013856
:108230000860002010BD09F10201F8B2C9B2285C43
:10824000695C40EA012009F10301C9B2695C40EAB6
:1082500001406421704713460A46014670470022D8
:10826000002304F04BBE00200021002207F062B979
:10827000204601F0BDBDCA22CA605322CA600A6806
:108280007047016851E8021F026821F4000142E8CA
:108290000213002B7047204607F038BB29460AF02E
:1082A00009BA016841F0010101602046704704F5F8
:1082B000906184F88504D4F8440370470146284649
:1082C0000AF0F8B9002532463B4684F841004020C8
:1082D00084F842006564C4F824B06563A4F82A8079
:1082E0008846704730460AF091B804460068D0F8D6
:1082F0001CA001688268B4F86050D4F88830222B42
:1083000070472068616A406A0870608D0138608536
:10831000606A01306062208D411E21850904608DF4
:10832000704751460AF072B851E8001F026821F404
:10833000907142E80013002B70472046FCF7ECB91F
:10834000294609F005BE616A206811F8012B826296
:10835000608D013860856162208D411E2185090490
:10836000608D704753E8003F046843F0806344E841
:108370000035002D704759460AF048B828460AF0E3
:1083800099B904210162D4F88C0040F00200C4F8CD
:108390008C0070476064202084F84100002084F83D
:1083A000400084F84200704741460AF02FB802228C
:1083B0000262D4F88C2042F00402C4F88C2070478A
:1083C0004FF400610022F9F759BF002084F85400EF
:1083D000A06D40F00400A0650320BDE8F0810546D3
:1083E000D4F88C0041F288367047016841F00201F0
:1083F00001607047FF20F8600020226B84F82C0099
:1084000011432163012184F82D10704700200121C0
:108410006071A068A1710028704750E8020F2168C0
:1084200020F0400041E80202002A7047B3185B7850
:10843000DF0947EA4101B15401321946704709F199
:108440000300C0B2285C41EA002009F10401C9B26E
:10845000695C40EA0140642148437047012205F00D
:108460000BB8002004F0F8BE394609F071BD0122B6
:108470000262D4F88C2042F00102C4F88C207047CC
:10848000B0F85C10FBF7E5BC394609F0BFBF20200F
:10849000C4F88800C4F870B0E06E01287047214627
:1084A0000AF008B90027C16142681A40426084F8A6
:1084B000411084F8407084F842707047014630469D
:1084C0000AF0F8B8D1E90123C9681A4342EA012148
:1084D000826822F47F421143816081687047494677
:1084E00009F094BF886940F0080088617047002552
:1084F000C16142681A40426084F8411084F84050DB
:1085000084F842507047294609F080BF002084F863
:108510003C0020467047314609F078BFC36601230E
:1085200080F880300368A3427047044607F026BBFA
:10853000C9F800400760BDE8F88F214609F066BF22
:10854000B4F85C102046FBF784BC514609F000BD2E
:108550002046F7F7A7BF411B032002297047016897
:1085600021F00101016070470868894620F400404D
:1085700008602046704741E80202002A704704461E
:1085800090F8800001287047207A072295F875102E
:108590007047016000200021A06594F8560004F0A7
:1085A00078BE0146204609F0D3BC834699468A46E8
:1085B00000244FF001087047284609F027BF51E812
:1085C000001F026841F4807142E80013002B7047DD
:1085D000FF21FF224FF080732185009070470146F4
:1085E000304609F0B5BC2068416821F490414160F3
:1085F00081687047618D4FF0007321850090CAB289
:10860000704731460AF056B802F0010901F480784B
:108610004FF0000B7047414609F09ABC204606F027
:1086200013B984F84100102084F8420000206064EF
:10863000668560636562704780F88010016982F426
:1086400080520A4370472046FBF75DBF51460AF04F
:1086500031B8314609F07CBC012004F077B9012023
:108660000021012206F066BF044690F8540001285C
:1086700070473860F9F708BEF26F22EA114289B2FA
:108680001143F1677047CA21F9605321F9603968D5
:10869000AA6AB2F5807F7047D8F8000040F4004025
:1086A000C8F80000204604F017BA016851E8001F1E
:1086B000026841F0400142E80013002B704711436B
:1086C0008160204606F09EB894F8400003F091BD0A
:1086D0002046FDF7CFBE214600F11C05284607F0D5
:1086E00015B905463846394609F090BE191D03F103
:1086F00008020C331B88126809688381826041601C
:108700000020704701271E461546884684F84070B1
:10871000F9F7BABD2068290A3A46816220464146E7
:10872000FCF79FB8204609F071BE284609F010BC3E
:1087300001251F4616468A4684F84050F9F7A4BD25
:10874000204631462A46FBF7EDBE594609F0B2BF36
:10875000404609F0AFBF90F83C2004460220012AB1
:10876000704702400020062A7047608DB0F5807F78
:108770007047494609F09EBF28464FF400722146D3
:1087800007F012BE012084F854002046F7F752BFCC
:10879000C4F89000F9F778BD84F82C0057F80C0C59
:1087A00000F44079B9F5807F7047C2EBC202C2F392
:1087B0004C425A43704741E80002002A704794F83F
:1087C0004000012870470122FCF744BE4FF40051DD
:1087D0000160201D07F0E8B8D6E90007014609F05E
:1087E00015BE4FF07C5109F011BE608D51464FF01F
:1087F00000732085C2B2204600977047414609F0B9
:1088000059BF044690F83D0000287047384609F0EB
:10881000FDBD384609F09CBB268500972046514691
:10882000FF224FF080737047086840F00100086035
:1088300000207047608D41464FF000732085C2B222
:10884000204670474FF4807107F0C5BDA06D40F21F
:10885000011188430130A0650020704740EA0800FC
:1088600040EA060895F8240058472046314604F0AF
:10887000B3B8D4F8400320F02000C4F84003704798
:10888000012001F055BE394609F014BF2046FBF720
:10889000F3B92046FBF79ABA4A46FBF7C7BF002157
:1088A00084F83C10012184F83D107047012180F8C4
:1088B0003D1000207047FF224FF08073208500207C
:1088C0000090704700222B4609F02EB9002184F851
:1088D000541010BD21F40851396002217964B9F5B2
:1088E000807F70470446807901287047016851E80D
:1088F000021F026821F0010142E80213002B7047B9
:10890000D4F8400320F00200C4F84003704740F25E
:10891000FF1004F087BD214609F01ABB4FF4007028
:10892000606470472046FBF750BA3846BDE8F883CC
:108930004B68CA68194605F05DBD2068E9B200229F
:108940004346816220467047416841F4804141605E
:1089500070472046F7F740BE21F488513960012165
:108960007964B9F5807F70470868884620F4004034
:108970000860204670470220211D84F83D002068D1
:1089800005F000BD016851E8001F026821F01001E8
:1089900042E80013002B70471421F8F7DDB8504669
:1089A00006F8387F04F040B920464146FF224FF0D8
:1089B000807326857047204641463A46FBF751BFF3
:1089C000002084F840002046704702460B4609F01C
:1089D00003B8116821F0E071214370474AEA084169
:1089E00041EA0028A878584716F8011B204604F0F1
:1089F00021B8002084F880002046FBF721BC2046E7
:108A00004FF4004101221923FBF79CBE204606F0DB
:108A100095BF000010B5EE4C04F57E7006F0C4FF63
:108A200094F8140410B1012084F81304094890F854
:108A30000401022805D194F8850440F0200084F850
:108A40008504D4F8480320B1006910B1BDE8104096
:108A5000004710BD288700202DE9F0438DB078B382
:108A6000417802290AD0032914BF20A317A3FFF7D6
:108A700083FB0DB0BDE8F04306F05CBD837E90F84B
:108A800010E0B0F9128090F91490D0F804C0C568D5
:108A9000467D877DC47D017E427EC07E0A930A4B5F
:108AA000089109920B90022000210022CDE900E8F4
:108AB000CDE90295CDE904C6CDE9067406F03AFD8C
:108AC0000DB0BDE8F08300BF528401080D0A2323D6
:108AD0002323232320424541434F4E204E4F542011
:108AE00052454345495645440D0A00000D0A2323CB
:108AF0002323232320424541434F4E204C4F5354C0
:108B00000D0A0000E0B505A105A30022085C0021C4
:108B10000090022006F00EFD8CBD00BF41424300D4
:108B200053776974636820746F20436C617373209A
:108B3000256320646F6E650D0A000000FCF7C2BB60
:108B40007CB550B10446407940B118A3FFF714FB3F
:108B500002B0BDE8704006F0EDBC7CBD1A4D05F1D9
:108B6000380006F021FF1948FFF72AFC1E4E18A313
:108B7000022000210022B047A0791CA123A30128D4
:108B800008BF0B46022000210022B047A0794FF415
:108B90007A7168706868484300F0CEFB6868234BC0
:108BA0000021002200900120B0477CBD0D0A232344
:108BB00023232323203D204A4F494E204641494C40
:108BC00045440D0A0000000048030020000400484E
:108BD0000D0A232323232323203D204A4F494E45BA
:108BE00044203D200000000035F50008414250209F
:108BF0003D3D3D3D3D3D3D3D3D3D3D3D3D3D3D3DA5
:108C00003D3D3D3D3D3D0D0A000000004F544141BA
:108C1000203D3D3D3D3D3D3D3D3D3D3D3D3D3D3DA1
:108C20003D3D3D3D3D3D0D0A0000000046830108ED
:108C3000EF484FF40061F9F719BB00BF0120002194
:108C400006F0D6BD06A10BA3012808BF0B464DF8C0
:108C500008EDFFF791FA5DF808EB06F06BBC00BF7A
:108C60004E564D20444154412053544F5245440DDB
:108C70000A0000004E564D204441544120524553B5
:108C8000544F5245440D0A007F490876704700BF93
:108C90002DE9F0410F4F1C4615460E46804606F062
:108CA000D5FD3C757D823E82C7E90208387840F0E8
:108CB000080038700848D0F8480310B1006900B1C6
:108CC000804706A3022000210122BDE8F04106F002
:108CD00031BC00BF60020020D01200204D41432073
:108CE0007278446F6E650D0A000000003748017805
:108CF00041F002010170DD48D0F8480310B100696D
:108D000000B10047704700BF80B50A48017841F0C4
:108D1000010101700848D0F8480310B1006900B1A2
:108D2000804706A3022000210122BDE8804006F012
:108D300001BC00BF60020020D01200204D41432042
:108D4000727854696D654F75740D0A001CB506F094
:108D50007DFD0D4C6060684605F064F90B48DDE967
:108D60000012C0E9CE122178D0F8480341F010017A
:108D7000217010B1006900B1804705A302200021D5
:108D8000012206F0D7FB1CBD60020020D01200209B
:108D90004D4143207478446F6E650D0A0000000059
:108DA00080B50A48017841F0040101700848D0F804
:108DB000480310B1006900B1804706A302200021DA
:108DC0000122BDE8804006F0B5BB00BF6002002074
:108DD000D01200204D414320747854696D654F7561
:108DE000740D0A008AB2C44906F072BC10B5EB4C8F
:108DF00094F8240094F8251000EB800001EB40016A
:108E0000A948416094F826104D2904D14168C1EB6E
:108E1000011189000DE094F82610482904D1416819
:108E20004FF46162514304E094F82610532901D1B4
:108E30004168416041680B292CBF41680A214160AB
:108E4000417821B140684FF47A71484300E02068CE
:108E500000F072FA94F82200012813D194F8270048
:108E600003280FD194F8280008490870084994F89D
:108E700029000870074994F82A000870BDE81040DE
:108E800003F088BA10BD00BF00000020420000209F
:108E90004300002044000020B0B588B06D46044671
:108EA00020212846F7F7FEFABF492846202206F07F
:108EB0000FFC204629462022F7F753FA08B0B0BD30
:108EC000F0B587B000296DD0374D0C4606464FF4FB
:108ED000004101222846F9F7D1F9344F07F120006B
:108EE00006F02CFD0022002E46D02078002843D02A
:108EF0007068327800283FD0022A0ED0142A18D089
:108F0000032A39D17178012935D1007802282DD072
:108F100001282DD078BB00202BE096F901300222E9
:108F2000D9B2012928D0002B26D406F013F9022249
:108F300022E07178012917D1007810F00100F87053
:108F400008D11EA30320FFF749F828464FF400611B
:108F5000002207E016A30320FFF740F828464FF44D
:108F600000610122F9F78AF9142205E0022000E0ED
:108F70000120FBF787FF0322207C052812D8E16837
:108F800094F9083094F9095094F90A40CDE9045451
:108F90000DA454F8200003908DE80E00104B032020
:108FA000FFF71CF807B0F0BD00040048480300209C
:108FB0004C4544204F4E0D0A000000004C45442013
:108FC0004F46460D0A000000A9850108AB8501083F
:108FD0006A860108AD85010872860108B28501081C
:108FE000D5840108EB484FF400410022F9F746B957
:108FF00000040048CC490020A1F8CA0391F81504E8
:1090000081F8B803C94890F8612090F8753090F85D
:10901000800081F8C90381F8BB2381F8C83301F5CA
:10902000607001F56E7103F075B900BFEF4991F8FA
:109030008404C8B14FF48070A1F8DE0391F81504E0
:1090400081F8CC03E848426EC1F8D02390F875202F
:1090500090F8800081F8DD0381F8DC2301F566706B
:1090600001F5737103F056B9704700BFD0120020AC
:10907000B0B5C348807818B90820002106F0B8FBC5
:10908000C44C0A4D4FF4004100222046A847204618
:109090004FF400710022A84720464FF400610022DF
:1090A0002B46BDE8B0401847480300207D22000849
:1090B000B0B50C460546F8F76DFF00B1B0BD3848B5
:1090C00038490022006801EA80204FF47C31B1FB6E
:1090D000F0F148430121C0F57C30C00AF7F714FFD6
:1090E00028B90548294622460023F7F725FFBDE8A1
:1090F000B040F8F70BBF00BF00F0030810B588B010
:109100006846182100F10804FFF722FA9448032169
:1091100080F827104FF4B441ADF8001001218DF80C
:10912000031090F822108DF8021090F824108DF89A
:10913000041090F825108DF8051090F826108DF881
:10914000061090F827108DF807100021032905D08C
:10915000421892F8282062540131F7E7F8F71AFF15
:10916000C8B90F480F490022006801EA80204FF477
:109170007E31B1FBF0F148430121C0F57E30C00AD9
:10918000F7F7C2FE28B90848694620220023F7F7FE
:10919000D3FEF8F7BBFE08B010BD00BF00000020F2
:1091A000E075FF1F00FCFF0300F8030880B5FBF724
:1091B0002BFD18B9FBF7AEFD012800D080BD06F0ED
:1091C00053FC0000BFB588B30446007870B31C4858
:1091D0004FF400710122F9F751F81A48083006F0EF
:1091E000ADFB264D18A3FEF7C7FFA847E068217C1A
:1091F00094F90A2094F918308DE80F0020A3032079
:1092000000210022A8472BA3032000210022A84709
:10921000207A01280BD1607A30A22EA1304B002891
:1092200008BF0A4600920320FEF7D8FEBFBD25A363
:1092300003200021002204B0BDE8B04006F07AB956
:1092400000040048480300200D0A2323232323237E
:10925000203D3D3D3D3D3D3D3D3D3D204D43505339
:109260002D436F6E6669726D203D3D3D3D3D3D3D38
:109270003D3D3D3D3D3D0D0A0000000035F5000837
:1092800023232323232320552F4C204652414D4591
:109290003A25303464207C20504F52543A256420C3
:1092A0007C2044523A2564207C205057523A256451
:1092B00000000000207C204D534720545950453A6F
:1092C00000000000554E434F4E4649524D45440D57
:1092D0000A0000004E41434B0000000041434B0098
:1092E000C484010810B59C4C04F55A7006F05CFB70
:1092F000FFF7BFFA012004F00FF908B10B2800D1E5
:1093000010BD092084F83904944890F8390084F895
:109310003A0494F8120484F83D040920FCF74AFA50
:10932000BDE8104004F0A2BDD01200202887002024
:109330000B49C873704700BFB0B5094D114C0028E8
:1093400008BF42F210702860204606F02DFB296805
:10935000204606F0DBFA2046BDE8B04006F0EEBA43
:109360000000002080B50648012101700220002184
:1093700006F03EFA0348BDE8804006F0DFBA00BFC1
:10938000480300205419002002484FF400710022C5
:10939000F8F774BF000400487CB5704E6E4D736CD6
:1093A00096F8482096F9701096F8400005F5787404
:1093B000009402F0B9FE40F2012005F584622146D6
:1093C000A5F8F20396F8400002F0EEFE58B195F8C9
:1093D000200485F862040648416B0020884795F810
:1093E000F30385F884047CBD28870020D012002078
:1093F0004C290108704780B5FAF750FB0020012185
:10940000BDE88040F9F7A8BA80B5FAF747FB0448F1
:10941000012101600120BDE88040F9F77BBA00BF5F
:10942000880400587047FAF735B9000080B5FAF79C
:1094300031F908F0EDF9FEF7E5FBFEF75DFC0448B5
:10944000F8F77CFF0348BDE88040FAF77FBB00BF18
:109450003C4A0020CC4A00202DE9F04F89B000287A
:1094600053D08A460646DDE9121000244FF0010869
:109470009146CDF80D400494CDF80940CDE907445C
:10948000CDE90544CDF805408DF804808DF80A300B
:109490008DF80910010E8DF80E008DF81110010CD9
:1094A000000A8DF80F00180E8DF810108DF80D00C1
:1094B000180C8DF80C00180A8DF80B0005AF0FFA88
:1094C0008AFBBBF1010F22DB8DF8138001A810216C
:1094D0004A463B4604F080F9D8B9BBF1100F4FF073
:1094E0001000A8BF834608F10108E0B20021CAB20B
:1094F000934506DDBB5C02440131B55C6B40B3545F
:10950000F5E71034AAF1100AD9E70A2002E000209A
:1095100000E00F2009B0BDE8F08F704710B50E4C89
:10952000D4F8400340F08000C4F8400394F81404D9
:1095300010B10020FFF76EFA94F8850440F0220085
:1095400084F88504054890F80401022818BF062015
:1095500084F8840410BD00BFD012002028870020AA
:109560002DE9F04F93B012A9044604F097F90028B2
:1095700048D1042C07D825A3DFE804F00E03090B1B
:109580000D0040A308E07F2C0BD126A304E031A3FB
:1095900002E036A300E029A302200021002205F00A
:1095A000C9FF1298817990F801E090F8028090F854
:1095B000039090F804A090F805B090F808C0827A63
:1095C000C37A047B457B867BC77B1191C17910915F
:1095D000417A007C09920A930B940C950D960E9794
:1095E0002E4B002208910F90CDE900E802A800213F
:1095F00080E8000E119805901098CDE9060C022025
:1096000005F098FF13B0BDE8F08F00BF232323239C
:109610002323204170704B65793A202020202020A0
:1096200000000000232323232323204D434B454BDD
:1096300065793A20202020200000000023232323E6
:109640002323204D43526F6F744B65793A202020BD
:1096500000000000232323232323204E776B534B4A
:1096600065793A20202020200000000023232323B6
:10967000232320417070534B65793A20202020200D
:1096800000000000232323232323204E776B4B6508
:10969000793A2020202020200000000012860108B6
:1096A0002DE9F04F93B04FF00008054602F03F005F
:1096B000DFF8ACB4DFF8B0648A46002707908DF875
:1096C0004B80ADF848800EAC00200890B946FFB240
:1096D000574580F03F82E85DFBF708FF384450456E
:1096E00000F23882E81901780239112900F2328239
:1096F00009F10107DFE811F01200240128007D01C3
:109700003500400067007C00C0002E022E02BE0122
:109710002E022E02DE00F20006010F020420FCF7EA
:1097200011F80028D2D000200421FCF733F8F8B259
:1097300009F10307285C8BF8540409F10200C0B258
:10974000285C8BF85504C1E7F8B20121285C00F0D1
:109750000F0086F8070101FA00F0A6F80A010420BC
:109760003FE0DBF84803002800F0E38101680029AE
:1097700000F0DF818847DDE1032009F102010B944D
:10978000CDF83C808DF84B00F8B2C9B2285C695C1A
:109790008DF8300009F10500C0B2285C8DF840005A
:1097A000FEF74DFE0E9096F840000BA902F0EBFC80
:1097B00009F1060700288DF84B003FF587AF8DF8BB
:1097C0004800072052E1F8B24FF47A72285C10F09A
:1097D0000F0008BF013010FB02215043C6E91401FD
:1097E000082012A90022FBF735FE09F102076DE7F8
:1097F000F8B28DF82C80285CC0F340118DF82D1044
:10980000C10602D501218DF82C1000F00F0009F1DE
:1098100002078DF82E0096F840000BA902F0E3FC39
:1098200001303FF453AF9DF82D009DF82E10A14656
:109830009DF82C4086F87500CCA086F87440405CFA
:1098400008F068FDB067022049468DF83A404C4662
:109850008DF8380096F8400002F076FC96F9391041
:1098600040B28842B8BF084686F8390012A90920DC
:109870000022FBF7EFFD29E7032009F102018DF833
:109880004B00F8B2C9B2285C695C8DF83800FEF76D
:10989000D6FD21460F9096F8400002F04FFC09F1EA
:1098A000050700288DF84B003FF510AF8DF84800F4
:1098B0000A20DBE00D20FBF745FF00283FF406AF50
:1098C00000200D21FBF766FF9BF8840400F0FE00EA
:1098D00004283FF4FBAEFBF7B0FDF7E6FEF7ABFC68
:1098E000414309F10400C0B2285C00F00F00FBF70F
:1098F000A2FD8DF84800112012A9FEF764FF09F1BE
:109900000507E3E60E20FBF71DFF00283FF4DEAE5F
:1099100000200E21FBF73EFF09F10201F8B28F4A49
:10992000C9B2285C695C926840EA012009F1030130
:10993000C9B280B2695CFBF76BFD09F10407C5E6AB
:1099400008998DF82C808DF837808DF836808DF849
:109950003580C90740F0FB800F90AAEB090096F80C
:10996000381096F8392096F860308DF8400096F857
:1099700006018DF84410D6F814118DF845308DF895
:1099800043200DF137038DF8420096F874000E91D4
:109990000DF136018DF8410000910DF1350196F879
:1099A0004000019121460BAA02F0E1FB8DF84B002B
:1099B00000F0070007280BD19DF82C0086F839002D
:1099C0009DF8370086F838009DF8360086F860006C
:1099D00000279DF835000521FAB2B0FBF1F1914264
:1099E00040F2B38003200DF14B01FEF7ECFE01378E
:1099F000EFE707208DF84B00F8B2285CC0F30211A6
:109A000000F00F008DF8391009F102018DF83800CF
:109A100009F10300C0B2C9B2285C695C41EA0020C8
:109A200009F10401C9B2695C40EA0140642148437C
:109A300021460F9096F8400002F0BDFB00F00701B0
:109A400009F105078DF84B0007290CD19DF8381056
:109A50009DF8392086F8701086F868100F9986F8FE
:109A60006120F16671668DF84800052012A9FEF7A5
:109A7000AAFE2BE60A20FBF765FE00283FF426AE7F
:109A800000200A21FBF786FE09F10500C0B2285C20
:109A9000069009F10400C0B2285C039009F10300AC
:109AA000C0B22E5CF8B22F5C09F10200C0B215F80A
:109AB0000080204604F0B6FA0E980399069A0590A5
:109AC0000F980490DBE9CE30009047EA08204FF071
:109AD000000840EA0640244E40EA01602149014462
:109AE0004FF47A705043020A09A804F0E7FADDE95E
:109AF0000930DDE904210090204604F065FADDE933
:109B00000E0104F0BBFAFBF784FC012009F1060703
:109B10008BF83404DAE5FEF78EFB4843FBF775FC5F
:109B20008DF84800132012A9FEF74DFE09F1040735
:109B3000CCE5FF2007998DF84800062002228DF819
:109B4000491012A9FBF786FCC0E500EB09070120CC
:109B50000890BBE513B0BDE8F08F00BF60020020A5
:109B6000D0120020803DD51228870020080A0C0D55
:109B70000E10121415181A1B1D1E212410B5F7F70C
:109B8000CDF81148006808F0C5FB104C214608F0DC
:109B90003DFC08F087FB0E4908600E48006808F09D
:109BA000B9FB214608F032FC08F07CFB0A4908604A
:109BB0000A48006808F0AEFB214608F027FC08F0D0
:109BC00071FB0749086010BD6C31002000007A402D
:109BD000C801002070310020C40100207431002031
:109BE000C0010020032816D8B0B5C5004FF480701E
:109BF000274C4FF48071E840C2B22046F8F73EFB94
:109C000006484FF40051E840C2B204F58060F8F70E
:109C100035FBBDE8B0400020704700BF00000101E7
:109C20001621002808BF0F21084670470220704700
:109C300070B586B0002402200594FAF765FE042072
:109C4000FAF762FE0320CDE903400120104C029098
:109C50004FF48070019001AD20462946F8F742FA92
:109C60004FF4005004F58066294601903046F8F71D
:109C700039FA30464FF400510022F8F7FFFA204637
:109C80004FF480710022F8F7F9FA002006B070BD99
:109C900000040048012070470020704770B53C2147
:109CA000234A01EA9000204908582049096801F038
:109CB0000F0152F82110B0FBF1F01E49B0FBF1F496
:109CC000F8F73CFEB0F5007F09D11D4900200328BC
:109CD0000FD031F8102094420DD90130F7E7164922
:109CE0000020032805D031F81020944203D9013018
:109CF000F7E7002502E0114951F82050114E306875
:109D000020F007002843FEF741FA0446306800F0CF
:109D10000700A84206D0F8F7B7FA001B0328F5D3CE
:109D2000032070BD002070BD0C29010808010058F7
:109D3000D027010840420F00A4270108AC270108E2
:109D40009E2701080040005870477047FEF703BA8D
:109D50000020704700207047FEF7FDB9FEF7FBB901
:109D6000704770477047FEF7F6B9FEF7F4B9000088
:109D70000148F9F733BB00BF884A00200928014693
:109D800098BF0921CAB20A23B2FBF3F202EB8203A5
:109D9000A1EB4303591A084440EA0210C0B27047CD
:109DA0002DE9F041114E80463068400619D43068E4
:109DB0000027012440F080003060F8F765FA05467E
:109DC0003068E14341EA9010C0070BD1F8F75CFA24
:109DD000401BB0F57A7FF3D90327002488F82D7053
:109DE000EEE70027F8B2BDE8F08100BF0C28004084
:109DF000B0B5124D044655F80C0C20F0800045F823
:109E00000C0C2868800606D4F9F72CFC70B10320EE
:109E100084F82D00B0BD286820F020002860F9F7F4
:109E200021FC28B1032084F82D0002E00020B0BD01
:109E30000020296841F020012960B0BD18280040A9
:109E40000120704780B502F001FF0438C0B203283A
:109E500005D80449C00021FA00F0C0B280BD00203E
:109E600080BD00BF0201000380B502F043FF033054
:109E700080BD0000F8B5F94EEA4F00253446BD65B7
:109E8000C7E901557D7001C4184802F08FFFBD81FC
:109E900003F041F90020002102F0F9FF0120002128
:109EA000042203F049FA4FF6FF704FF6FF71FEF7F8
:109EB000D6F900F0F9FF0E4B20464FF0FF3100229B
:109EC000009505F0A9FC009506F11C05094B4FF023
:109ED000FF310022284605F09FFC204605F064FD76
:109EE0002846BDE8F84005F05FBD00BF19A2000894
:109EF00041A2000829A200087CB58D4C00208DF8F5
:109F000007000090B4F85400411E072927D91028F3
:109F100000F0B080202800F0AF80402800F0BE8024
:109F2000802800F0C780B0F5807F00F0CC80B0F5CD
:109F3000007F40F0E68091A3FEF710F902F086FE64
:109F4000042840F0CA80C4487E4CFEF73FFCFEF770
:109F500088FA2068002800F0D4804068CFE0DFE86D
:109F600001F00416D052D0D0D07FBB48754CFEF71C
:109F70002DFCFEF776FAFFF7EDFE012808BFFFF78C
:109F8000E4FE2068002800F0BC800068B7E0B2481A
:109F90006C4D4FF48051016005F11C0005F004FD8B
:109FA000607880B9FEF75DFA40F60210002103F0F8
:109FB00071FA40F6441002F045FF40F0020140F60D
:109FC000441003F067FA72480DF10701FF2202F016
:109FD00079FE04F1240002F03DFE2868002800F01C
:109FE00090808668002E00F08C8094F82400012870
:109FF00040F0888094F9313094F930209DF80710B2
:10A000006348B0477CBD59A30220002101220025EE
:10A0100005F090FAA06D002873D0574EC0F30741A9
:10A0200040F60310B04794F8591040F60410B047BA
:10A0300094F8581040F60510B04740F6021002F0B0
:10A0400001FF40F0010140F60210B04740F26220EB
:10A0500040F2622100220023A56502F04FFF7CBD83
:10A060003FA3FEF77BF8FFF773FE012849D1FFF706
:10A0700077FE7CBD37A30EE0324D05F11C0005F0E4
:10A0800093FC607808B9FEF7ECF92868C8B3C0689B
:10A09000B8B380472CA3FEF761F87CBD25A3FEF77B
:10A0A0005DF8607808B9FEF7DCF92648006840B32F
:10A0B000006924E0FEF7D5F92248006808B38169F9
:10A0C000F9B1002007E0FEF7CCF91E480068C0B1E6
:10A0D0008169B1B1012088477CBD02F0B7FD052838
:10A0E0000FD15D48174C4FF48051016004F11C0002
:10A0F00005F05AFCFEF7B5F9206810B1C06800B150
:10A1000080477CBDE06B694602F050FD00984FF43B
:10A110007A7194F9292000F5FA7090FBF1F09DF81E
:10A12000071043B228688468EE48A0477CBD00BF92
:10A13000EC1800204952515F4352435F4552524F41
:10A14000520D0A0084020020484452204B4F0D0A51
:10A1500000000000484452204F4B0D0A0000000050
:10A1600053594E43204F4B0D0A00000050524520DA
:10A170004F4B0D0A0000000095D400084952515F72
:10A1800052585F54585F54494D454F55540D0A007D
:10A19000DF1700202DE9F0418AB01C46154688469D
:10A1A000074600F08AFE0020002600F0C1F938467C
:10A1B00002F0C2FF012041464FF416720023CDE9A0
:10A1C00008600320CDE900800020CDE90266CDE9DA
:10A1D0000466CDE9066600F0F3F9002000F052F8BD
:10A1E000FFF742FEF7F701FE05F030FB064630466A
:10A1F00005F036FB0746A04203D202F0AFFDA842AD
:10A20000F5DD0025A74228BF012500F056FE2846AF
:10A210000AB0BDE8F0810000E849A1F85400FFF75A
:10A220006BBE00BFEC1800200B484FF4805101605A
:10A23000B448006810B1C06800B10047704700BF63
:10A2400005484FF400510160AE48006810B1406805
:10A2500000B10047704700BF280400488402002076
:10A2600080B500200021FDF7FAFFBDE8804002F034
:10A2700043BD02F0E7BD02F0F1BD80B502F06EFD16
:10A2800080BD0000B0B50446FFF762FD012802D191
:10A29000FFF762FD05E040F2622040F26221FDF727
:10A2A000DEFF2CB19748FEF716FA284605F046FB6C
:10A2B0008A484FF48051C14CFEF76BF961786FF01A
:10A2C0007F40A268002908BF9001BDE8B04002F0BD
:10A2D00063BF00BFB0B50446FFF73AFD012802D1C5
:10A2E000FFF73AFD05E040F2622040F26221FDF7FF
:10A2F000B6FF2CB18348FEF7EEF9284605F01EFBA9
:10A3000076484FF48051AD4CFEF743F961786FF019
:10A310007F40A268002908BF9001BDE8B04002F06C
:10A320004FBF00BF2DE9F84F8B46814640F2012018
:10A3300040F20121FDF793FF68484FF40051DFF828
:10A34000A0810160012198F8560002F0A2FF98F860
:10A35000000098F8511081F0060180F0010050EAE9
:10A36000010640F6890018BF012602F06BFD00F0DF
:10A37000FB0040EA860140F6890003F08BF898F86C
:10A380000000042800F29180DFE800F003150318B4
:10A390001F00FFF7DDFC012824D10DF10302484620
:10A3A0005946FFF7E0FC002800F08B804FA3FDF733
:10A3B000D5FEBDE8F88F88F81FB015E002214046B1
:10A3C00000F80E1F80F80CB010E0464800215A46F5
:10A3D0004B468AB11E78013AF64303F8016B00F848
:10A3E000011BF6E788F816B008F10E0002F026FE11
:10A3F00048465946002256E03A4E4FEACB07002025
:10A4000007210022974215D0C2F3C70421EA0203B4
:10A41000013219F8044024FA03F321EA020403F09C
:10A4200001035840C3B2A340C2F3C704355D2B43B8
:10A430003355E7E7C10145460BF1010941EA8011B7
:10A44000C0B2B0FA80F0400941EA401006F80B00B3
:10A45000022005F80E0F284685F80C9002F0EEFD5C
:10A46000DFF884A0F1200021D047F0200021D04760
:10A47000D5F83A40E121642C08BF7021F320D04781
:10A480000421642C08BF1D21F220D0474FEA5B1144
:10A49000F420D047B81CC1B2F520D0475FFA89F14B
:10A4A00030466FF07F4202F0E9FC1648D8F80410FD
:10A4B000041D204605F02AFA204605F03FFABDE8C3
:10A4C000F88F9DF8030088F8160008F10E0002F0DE
:10A4D000B5FD9DF8031048468CE700BF18040048FE
:10A4E000EC180020DF17002095D400085261646941
:10A4F0006F53656E64204F76657273697A650D0AD5
:10A50000000000008402002002F016BE012802D1E3
:10A51000DA48C17705E0D948427D012A18BF704763
:10A520008175C5480170D5480E3002F087BD00BF67
:10A53000B0B5D24D04462870FFF714FC052C14D892
:10A54000DFE804F0050B1303030502200EE00020F2
:10A55000002402F0C7FD6C7306E0012002F0C2FD8A
:10A56000287B697B814206D1B0BD032002F0BAFD91
:10A5700000206873B0BD6873002818BF0120BDE8D3
:10A58000B04000F001B800BF10B50446BB484473AA
:10A590000473FEF775F914214FF4E860002C18BF1E
:10A5A000342102F077FF242140F24170002C18BFC3
:10A5B0004421BDE8104002F06DBF00BFEC18002040
:10A5C0002DE9F04F85B0DDE91185DFF87CBA179CE5
:10A5D0001F4691468A4606468BF80140B8F1000FA7
:10A5E00008BF4FF0FF35FFF7AFFB9349002C1098E1
:10A5F0000F9C0D7018BF0020002E6AD0012E00F0B5
:10A60000B080052E40F0148100900120884602F0B1
:10A6100037FE092000275E468BF844004FF448704F
:10A62000CBE90F90FEF7BBF95D4605F80E7F85F884
:10A6300037004FF480506860E00068800120A5F882
:10A64000090098F8000028720520FFF771FF3046D6
:10A6500002F08CFC284602F0F1FC42F2B270CDF818
:10A660000E70ADF81270ADF80C0003A802F027FED2
:10A67000FEF74DF9724E40F6B800B047714D00F04C
:10A68000EF0140F6B800A84740F6B9000421A847FA
:10A6900040F69B00B04700F0E30000F1080140F6EF
:10A6A0009B00A84740F2D160B04740F0180140F24B
:10A6B000D160A84740F2AC60B04700F08F0000F1D5
:10A6C000500140F2AC60A84700994FF4FA5048435B
:10A6D00044E004460020002702F0D2FD0B205E4635
:10A6E000CBF83C908BF84400FEF759F95D4613997E
:10A6F00005F80E7F85F8370088F00100AF71E8712A
:10A7000041F60400A8800F98C00068800120A8725C
:10A71000002918BF6FF00D00687247480078287252
:10A7200000F0CBFB0020FFF703FF304602F01EFCD9
:10A73000284602F083FCC120CDF807708DF80B701D
:10A740008DF8060049F2C140ADF8040001A802F0FE
:10A75000B6FDFEF7DCF84FF4FA506043B0FBF9F0B9
:10A7600064E0009000205D464FF0000B02F088FD91
:10A77000324901202E4622468AF0010306F8380F9E
:10A780000C2C11F80A10B77686F8189006F81A8C77
:10A7900071766FF0040198BF0C2251FA89F10229F9
:10A7A000169928BF224626F81C2C344689F00C0244
:10A7B00006F8171C139906F8181C1F49097806F8A3
:10A7C000191CA9F10B01022938BF4FF0010BBAFA8D
:10A7D0008AF104F82A0D1A434909B2FA82F201EA11
:10A7E0000B01AB4652091143F17600F066FBFEF710
:10A7F00047F8304602F0BAFB204602F01FFC0098F2
:10A80000C0B202F096FB16F8170C441E40F23670E8
:10A8100018BF012402F016FB00F0FB0040EA84019F
:10A8200040F2367002F036FE4FF6FF70CBF80800AB
:10A8300005B0BDE8F08F00BF4001002030280108BE
:10A8400045CE000895D4000870B5EB4E054601EBE7
:10A8500040000C464FF6FF7100220023B0654FF612
:10A86000FF7002F04BFB96F85600002102F011FD3C
:10A8700028462146BDE8704002F0BCBCEC18002020
:10A880002DE9F04387B000279846154689460646CD
:10A89000CDE90477FFF758FAD74C002D18BF0125F2
:10A8A000657018BFB846012E40D0002E40F0B88029
:10A8B000D9F80800002800F0B180D9F80C00002871
:10A8C00000F0AC8099F81E20082A00F2A780D9F881
:10A8D000101004A804F0FCFED9F80000002818BFEE
:10A8E000012002F0CDFC002584F83850D9E901019F
:10A8F000E16399F8201084F8441002F095F984F887
:10A900004500A57399F81F2099F8213099F81E1079
:10A9100099F82200A2742375C900B9F80C20E174DB
:10A92000D200002822825CD0FF215CE0B9F8300020
:10A93000002873D099F8320001280CBFD9F81450C0
:10A94000FF25D9F82800002818BF012002F098FC44
:10A950005FFA88F002F0EDFA012084F8380099F8E7
:10A960002C1099F82F0084F850100228B9F82D20E7
:10A97000A4F8512005D306D10B390020022938BF95
:10A98000012084F85300012004F80E0FB9F83000BC
:10A990006574E08199F832002074B9F8340060825F
:10A9A00000F08BFAFDF76CFF04F12A0002F0DEFAEA
:10A9B000204602F043FBE07C451E40F2367018BF93
:10A9C000012502F03FFA00F0FB0040EA850140F269
:10A9D000367002F05FFD4FF6FF70002744F8060C5A
:10A9E0001EE0D9F81410A17599F82410022918BF97
:10A9F000022819D199F82300A0F1F101022901D30D
:10AA000001280BD18D4A0025CDF808908DF80C5007
:10AA100052F81C1B01A8FFF799F958B14FF0FF3706
:10AA2000384607B0BDE8F083607599F823002176B9
:10AA3000E07503E001206575A4F8170000F03DFA09
:10AA400000200027FFF774FD04F1380002F08EFAB1
:10AA500004F10E0002F0F2FA04A802F030FCB9F89A
:10AA60001C0002F0DFFCB9F8180002F027FA4FF4DE
:10AA7000FA50D9F8081008FB00F0B0FBF1F0A06024
:10AA8000CEE700BF2DE9FE4F1D4617468846044617
:10AA9000FFF75AF9149EDDF830A0042C4DD0DDF8F4
:10AAA0004090DDE90EB3012C55D0002C40F0998088
:10AAB000FB4E0B2086F844002846C6F83CA04FF019
:10AAC000000A34461D4604F838AF02F0ADF806F827
:10AAD0000EAF86F837000120C6F83270B072B9F1B7
:10AAE000000F18BF6FF00D00707286F806A085F099
:10AAF0000100F07141F60400B0804FEACB00708095
:10AB000000F0DBF90020FFF713FD204602F02EFADB
:10AB10003046149E02F092FAC120CDF807A08DF8BD
:10AB20000BA08DF8060049F2C140ADF8040001A861
:10AB300002F0C5FBFDF7EBFE53E00420FFF7F8FC45
:10AB4000E848022100F8381F16210175C0F810A04E
:10AB500002F00CFA45E03746E24E012013990D9AB7
:10AB6000BBF10C0F06F80E0F86F84420234AF1744F
:10AB70002349337486F842A086F8129085F00103C9
:10AB80003446525D097886F8432071746FF00401F1
:10AB90005A4651FA8AF198BF0C22022928BF5A4618
:10ABA000F281AAF10B0100220229B5FA85F138BF22
:10ABB000012204F82A0F490911408AF00C021A43B5
:10ABC000B2FA82F25209114386F8451000F075F985
:10ABD000FDF756FE204602F0C9F930463E4602F027
:10ABE0002DFA404602F0C4FABE4C84F85600FFF736
:10ABF000B8F86660BDE8FE8FEC1800203028010828
:10AC000040010020B0B514460D4602F095FA2846E2
:10AC100002F0AEFA012102F03CFB4FF47A7044439B
:10AC200002F080FB9F482146051D284604F06EFE79
:10AC30002846BDE8B04004F081BE00BF8402002079
:10AC40002DE9F04387B0074600201C4615460E4606
:10AC5000CDE90400FFF778F8032F00F21481DFE854
:10AC600007F0024384983068002800F0DF80B27C4F
:10AC7000082A00F2DB80B16804A804F029FDF24F35
:10AC80000020042287F838003168B873F963F17C3A
:10AC900087F84410B1693964B188BA74C90039823F
:10ACA000B17C3875C800F874B07D022803D0307DBF
:10ACB000022840F0BE80707DA0F1F101022902D38C
:10ACC000012840F0B380774A4FF0010801968DF8D3
:10ACD0000C8002CA01A8FFF739F8002840F0A680CE
:10ACE000A7F817800020A9E0D74F012087F8380087
:10ACF000307887F85000707887F85100B07887F87E
:10AD00005200F078022807D308D13078A0F10B0167
:10AD10000020022938BF012087F85300012007F8DE
:10AD20000E0FB088F881B0793874F079B874307A41
:10AD3000F87400F0C2F8FDF7A3FD07F12A0002F055
:10AD400015F9384602F07AF997F8436040F6890021
:10AD500002F078F8062E0CBF00F0FB0140F0040171
:10AD600040F6890002F096FB8DE0306800285DD047
:10AD7000B0F57A7F5AD80320FFF7DAFBB2480221F8
:10AD8000162200F8381F31680275016102F0EEF8F2
:10AD900079E0B27C082A49D8B16804A804F098FC8C
:10ADA0003068002842D042F2107188420CD8A64880
:10ADB00003214FF0020880F8381081733168C163B5
:10ADC000F17C80F844100EE09F484FF0000880F8B6
:10ADD000388080F80E803168C163F17C80F84410BF
:10ADE000316889080164B088974F0421B974C000A4
:10ADF00000213882B07C3975C000F874B07D02281B
:10AE000002D0307D02281ED1707DA0F1F10102290F
:10AE100001D301280AD1234A4FF0010901968DF888
:10AE20000C9002CA01A8FEF791FF90B14FF0FF30DD
:10AE300033E0707DF875B07D3876307D787500F040
:10AE40003CF800200CE0707DF875B07D3876307DE0
:10AE500002E0A7F817900020787500F02EF8404621
:10AE6000FFF766FB07F1380002F080F807F10E00EB
:10AE700002F0E4F804A802F022FA308A02F0D2FAD2
:10AE8000B08902F01BF8284602F072F96E4D85F881
:10AE90005600FEF766FF6C60002007B0BDE8F08347
:10AEA000EC1800208402002080B5042002F0BEF9D6
:10AEB0000220BDE88040F6F798BF002002F0CCB930
:10AEC00080B56148002190F8560002F0E2F94FF495
:10AED000C0704FF4C071FDF7C2F9BDE8804001F0C9
:10AEE000E3BF00BFEC180020F0B50DF1140C089E74
:10AEF00001289CE8901010D000285FD10CEB0400D2
:10AF0000002E18BF02302021002F18BF182101EB9E
:10AF1000C0004FF47A71484352E019B9A2F10B0016
:10AF2000022804D30020012908BF0C2A00D10120E7
:10AF30001425002F18BF0025A5EB8205002E6FF009
:10AF4000070618BF1035072A05EBCC0528BF0835C2
:10AF50009700002818BF06EB82070C26072A38BF87
:10AF600097003846002DC8BF284401380C250C2C0A
:10AF700090FBF7F088BF2646571F022F28BF2646B2
:10AF8000072A38BF0E25AC190433023A00FB0340F0
:10AF90008000013090404FF47A725043174A515C60
:10AFA00000220A290CD8DFE801F006101316191B3D
:10AFB0001D0B1F22250041F6846201E001220020C2
:10AFC00010440138B0FBF2F0F0BD43F60952F7E748
:10AFD00047F61222F4E74FF22442F1E70A4AEFE77C
:10AFE000084AEDE7064AEBE742F6B102E8E745F228
:10AFF0006112E5E74AF2C322E2E700BF3028010808
:10B0000020A1070090D0030048E8010080B502F0BD
:10B01000AFF8012102F03DF9BDE8804002F082B9AD
:10B0200080B50948012190F8560002F032F94FF43A
:10B03000D7602D2102F02EFA02F079F90348BDE81D
:10B04000804002F059B900BFEC180020FFFF0F004C
:10B0500002F020BA02F02ABA10B50446FEF71AFE32
:10B06000012818BF10BD40F6231001F0EBFE00F0E0
:10B07000F90040EA040140F62310BDE8104002F058
:10B0800009BA022070472DE9F04F87B004465020DE
:10B090008DF818002079102802D12068C07B10B1EB
:10B0A00007B0BDE8F08F022700254FF064090DF1CD
:10B0B000100A0DF108080DF1040B00260F2FEFD830
:10B0C000072F17D22068815D30440491427841EA0D
:10B0D000022104918078059541EA004000FB09F1C6
:10B0E000049158B140468DF80C70CDF808A000F0DE
:10B0F00039F808E08DF81850CDE9045558468DF818
:10B10000047000F083F801370336D7E707A301384E
:10B110009A56B0FA80F04009891AB1EB400FB8BFD7
:10B1200041000529A8BF0521C8B2704700010203EC
:10B130000405FFFE10B50179012905D079B9DF4971
:10B14000096801F5906203E0DC49096801F28C426C
:10B15000016810460122012400F0B6FC00E0002442
:10B16000204610BDF8B50579022D01D20620F8BDA4
:10B170000F2D01D90320F8BD0446006800210722E5
:10B180000026007A40F3030000F0C6FFB0FA80F01A
:10B19000002107224709206890F90800001100F0FB
:10B1A000BBFF2168B0FA80F0400991F908203843CC
:10B1B00042F30303B3EB221FC8BF0126064308680E
:10B1C00004F028FC01460620002918BF0520002EA7
:10B1D00004BF05200420C6B991F0010115D1B74F75
:10B1E00005EB450621680C22386800EB860006F066
:10B1F00034F83968002001EB8602B1F880345072CF
:10B200000122AA401A43A1F88024F8BD017802293E
:10B2100001D200207047A94801EB410200230068D9
:10B2200040F8223000EB820200F5906013815360F9
:10B23000102200F02CBC00BFFEB57D4F0D46072844
:10B24000A8BF07201E4614465870394600F046FD38
:10B2500096F90110B070072903D1322000F0A5FC47
:10B2600005E07248405C57F8211000F0A3FC074647
:10B270000748C06D8047034606F10C0006F108013F
:10B280002246CDE900103846294600F05DFCFEBD9F
:10B290004C290108B0B50446406804F0BBFB0146E8
:10B2A000DE480268207800EB4003022052F8235069
:10B2B000002918BF0320002D08BF00F0010003285B
:10B2C00003D102EB830162684A60B0BDF8B5014664
:10B2D0000078421E0020382A00F29B80DFE802F04E
:10B2E00025279999991D999999992D2F3137993E2B
:10B2F0004144474A4D5099581D5A5F64661F1F6963
:10B300006C6E99999999999999999999999999217D
:10B31000882399992123998B8F00022079E00120BD
:10B3200077E0674875E0032073E0C87800E088782C
:10B33000002818BF012040006BE0402069E0202079
:10B3400067E091F90100897831B9374960E091F9F6
:10B350000100897800295AD0314959E040F6B830C7
:10B3600057E04FF47A7054E04FF4FA6051E041F244
:10B3700088304EE041F270704BE04FF4804048E07E
:10B3800026484FF47A7105F0F3FF00F5FA6040E0CB
:10B390004C483EE0EE48006800F5906039E0EC482B
:10B3A000006800F28C4034E0102032E0E848006889
:10B3B0002FE04FF083402CE017482AE007208DF85B
:10B3C000050010208DF80700487889788DF8040072
:10B3D000DF4800290068039000F59060029018BFD4
:10B3E000012148008DF8060001A800F087FC10E05C
:10B3F00040F211200DE091F901000C4908E091F9AB
:10B4000001000B4904B0BDE8804000F067BC05496D
:10B41000085C04B080BD00BF9A99094018FCFFFF8A
:10B42000F07F0108F87F0108E87F0108542801082F
:10B430003428010870B586B01F4991E87C0049693D
:10B440008DE87C000591017A02291DD0012925D0C3
:10B4500081BB026872B3406860B3FA4C6946C4E9C4
:10B4600000021046182205F0F8FE21680320144B54
:10B470000022A1F88C0450208882C1E9033208819F
:10B480001048C1E900020EE0EE480068B0F88C14E4
:10B49000B0F880241143A0F880140BE0E94801685B
:10B4A00000200861486001F5906001F28C410122A2
:10B4B00000F00AFB06B070BDB82701085802002052
:10B4C00040F7093700EA06372DE9F04F8FB0002525
:10B4D000DFF81C95CDE901238B4607464FF0070A9C
:10B4E0004FF00108ADF838500D95ADF832500DAC65
:10B4F000387AE9B2814239D27868214650FA85F02B
:10B5000000F0B3FC90B3BDF8381005449DF8370047
:10B510004FF0060A51EA0002ADF83210E8D0421EA0
:10B520004FF0060A052AE3D34FF0060A0628DFD8B3
:10B53000D9F800204FF0070A0023102BD8D0062896
:10B5400008D116687EB108FA03F6B6B23143ADF8F9
:10B55000321008E021FA03F6F60704D01668002E30
:10B5600008BF2AF0010A0C320133E6E702208DF809
:10B570002C00787A8DF82E000BA8FFF7A7FE8DF827
:10B5800020000DF1320007218DF810A0A21C2346E7
:10B59000079010208DF82110ADF82810F97A8DF859
:10B5A0001800B87A8DF81510611C8DF81100BDF8DF
:10B5B0003500ADF812009DF834008DF81400B889FC
:10B5C000ADF81600D9F8000009903868039003A878
:10B5D00000F0FAFB044607280DD1D9F8000000213D
:10B5E0000C2200F5906005F04CFED9F80000BDF883
:10B5F0003210A0F880149DF835109DF836209DF883
:10B6000034008BF8001001990A700299087018989C
:10B61000057020460FB0BDE8F08F00BF5802002033
:10B62000F8B501680A6892B1007902918DF80C00B2
:10B6300002A8FFF797FD062807D801460320DFE898
:10B6400001F0130404041012040000200CE000793F
:10B650008DF8040001A8FFF7D9FD002818BF0320CA
:10B6600002E0022000E0012004B080BD2DE9F0439B
:10B6700097B007460020DE4C16468846002101227E
:10B6800099460125CDE914008DF85B008DF85A002C
:10B69000CDE912000320ADF80E00206800F590609F
:10B6A00000F0A2FA216828B9B1F8800440F0030044
:10B6B000A1F880040DF10E008DF831500990102092
:10B6C000ADF82000D7E90302CDE90D026268787A6F
:10B6D00007928DF8100097F908008DF81100D7E94E
:10B6E0000023069101F590610591CDE90A23397D8A
:10B6F000BA7A8DF83C10F98A8DF83020F5F7F8FD0C
:10B7000004A90DF15B03CDE910010DF15A00494682
:10B71000CDE900060AA812AE324600F00BFB054642
:10B720000C280AD085B99DF85B00411E002005F069
:10B730001FFE305C88F8000006E02068B0F8801436
:10B7400041F00301A0F88014284617B0BDE8F0834B
:10B75000580200202DE9F04F8BB0DFF8F0AB064621
:10B76000D0F804B090F901708846DAF804008047F8
:10B77000054600285FD1F07C5FFA87F960B99C48E4
:10B780003178006801EB410150F821B000EB8100F5
:10B790004068002818BF8346DAF80C10DAF8184021
:10B7A000584688479548B9F1070FC25719D1B17C5F
:10B7B000A446308900240023CDE908410121CDE9C8
:10B7C0000644CDE90441CDE9020405204CF2503194
:10B7D00001901D4800904FF47A7042430020E047EA
:10B7E00014E0B37CA64630890124B1784FF0080CF0
:10B7F000CDE908430023CDE9003CCDE90203CDE9C2
:10B800000433CDE9063301200123F047707C104A50
:10B810000E49002808BF0A46D05DDAF854200D30E2
:10B82000C1B220469047F07C4FFA89F2594600F0A9
:10B8300037FB88F80090B5FA85F040090BB0BDE8F9
:10B84000F08F00BF5802002085450100E87F010805
:10B85000F87F010870B50446406804F0DBF805463F
:10B8600094F900000021072200F056FC0626002D66
:10B8700018BF0726002808BF06F0050694F9010046
:10B880000021072200F048FC002808BF06F003064C
:10B89000304670BDBCB556494278D1E900340178D4
:10B8A00001EB410103EB81014D7AD0E902130069FC
:10B8B000009005EB450004EBC00000F02DFBBCBD83
:10B8C000B0B504464A4D2278D5E90001FCF72CFCBE
:10B8D00094F9020000F074FA2278296802EB42021F
:10B8E00051F82250D4E9011200F06CF901464248A7
:10B8F000A289C36B2846BDE8B04018472DE9F04F38
:10B900008BB0CDE909210646DFF8E4B0327896F92C
:10B910000150DBE90001FCF707FC96F9020000F09A
:10B920004FFA074696F90100324900F0D7F9D6E9F7
:10B9300001128246384600F045F931780446DFF8B6
:10B940000C8ADBF8000001EB4101D8F81C9050F89C
:10B950002100D8F80C1088472848717840570729EB
:10B9600015D14FF47A614FF47A73002505220891BE
:10B9700058430121CDE90005CDE90225CDE90415A3
:10B98000CDE906550020214646F2A81210E04FF4FA
:10B990007A610125082208910021CDE900050120E6
:10B9A000CDE90221CDE90451CDE90611214600225D
:10B9B0005346C8473178DBF8000001EB410150F8ED
:10B9C000210096F9011000F0B7FAB18996F901004B
:10B9D000F5F78EFC0999D8F854200860317B284689
:10B9E00090470A98077001200BB0BDE8F08F00BFA8
:10B9F00058020020342801084C2901085428010865
:10BA00000020704780B5024600200A2924D8DFE8CC
:10BA100001F009232323230E11162306060092F9B1
:10BA2000000012E01068BDE8804003F0F3BF10781A
:10BA3000917806E092F900000021052207E01078D5
:10BA4000517840B209B1022100E00021072200F044
:10BA500063FB002818BF012080BD08B1002070479B
:10BA600008461146FFF70DBB00B170470846FFF7C7
:10BA70000ABB08B1D0B27047084611461A46FFF714
:10BA800045BB08B1002070470846FFF753BBB0B56F
:10BA900000230024914238BF01241209B2EB111F88
:10BAA00028BF012304EA0302012A0BD10B0901F08C
:10BAB0000F01012530F8134005FA01F124EA0101D4
:10BAC00020F813101046B0BD38B131B12AB131F8A9
:10BAD000023B013A20F8023BF8E770472DE9F041BC
:10BAE0009A4202DB069B9A4202DD0020BDE8F0810B
:10BAF000079B4FF0000E03F1080C00235FFA83F858
:10BB00008045F2D208EB48030CEB83065FFA8EF314
:10BB100031F813700023102B0ED027FA03F4E4073A
:10BB200007D0347804F00F059542D8BFB2EB141F4C
:10BB300007DD0C360133EEE70EF1010E08F11003BC
:10BB4000DCE70120BDE8F08170B54FF4FA64624390
:10BB50006FF0070404EB410404FB0025DDE9044217
:10BB600055B14619013EB6FBF0F68E428CBF00215E
:10BB70000E46002D18BF31462160414385004C1C04
:10BB8000A5EB5404002908BF84004FF47A70002507
:10BB900003FB00F18C42C8BF40F2E73503FB1051B4
:10BBA000214491FBF0F0106070BD4FF4FA51B1FBED
:10BBB000F0F07047024A02FA00F0B0FBF1F0704773
:10BBC00040420F00B0B5400014460D4606F0A2FBFF
:10BBD0000146284606F06EFD214606F06BFD05F095
:10BBE00075FE06F043FBB0BDB8B1F0B50023CCB292
:10BBF00094420FD230F8144000250026102D06D0B4
:10BC000024FA05F7FF0718BF01360135F6E733447C
:10BC10000131ECE7BDE8F04000E00023D8B2704706
:10BC20002DE9FE4F02914FF000084FF0010A00216C
:10BC300000244FF0000ECDE90023038A5FFA84F957
:10BC4000994543D209EB49035FFA8EFB00259C001E
:10BC5000102D36D043680AFA05F633F81B301E4221
:10BC60002CD087683B594BB30378E3B13E1990F968
:10BC70000130377A3A07B3EB227F1FDB7AB2B3EB9E
:10BC8000221F1BDC727AC36802EB420203EBC20282
:10BC9000127D92B1029E5FFA88F309EB050208F16A
:10BCA0000108F2540AE0D0F814C0BCF1000FDDD056
:10BCB0003CF81B301E42D9D100E001310C34013573
:10BCC000C6E70EF1010E09F11004B6E7009880F8FE
:10BCD000008001980170BDE8FE8F000051F820102F
:10BCE0000448054A0844B0FA80F04009914208BF70
:10BCF00002207047702FFCFF20A10700FEB50678D8
:10BD00008778BE4214D004467DB2013EF0B2B842FC
:10BD10000DD0D4E9011294F90130E078CDE9003278
:10BD200072B22B46FFF7DAFE0028EED000E03E4666
:10BD300070B2FEBD2DE9F04F85B0074640689B46C6
:10BD400090460D4603F08CFD3968DDF83C90DDF837
:10BD500038A0091AC9F8001001218AF80010002142
:10BD60008BF800107A6812B13A6882421FD82960B5
:10BD70003B7A7A7A3E7DD7E906C0D7E90354C16899
:10BD80000078CDE90065CDE9024C00F0EBF8C9F888
:10BD90000000F86941465A465346FFF741FF9BF8B9
:10BDA000000020B10020C9F80000002005E09AF84A
:10BDB00000100B20002908BF0C2005B0BDE8F08F53
:10BDC0008842D8BF084670472DE9FE4F04460579E2
:10BDD00040798A46062198469146002808BF0921E5
:10BDE00014F801B04FF0070108BF0A216656082178
:10BDF000002808BF0B21675C2DB1BBF10F0F04D1E8
:10BE000094F809B013E0002521E094F91520D4F846
:10BE100018C094F914302169207BCDE9002C4FFA29
:10BE20008BF2FFF75BFE002808BF05F0FD050F2E23
:10BE300001D1A67A0BE094F91D00864201DA06468C
:10BE400005E094F91C008642C8BF05F0FB0585F0AB
:10BE500007008AF800B089F80060384308BF01275E
:10BE600088F800702846BDE8FE8F0278032A14D1B6
:10BE70004278130902F00F024B708A7082788A8030
:10BE8000C37842EA03228A80007900F00F02C0F3EF
:10BE90000210C87005200A7070470020704700002B
:10BEA000F8B5052807D8CDE901120DA112A351F864
:10BEB0002000009002E003A3CDE90012FCF740F956
:10BEC0008FBD00BF5258206F6E20667265712025AD
:10BED0006420487A2061742044522025640D0A00B1
:10BEE000A9850108AB8501086A86010864860108F6
:10BEF000728601086C86010852585F2573206F6EA8
:10BF0000206672657120256420487A20617420447F
:10BF1000522025640D0A000070B51E46049B0C4695
:10BF2000114605463246F5F741F9E9686043081ABB
:10BF300038BF0020E86070BDE0B5CDE9000102A384
:10BF4000FCF7FEF88CBD00BF5458206F6E2066725F
:10BF5000657120256420487A206174204452202590
:10BF6000640D0A002DE9F04F8DB0664D0E46074670
:10BF7000624817991446624A01350844A9424FF0B5
:10BF80000001B0FBF2F0039588BF00FB0221029193
:10BF900005935D4900FB0210019016981843049028
:10BFA00087F001001843079003F050FC4FF0FF3B6F
:10BFB0004FF000090690002C00F096800894179C22
:10BFC000189D2046294602F089F8824630463946B7
:10BFD00022462B46F5F7EAF880462FB105984B4CE0
:10BFE000A8BB4A4CF46032E0B8F1640F09D0B8F550
:10BFF0007A7F07BFC6F808A0454CD6F808A0454C84
:10C0000002E0424CC6F808A009A8514601F0F0FF32
:10C01000DDE90930DDE9171200900BA802F04EF8B7
:10C0200004990C9831B13169A14203D10B99344A7A
:10C0300091420CD31799334AF460914207D94FF6D5
:10C04000FF7120EA0101019802F048F8B0607068C1
:10C0500000B9F460346137B103F002FCD6E903148F
:10C060000844F06000E0F068A04284BFF46020461D
:10C07000002206997160199908FB01F1814228BFDD
:10C080000122079B134227D000228C42327588BFC1
:10C0900009F101090A1A934538BF5A468C4288BFF4
:10C0A0009346EFB91898B8F57A7F179B00900398DC
:10C0B00008BF49F6B020B8F1640F08BF4FF46160C3
:10C0C0000299002201440BA801F0F8FFDDE90B0101
:10C0D00002F004F8834603E0012009F101093075FC
:10C0E000089C1836013C66E75FEA096108BF4FF01B
:10C0F000FF3B58460DB0BDE8F08F00BFD013FEFFE8
:10C10000805101002FEC010030EC010040771B0052
:10C1100080A81201002E9302884201DB904201DDCB
:10C12000002070470120704700B1704710B5029C95
:10C13000FBF7F5FFBDE81040FFF77EB808B100201F
:10C1400070470846FFF7A6B808B1002070470846B8
:10C15000FFF7BCB8004870470300010100B1704709
:10C160000846FFF767B9B0FA80F04009704708B198
:10C17000002070471CB5DDE904400090FBF7CFFFBD
:10C18000FFF7A2F91CBD08B1002070470846FFF771
:10C1900047BA08B10920704710B5029CFBF7BFFFF2
:10C1A000BDE81040FFF762BA08B1002070470846AA
:10C1B0001146FFF7CFBA08B1002070470846FFF7D5
:10C1C00049BB00B170470846FFF764BB00B1704738
:10C1D0000846FFF775BB08B10020704708461146B6
:10C1E0001A46FFF78BBB08B1002070470846FFF7DF
:10C1F00007BC08B10020704708461146FFF702BC93
:10C20000F0B58DB0534D4248514C0026C5F810048E
:10C21000012084F81861A66284F8076104F1A80778
:10C2200004F1640C85F81464A4F80A018DF8080080
:10C230008ECFACE88E0084F83A60B4F8CC10218739
:10C2400094F8A51084F8611094F8B81084F874106C
:10C2500094F8B91084F87510D4E92F12C4E91E12AD
:10C2600004F51D71019104F5F07194F840000091FE
:10C270006946FFF773FF4FF48070616E85F8CC63F9
:10C2800085F81564CDE90B66A5F8DE0394F8750012
:10C29000D5F8CC7385F8DC0394F8800085F8DD03CD
:10C2A000D5F8DC03C5F8D013D5E9F523C5E9F87155
:10C2B000C5E9FA23C5F8F00340F20120A5F8F2031E
:10C2C000D5F8480318B141680069CDE90B1004F1B5
:10C2D000D80004F5E2620A9004F14400099004F1E8
:10C2E0004000089004F1D400079005F285400690C4
:10C2F00005F24C40059005F21C40049005F58C6059
:10C30000039003A80BA9F9F786F80DB0F0BD00BFA4
:10C3100000010100F8B50C4603F046FB0B4D286BFD
:10C3200080470B4F0B4E214697F8400006F584627C
:10C33000FFF73AFF48B196F82004696B86F862046B
:10C34000F86C8847E07C86F88404F8BD4C29010825
:10C3500028870020D012002000210D4AB0F5803F30
:10C3600038BF012138BF00040901B0F1807F3CBF14
:10C3700008310002B0F1805F38BF043138BF0001DE
:10C38000000F81F01F01105C081AC0B2704700BF97
:10C39000D0290108F4F724BAE748811C021DF4F7FC
:10C3A00001BA00BFF8B5044600200D4600F0BAFA05
:10C3B000F6F72AFA01F0DEFEFBF7C2FBFBF722FCE0
:10C3C000FBF79AFC3748F5F7B6FF202802D036A3D2
:10C3D000FBF708FE00F0FAF8F4F738FA3220F5F728
:10C3E00004FDD54F0026AE4229D2FFF7D5FF00F05D
:10C3F00071F8388A2188084461882080B889084407
:10C40000A188608038890844A080F86905F02EFF73
:10C41000E18801360144E18021890144218161895B
:10C42000084439886081A0890844E189A08178881E
:10C430000844218AE081B88808442082D3E7B4F90F
:10C440000000B4F90210B4F90420B4F9063090FBEE
:10C45000F5F0208091FBF5F0608092FBF5F0A08074
:10C4600093FBF5F0E080B4F9080090FBF5F0208133
:10C47000B4F90A0090FBF5F06081B4F90C0090FB70
:10C48000F5F0A081B4F90E0090FBF5F0E081B4F96D
:10C49000100090FBF5F02082F4F7A2F9A5480021E6
:10C4A0000170F8BD3C4A00200D0A202E2E2E2E20B1
:10C4B0004D4F54494F4E2053454E534F5220493211
:10C4C00043204E6F74205265616479202E2E2E2EEB
:10C4D000200D0A0070B51F48F5F72DFF202802D067
:10C4E0001DA3FBF77FFDF4F7B1F902F083F8FDF728
:10C4F00045FB914E308AB16A0844716AB062B089D6
:10C50000084431897062D6E90702D6E9054511442D
:10C510003162B16B0131B16305F0A8FE05F0FAFE9E
:10C520000146706B05F014FD7063284605F09EFE11
:10C5300005F0F0FE0146306B05F00AFD3063204641
:10C5400005F094FE05F0E6FE0146F06A05F000FDF8
:10C55000F06270BD3C4A00200D0A2E2E4932432065
:10C56000494E495449414C495A494E472020455269
:10C57000524F52200D0A0000BCB504463020F4F79B
:10C58000FBF80546C00601D4002006E0684601F02D
:10C5900069FD69480099816401202070280701D451
:10C5A000002006E0684601F05DFD634800994164A3
:10C5B00001206070BCBD00BF10B50020002400F059
:10C5C000B1F9F4F70DF95B48047010BD5A48002129
:10C5D000632280F84C1080F84F10A0F85010A0F89B
:10C5E0005210A0F85410A0F85610A0F85810A0F857
:10C5F0005A1080F85E20C163C0E90A11C0E90C112D
:10C600008163C0E90211C0E90411C0E90611C0E963
:10C6100008110164704700BF2DE9F843464C4FF004
:10C62000010984F84C90E06B84F84F00A06BD4E9CA
:10C630000923D4E90761D4E90585B3FBF0F3B2FB24
:10C64000F0F2B1FBF0F1A4F85030A4F85220A4F8B5
:10C65000541005F05FFE07463046394605F010FDE0
:10C6600005F004FEA4F856002846394605F008FDFA
:10C6700005F0FCFDA4F858004046394605F000FDE1
:10C6800005F0F4FDA4F85A000020E063C4E90800B6
:10C69000C4E90A00C4E90C00A063C4F84090BDE8F6
:10C6A000F88300BF244991F84C20027091F84F2084
:10C6B000C270B1F850208280B1F85220C280B1F827
:10C6C00054200281B1F856204281B1F8582082816D
:10C6D000B1F85A10C1817047BCB5164C207838B3F8
:10C6E00001A8FFF749FF9DF8040050B1FFF754FE81
:10C6F000FFF76CFF0025022D03D8FFF7EBFE013595
:10C70000F9E79DF8050078B1FFF746FE0A4D686C21
:10C71000A96C401AFA21B0FBF1F202FB1100E863A8
:10C72000FFF77AFF0120286400202070F4F758F802
:10C73000BCBD00BFB84B0020B8010020B0B588B028
:10C740006C462021FBF704FF22492046202202F0FC
:10C75000BFFF9DF80010FF2931D09DF80120FF2A6E
:10C760002DD09DF80230FF2B29D01B4880F82010D7
:10C7700080F8212080F822309DF803109DF80420D5
:10C780009DF805309DF8065080F8231080F824208D
:10C7900080F8253080F8265000229DF8071001F01F
:10C7A0001F0180F8271004F1080190F827309A4201
:10C7B0000BD28C5C8318013283F82840F5E707A37D
:10C7C0000120FBF70BFCFCF799FCFCF70FFB08B012
:10C7D000B0BD00BF00F8030800000020496E697476
:10C7E00069616C20426F6F74207769746820456DB1
:10C7F00070747920436F6E6669672C20466C617394
:10C800006820776974682064656661756C7420635C
:10C810006F6E6669672E2E2E2E0D0A00B0B58EB093
:10C8200006A81A210630F3F71BFE30480125002424
:10C830008DF81C508DF817400690F4F78BFCFD28FE
:10C840000DF1170088BF63248DF81D4000F050F8EB
:10C8500000283FD001AC12211225FBF779FE2046BB
:10C860000A21FFF79FFDBDF80610BDF8040009BAC4
:10C870008DF82000000A090CADF82110BDF8081051
:10C8800009BA090CADF82310BDF80A1009BA090C51
:10C89000ADF82510BDF80C1009BA090CADF8271039
:10C8A000BDF80E1009BA090CADF82910BDF810102A
:10C8B00009BA090CADF82B10BDF8121009BA090C11
:10C8C000ADF82D10BDF8141009BA090CADF82F10F1
:10C8D000192101E0082158208DF81F008DF81E5005
:10C8E00006AAFBF7B9FE0EB0B0BD00BF53005A0157
:10C8F00010B50446F3F720FF2070E52818BF00208C
:10C9000010BD0000022888BF70470A48102101228C
:10C91000F5F7B4BC022888BF7047064810210022F2
:10C92000F5F7ACBC022888BF7047024810210122ED
:10C93000F5F7A4BC0004004802A20120052100F084
:10C9400005B800BF50565858580000007CB5164B2B
:10C950000024A14204D0155D9E6835550134F8E7E6
:10C9600003F8040F00225970D97A1846F8F7D2FA62
:10C9700088B1C0B2FA280DD1F8F71AF950B14FF4C6
:10C980007A710A4B0122B0FBF1F0002100900120E6
:10C9900002F0D0FD7CBD064B01200021012202B037
:10C9A000BDE8704002F0C6BD00000020E38301082E
:10C9B00001840108074940F441700A6822F04002EE
:10C9C0000A6008604FF4B8504860086840F04000C2
:10C9D0000860704700000158B8B54E4C64232268C7
:10C9E000FBF7E3FE294B0092009A3AB1009A013A14
:10C9F00000921A689207F7D5002201E001228260B6
:10CA0000FF251D7164252468C4EBC404C4F34C44A1
:10CA10006C430094009C34B1009C013C00941C6861
:10CA2000E407F7D001E001228260586808701046E0
:10CA3000B8BD00BF18B5374C64232268FBF7B5FEBC
:10CA4000124B0092009A3AB1009A013A00921A6889
:10CA50009207F7D5002201E0012282601971216856
:10CA60006424C1EBC101C1F34C41614300910099C1
:10CA700031B10099013900911968C907F7D001E077
:10CA8000012282605868104618BD00BF0800015896
:10CA900081B00179012915D11E49096801EB4101D5
:10CAA000C1F34F31009109490A6822F400420A603B
:10CAB000009A013A0092009A002AF9D10A6842F4D9
:10CAC00000420A6001B000F007B800BF90040058AF
:10CAD000E948F6F765BE00BF81B00E4964220968D7
:10CAE00001EB4101C1F34B41514300910A490A68EE
:10CAF000009B53B1009B9208013B00930B6802EA34
:10CB00005302D207F3D1002002E00221816001200C
:10CB100001B070474401002014040058E0B500F053
:10CB20007F000DF1070101228DF80700892000F038
:10CB3000A3FC8CBDE0B51849884204D3E1208DF8F0
:10CB40000600E9201EE01549884204D3D7208DF85D
:10CB50000600DB2016E01249884204D3C1208DF87C
:10CB60000600C5200EE00F49884204D375208DF8D9
:10CB70000600812006E00C49884205D36B208DF821
:10CB800006006F208DF807000DF1060198200222A3
:10CB900000F072FC8CBD00BF01E9A43581F8A93218
:10CBA0008144E52D010B6B1B41FC54192DE9F84321
:10CBB000194C814640F607008846A04706464FF4C8
:10CBC000D660A047074600F00F0540F2B160A047CD
:10CBD0003A0740EA0520114948BF0843C6F3C1019E
:10CBE0000FA20123515C06F00702013A91400D4A61
:10CBF000B2FBF1F1B1FBF9F2082A38BF02235A4324
:10CC0000042A38BF0423594349094843C011C8F8CE
:10CC10000000BDE8F88300BF45CE000800F0FFFF2C
:10CC200004080A0C0048E80160B1074A0021B02955
:10CC300007D0535808318342F9D9501810F8040C22
:10CC40007047FEE71F2070475C280108F1484078D4
:10CC5000704700BF1CB504460DF1050114200322E6
:10CC600000F0E2F8EB4881780129217010D009BB6F
:10CC70009DF805009DF806109DF807202071002002
:10CC8000A06048424008A0715042400860711CBD3D
:10CC900040689DF8071020619DF80500404240085B
:10CCA00020739DF9060002308008607348424008F6
:10CCB000A0731CBD20460021142202F012FD0F209B
:10CCC00020701CBD7CB50E46044600200DF1070106
:10CCD00015468DF80700304600F04CF83278AA422D
:10CCE00001D901207CBD9DF80700214600F08EF897
:10CCF00000207CBD0A2070477CB50020019040F6E2
:10CD0000E20000F09FF8144E044600F0FE0140F6E9
:10CD1000E200B04740F6E50000F094F8054600F068
:10CD20007F0140F6E500B0476FF07F4000F034FA35
:10CD300001A940F61900042200F090F8002000F04C
:10CD40008BFA40F6E2002146B04740F6E50029465E
:10CD5000B04701987CBD00BF95D40008E0B50DF147
:10CD600007011520012200F05FF89DF807004042FE
:10CD700040108CBDBCB50C4605460DF106011320D4
:10CD8000022200F051F8E0488178012907D1C078EB
:10CD9000012804D140F2027000F054F801E09DF83F
:10CDA000060028709DF807002070BCBD10B508B1C2
:10CDB000ED498860FAF792FF0220FEF74DF9EA4C40
:10CDC00000202070002000F047FAFCF765FF0128E2
:10CDD0000DD101204FF4207100F07AFA40F61110C5
:10CDE000002100F057FB7F20FFF798FE09E040F696
:10CDF0001110102100F04EFB40F61210102100F02F
:10CE000049FBFCF715FF0120607010BD10B5FBF762
:10CE100022FAEFF31084EFF3108072B61648F6F79B
:10CE200073FD84F3108810BD10B5FBF714FAEFF30F
:10CE30001084EFF3108072B60F48F6F743FC84F3CA
:10CE4000108810BDE0B501460B480DF10702012323
:10CE5000F6F786FD9DF807008CBD00BF10B5FBF707
:10CE6000FAF9EFF31084EFF3108072B60248F6F788
:10CE700077FD84F3108810BDC04A002010B5144619
:10CE800000F044F92046BDE8104000F035BAE0B5A6
:10CE90008DF807108DF806000DF106018F20022293
:10CEA00000F0EAFA8CBD000080B5C5200021002208
:10CEB00000F0E2FAF1480721417080BDE0B540BAC8
:10CEC000ADF80600ED48807800B18CBD0DF106018B
:10CED00040F2BE60022200F0E9FA8CBDE0B540BA33
:10CEE000ADF80600E548807800B18CBD0DF1060173
:10CEF00040F2BC60022200F0D9FA8CBDE0B58DF89A
:10CF00000520120A8DF80310090A8DF80100000AA5
:10CF10008DF807301B0A8DF804208DF802108DF86B
:10CF200000006946082008228DF8063000F0A4FAB7
:10CF30008CBDE0B58DF807000DF10701A020FBF7CF
:10CF40008DFA9DF8070040280ED341080020CAB290
:10CF5000202A02D301309108F9E700EBC100C1B2E9
:10CF600040F2067000F096FA8CBD00001CB5EC494A
:10CF700004460020CDE9000020788978814202D063
:10CF800000F0B0F82178032942D8DFE801F002224E
:10CF9000262DA089204A0023ADF80300D4E9010121
:10CFA000B2FBF0F0020A8DF80200000C8DF80120AF
:10CFB0006E4A8DF800004806C909F3F73BF9010AEB
:10CFC0008DF80700000C08228DF806108DF805007A
:10CFD0001AE0A0690422009016E0207D0E49042288
:10CFE0008DF80300206905E0A0890B490522ADF802
:10CFF00003006068B1FBF0F0010A8DF80200000C3C
:10D000008DF801108DF8000069468B2000F034FA8D
:10D010001CBD00BF780200200000093DE0B58DF87E
:10D0200006208DF804008DF807308DF8051001A951
:10D030009520042200F020FA8CBD00007FB5044644
:10D040000020B74D8DF80C00CDE901002078A978BB
:10D05000814202D000F046F82178032940D8DFE869
:10D0600001F0020D1A02667AF12E19D0F22E21D1AA
:10D07000062641F2210541F60F5016E0207C617C26
:10D080000622E8708DF806008DF80710608AADF86A
:10D090000800E0891CE0207B01228DF804001BE0E1
:10D0A000022648F205054FF6FF70FFF717FF2846E6
:10D0B000FFF704FF20798DF80B6009228DF8060038
:10D0C000D4F80500CDF80700A07A8DF80C00608830
:10D0D00000BA000CADF8040001A98C2000F0CCF9D6
:10D0E0007FBD00BFE0B5DC498DF80700887020B92E
:10D0F00040F2AC60002100F0CDF90DF107018A206B
:10D10000FBF7ACF98CBD00BF780200200A4601464F
:10D11000002000F0A3B9E0B5FCF7BCFD01380DF12B
:10D1200007010122B0FA80F040098DF8070096202F
:10D1300000F0A2F98CBD0000BCB5C74D04462878AC
:10D1400020B92046FFF7F6FC01202870074A600648
:10D15000E1090023F3F76EF800BA0422019001A957
:10D16000862000F089F9BCBD780200200048E80163
:10D17000B0B50446FCF75AFD022805D0012520B9B8
:10D180000F2CC8BF022500E00225284621460222B6
:10D1900000F0D2F82846B0BDE0B5AF4905228DF8C1
:10D1A00007004A70010A000C03228DF806108DF862
:10D1B00005000DF10501822000F05EF98CBD00BF75
:10D1C0001CB50446A4480521417040F6AC009721E7
:10D1D00000F060F9200A0DF1050103228DF80740E7
:10D1E0008DF80600200C8DF80500822000F044F92F
:10D1F0001CBD00BF1CB50A0A8DF80710090C8DF87C
:10D20000040006248DF80510010A000C8DF8062094
:10D2100006228DF803108DF802000DF10201942012
:10D2200000F02AF98C4844701CBD00BFBCB5044610
:10D2300000200025FCF7D6FC0220FDF70DFF04F0CE
:10D2400007000DF1070101228DF80700842000F08E
:10D2500013F981484570BCBDE0B58DF807000DF1AC
:10D2600007018020FBF7FAF89DF80710022000293B
:10D27000794908BF012048708CBD00BF78020020AA
:10D28000E0B58DF807000DF107019F20FBF7E6F8E8
:10D290008CBD012908D110B50446012807D104200E
:10D2A000FDF7DAFE022003E00120FCF79BBC012021
:10D2B000022C08BF0320BDE81040FCF793BC80B5EA
:10D2C00001464FF4D860082200F0F0F8002080BD3D
:10D2D000E0B500F007008DF8071004228DF8040077
:10D2E000080A8DF80600080C8DF8050001A99720A2
:10D2F00000F0C2F88CBD0000E0B5574904228DF85B
:10D3000007004A70010A000C03228DF806108DF800
:10D3100005000DF10501832000F0AEF88CBD00BFC3
:10D3200078020020D1200021002200F0A5B8D220F0
:10D330000021002200F0A0B87CB514460D4601285B
:10D3400010D10020FCF76CFCA842B8BF05460A28A3
:10D3500026D006460E282AD1042000210122FAF701
:10D36000F7FE2CE040F6D800FFF76CFD40F01E0100
:10D3700040F6D80000F08EF80120FCF751FCA842DE
:10D38000B8BF05460E2822D00646112825D0142EF7
:10D390002AD1032005210022FAF7DAFE02352BE01C
:10D3A000012000210122FAF7D3FE033507E0062011
:10D3B00000210122FAF7CCFEA81B00F10E0568B28D
:10D3C00010F1110FD8BF6FF0100518211BE00220DB
:10D3D00002210022FAF7BCFE0EE002200321002207
:10D3E000FAF7B6FE053507E0042007210022FAF718
:10D3F000AFFEA81B00F1160568B210F1090FD8BFE7
:10D400006FF00805382140F6E70000F043F80DF111
:10D4100006018E2002228DF807408DF8065000F09C
:10D420002BF87CBD10B504460B48807800B110BDC8
:10D430004FF4D760FFF706FDC4F3002100F0FE00B3
:10D4400001444FF4D76000F025F8E1B240F2B96032
:10D45000BDE8104000F01EB87802002010B5FAF7C1
:10D46000FAFEEFF31084EFF3108072B61648F6F769
:10D47000BBFA84F3108810BD10B5FAF7ECFEEFF399
:10D480001084EFF3108072B60F48F6F745F984F375
:10D49000108810BDE0B503460B488DF807100DF15C
:10D4A000070219460123F6F7C5FA8CBD10B5FAF745
:10D4B000D2FEEFF31084EFF3108072B60248F6F755
:10D4C000B9FA84F3108810BDC04A002070470000EC
:10D4D00080B50B48F3F7FCF878B10A4940F6E4420E
:10D4E0004FF6FF7309884A43994204BF40F6D802B9
:10D4F000C0F24C02B2FBF0F000E0002080B280BD30
:10D50000002000B4AA75FF1F01480249016070475E
:10D51000784900200024014070B590B00446F7F728
:10D520007DFF08B10E2020E1A94D95F804010128E6
:10D5300007D1F7F779FF10B9F7F774FF08B10F209B
:10D5400013E1286B38B9A349B5F80A01D1F81814CA
:10D550004843401A28639F4E96F80401042807D0D8
:10D56000002840F0018106F58470FAF718F903E00D
:10D5700006F58470FAF7ACF808B11120F5E096F8DA
:10D580000C013080286B039095F839008DF8140059
:10D5900095F808018DF8160001A800F063FDD5E9A3
:10D5A0004330DDE9011200900AA800F087FDDDE9B3
:10D5B0000A01EA6ACDE906010492328800200121BD
:10D5C0008DF820008DF81510ADF8222095F818215F
:10D5D0001AB98DF815008DF8201005F1300195F875
:10D5E000400006F2154206F59163009103A9FEF78B
:10D5F000D0FDA8B10B2840F0B880002C46D0D6F85A
:10D60000881459B1D6F8400306F55A7440F020004A
:10D61000C6F84003FAF73FFEFBF7F8F90020A4E054
:10D6200095F8404095F9613095F9392095F87510D5
:10D630002046FEF71EFA06F56E716B6C95F84820D1
:10D64000009141B22046FEF76FFD6B6C95F84820C3
:10D6500095F9681095F8400006F573740094FEF78C
:10D6600063FDD5E91423D6F8C403D6F8D8130244D1
:10D670000B44C6E9EC2395F818214AB100200A9022
:10D680000AA8F7F74FFF60B113206EE00B206CE0A3
:10D69000D5E9162310441944C6E9EC0100200A908C
:10D6A0000EE096F837029DF828100C1895F939000D
:10D6B000F3F7FAFD01460820FF2C98BF8C4254D89E
:10D6C00095F8381095F8392096F8154495F84000EB
:10D6D00006F583638DF829208DF82A10D5E91E12EE
:10D6E0008DF82840CDE90B1231880DF12702ADF8F5
:10D6F000341000218DF827100AA9FEF76CFD0120D7
:10D70000C6F8484486F8390495F8390086F83A0492
:10D710009DF8270086F83B04D6F81804C6F8500494
:10D72000C6F84004F7F77CFE30B1D6F81804F7F7D6
:10D730007DFE08B1102018E095F80401012808BF0B
:10D74000F7F785FEF7F766FE002096F8154495F882
:10D7500039500F9096F80401042808D020B906F536
:10D760008470F8F731F918E0032010B070BD0FA8ED
:10D77000F8F79AF808B11220F7E796F8100418B9EC
:10D7800096F81204012821D90F9801380F9006F558
:10D79000847329462246F8F741F900287FF4EDAE5C
:10D7A000D6F8400396F80C1140F002003180C6F81C
:10D7B000400396F8140420B996F81004013086F856
:10D7C0001004BA4AB01C926A904727E70F98DEE728
:10D7D00028870020D01200202DE9F047BEB040B1CC
:10D7E0001C4633B106460D46080708D04FF0050A1F
:10D7F00001E04FF0020A50463EB0BDE8F087174600
:10D8000001A80021F02203F03CFD69463846F3F7F9
:10D810000FFD82460028EED100980DF1040810217A
:10D820004FF010094246013003F08AFC002728041B
:10D83000E1D056FA87F054FA87F1424603F024FB10
:10D8400059FA87F7103DF2E77E2B98BFF3F750B9EE
:10D85000032070471FB5A0B114460A467F2C01D1A2
:10D86000042A10D100216B46CDE90211CDE9001147
:10D870001021FFF7B1FF38B96946204600F032F9B0
:10D8800002E0022000E0032004B010BDAE480068B2
:10D89000704700BFAC4800680830704710B5AA4A0E
:10D8A0000023126803F11104BB2C06D013441B7C27
:10D8B00083422346F6D1FAF7B9BC032010BD00BF5E
:10D8C000B0B558B10C46A04D0549C022286003F000
:10D8D000C4FC0CB12868A0470020B0BD0220B0BD38
:10D8E00000E503082DE9F04389B01E4BDFF878808E
:10D8F000FAF711FC1D4D0020A8470120A8471C4B3A
:10D90000FAF709FC0320A8470220A847194BFAF7A9
:10D9100002FCDFF86490D9F800000178427883783F
:10D92000C678077944798579C0798DE8CE00CDE94C
:10D930000545079011A3FAF7EEFBD9F80000017A2C
:10D94000427A837AC47A057B467B877BC07B8DE8ED
:10D95000FE00079019A3FAF7DEFB002009B0BDE82E
:10D96000F08300BFFD85010835F5000861950008CA
:10D97000D3850108E8850108E81800202323232324
:10D980002323204465764575693A202020202020F5
:10D99000253032583A253032583A253032583A2517
:10D9A0003032583A253032583A253032583A2530FC
:10D9B00032583A253032580D0A0000002323232321
:10D9C0002323204170704575693A202020202020B3
:10D9D000253032583A253032583A253032583A25D7
:10D9E0003032583A253032583A253032583A2530BC
:10D9F00032583A253032580D0A00000010B5054C57
:10DA00000420A0477F20A0470220A0470320A04772
:10DA1000002010BD61950008F8B543B1079C34B1F2
:10DA2000089F27B1069D212D03D90520F8BD0220AE
:10DA3000F8BD204619462A461E4603F00EFC691E14
:10DA4000701C631C012289B2FFF7C6FE08B10720D3
:10DA5000F8BDE07AC10940B20028397017D4281FF8
:10DA60002A19215C12F8033C12F8025C12F8012C0E
:10DA700041EA0321012341EA054141EA026281B200
:10DA8000204600F063F8002818BF0120F8BD0420EC
:10DA9000F8BD000038B110B504460448406980471D
:10DAA0002060002010BD0220704700BF4C290108F3
:10DAB00040B180B5014624480822006803F0CDFB40
:10DAC000002080BD0220704748B180B501461E4845
:10DAD00008220068083003F0C0FB002080BD02204F
:10DAE000704700BFF0B585B009B3174E0023326808
:10DAF00003F11107BB2F1CD013441B7C83423B4610
:10DB0000F6D1802817D100207F22CDE90300CDE98E
:10DB1000010001AD084610212B46FFF75DFE0446CB
:10DB2000306829461022384403F097FB08E00224AD
:10DB300006E0032404E0D019102203F08EFB002439
:10DB4000204605B0F0BD00BFE8180020A0B11CB50C
:10DB500014460A4601460020019001A800900020CA
:10DB6000F2F7C6FF01460198A042084618BF0120FF
:10DB7000002918BF08461CBD022070472DE9F04F50
:10DB80008FB0F3F7E7FA04460AA8FEF78BFDB64E0E
:10DB9000AC4D14203071E878B1680870287860B115
:10DBA0001520FE2102273071002028706320604379
:10DBB000B0FBF1F0B168487000E001276D480178D2
:10DBC000002900F0968000210D220170B068C15537
:10DBD0005A21B068384441700121B06838448170DE
:10DBE0006320FE216043B0FBF1F0B1683944C87096
:10DBF000381DB1680A54B1689DF82B2001444A7061
:10DC0000B1689DF82D2001448A70B1689DF82C20E0
:10DC10000144CA70B1689DF82F2001440A71B168AF
:10DC20009DF82E2001444A71B1689DF831200144CD
:10DC30008A71B16808449DF83010C17107F10C0178
:10DC4000B0689DF833204254B0689DF832200844F3
:10DC50004270B0689DF8352008448270B0689DF825
:10DC600034200844C270B0689DF83720084402711F
:10DC7000B06808449DF836104171B168887A91F80F
:10DC80000EB091F80BA0CB7B91F80C904D7C0A7CE8
:10DC90008C7C91F8048091F806E091F807C0099017
:10DCA000487AC3EB0323C5EB05251A442C44324BB9
:10DCB000644D0890487B097A0592099ACDF81C803A
:10DCC0000694C0EB002058440490CAEB0A20484454
:10DCD00003900898C0EB0020104400220290CCEB87
:10DCE0000C2008440021CDE900E0022001F022FCD4
:10DCF000123795F84100777150B1F7F70BF801280A
:10DD000006D105F1380001F04FFE3E48FAF758FB06
:10DD1000022F1CD3F17B301D00220024F7F7FAF804
:10DD2000811D04D0C0B298B9154B002409E0F6F764
:10DD30003FFF60B104464FF47A70104BB4FBF0F033
:10DD4000009001200021012201F0F4FB00E00024FA
:10DD50002E4D284601F028FE316828468C4288BFA7
:10DD6000214601F0D3FD284601F0E8FD0FB0BDE8E3
:10DD7000F08F00BFF80100201C850108E383010833
:10DD80000184010870B51F4C1F4E4FF40041012261
:10DD900001252046B04720464FF400710122B047CC
:10DDA00020464FF400610122B047184801F0FCFD05
:10DDB000F7F733F920B116A30220FAF70FF91BE0A9
:10DDC0001BA3FAF7D9F9022401F0B4FB1D4E1EA3E0
:10DDD000FAF7D2F9B57001F0ADFB23480C30F6F735
:10DDE000BFFDB078002818BF012420460121F6F7B6
:10DDF0003DFF064801F0A2FD12485030BDE87040DA
:10DE000001F09CBD000400487D2200085419002048
:10DE10004C6D48616E646C65722053746F70206F36
:10DE20006E20676F696E67202E2E2E0D0A0000008F
:10DE30004C6D48616E646C65722053746F707065D0
:10DE4000640D0A00480300204C6D48616E646C65E7
:10DE5000722073776974636820746F204142502088
:10DE60006D6F64650D0A000000000020544890F8B2
:10DE70008514890703D590F88314022906D34E49E7
:10DE800091F8062112B18A6A01328A62002180F873
:10DE90001014A0F81314D0F8401321F00201C0F8B8
:10DEA0004013704780B5F6F749FF10F1080105D01F
:10DEB000C0B2FF2818BF80BD0AA300E003A3FAF791
:10DEC0005BF9BDE8804001F035BB00BF4E564D20E8
:10DED0004441544120555020544F20444154450D55
:10DEE0000A0000004E564D20444154412053544FE7
:10DEF0005245204641494C45440D0A00F8B52E4E86
:10DF0000054696F8040102280CD001280DD050B91E
:10DF1000022D1AD0012D4BD02DB9D6E91901C6E931
:10DF20001B0100E055B1032440E02846F7F790FAC2
:10DF30000446D8BB86F80451002437E01F4800246B
:10DF400086F80441C06A804730E01D48022786F801
:10DF5000047100F5737500F5787C3ECDACE83E00A9
:10DF600096F8DA1080F8F373C1B140F2013196F8F7
:10DF7000F420A0F8F213D6F8F01086F8702096F886
:10DF80008020F166C0F8E41390F8151480F8F123AE
:10DF900080F8E01396F8751080F8F013002480F8EC
:10DFA00014440648C06A8047FBF7F6F92046F8BDDE
:10DFB00001250120BAE700BF288700204C2901086D
:10DFC000D01200207047000010B51944029B0024B5
:10DFD000C0E90014054C1A4413048280A34204DBF8
:10DFE000A2F57A7201318280016010BD0100E70361
:10DFF000F8B5054646480C464768C068804706465F
:10E00000B8470346B0B200904FF47A70B4FBF0F119
:10E01000034801FB004082B22846FFF7D5FFF8BD58
:10E0200018FCFFFF70B586B0394904460020CDE9E1
:10E03000040004A84E68D1E90351043088470490D5
:10E04000A8470546B0470146DDE90430AAB2009072
:10E0500002A8FFF7B9FFDDE90201C4E9000106B03B
:10E0600070BD00BF10B500210446016040F8041FD8
:10E07000274909698847206010BD00BFF0B587B007
:10E080000C46234905460020CDE9040004A80E688B
:10E090008F6809690430884703460490059829462B
:10E0A0002246009002A800F009F80298BDF90C4041
:10E0B000B0472046B84707B0F0BD00BF10B5C91A39
:10E0C000029B0024C0E90014D21A1304828004D5F4
:10E0D00002F57A7201398280016010BDFEB50546F5
:10E0E0000B480C464768C06880470646B847034659
:10E0F000B0B229462246009001A8FFF7DFFFBDF924
:10E100000810019A4FF47A7002FB0010FEBD00BFA8
:10E11000102A010880B51348016821F4004101600C
:10E1200001F0EEFB104801210170F2F733FD01F020
:10E1300055FA0E4801F072FA0D484FF400410160A3
:10E14000022001F06FFAFFF7DFF9F2F7BEFEFEF7EB
:10E1500033FA01F089FA01200121BDE8804001F085
:10E1600089BA00BF08000058E4180020E1E7000861
:10E1700010400058B0B59AB008AD4421281DF2F700
:10E1800091F902AC18212046F2F78CF9F4F7DCFB88
:10E19000164817490A5822F018020A500120109018
:10E1A0000A6860F34A220A600868B02100F4C0607F
:10E1B000019000201390CDE9110181200B902420C3
:10E1C000089001982846F4F711FE60B94F201421F9
:10E1D0000290201DF2F766F920460221F4F78CFC2C
:10E1E00008B91AB0B0BDF2F78BFE00BF90FCFFFF7C
:10E1F00000040058704700006148F5F7C3B800BF3D
:10E200000148F5F73ABD00BFCC4A00205C48022126
:10E21000F5F790B85A480021F5F78CB85848012115
:10E22000F5F788B8024656480221F5F787B800BFCF
:10E23000024653480021F5F781B800BF0246504816
:10E240000121F5F77BB800BF4FF47A71A0FB010103
:10E25000800A40EA8150704780B5F9F7B7FE80BD6B
:10E26000B0B5F9F7B3FE0446F3F772F80546F3F7D5
:10E270006FF8401BA04228BFB0BD00BFF7E70320E6
:10E28000704770B50446F3F763F805466FF39F20B7
:10E290004FF47A714843860AFFF7B8FFA90A26802F
:10E2A00041EA805070BD00002D480068704700BFF3
:10E2B00080B5F3F74DF82A490968401A80BD00BFC0
:10E2C00011480078012808BFF3F742B800207047D2
:10E2D00070B50D4D2878A0B9294C4FF0FF36266354
:10E2E000F9F7C2FC00F03EF8F9F741FF204626633B
:10E2F000F5F72AF80020FFF795FF00F007F8012056
:10E300002870002070BD00BFDE17002080B5F3F735
:10E310001FF81349086080BDB0B58CB001AD04464C
:10E3200028212846F2F7BEF800F01CF84FF480715F
:10E33000002001220B914FF000510890CDE9060119
:10E340000748294600682044C04302900C48F5F76E
:10E350001FF908B1F2F7D4FD00200CB0B0BD00BF2A
:10E36000E018002010B50548054C01210160F9F7BF
:10E37000FEFE4FF0FF302063002010BD5C280040FF
:10E38000884A002070B5184A0368904218BFB0F15F
:10E39000804F05D14C6823F070032343904208D08E
:10E3A000B0F1804F05D0114CA04202D0104CA042D9
:10E3B00003D1CC6823F4407323434E6923F08003D8
:10E3C0000C688D68334390420360C562846205D057
:10E3D000064A904202D0064A904201D1096901637F
:10E3E0000121416170BD00BF002C01400048014087
:10E3F0000044014010B5036A046A24F00104046279
:10E40000846924F0F00444EA0212826123F00A02D3
:10E410001143016210BD036A23F010030362836994
:10E4200023F4704343EA0232036A826123F0A002BC
:10E4300042EA011101627047F0B5EFF31082EFF389
:10E44000108372B66A4B1E8A5C8AA6420CD1C4F550
:10E450008066B5B2854216D8844214D900250126BB
:10E460001C805D829E7010E00CD2C4F58067BDB246
:10E4700085421BD8864219D900251C8001245D8263
:10E480009C7001E0361B25463446A4B2844207D96D
:10E490000D80598A08446FF39F205882002001E0C4
:10E4A0004FF6FF7082F3108800B2F0BD25463C465F
:10E4B000EBE700BFEFF31080EFF3108172B64C4929
:10E4C000CA8A0132CA8280F310887047B0B5484DBD
:10E4D000EFF31084EFF3108072B6E88A10B184F382
:10E4E000108809E0FFF7E6FF688A298A814205D192
:10E4F00000F072F884F310880020B0BDAA786AB1E9
:10E50000012A13D12B880222AA7000225B1A2A80CA
:10E51000AB821B040AD12A82AA7000E00A46114687
:10E52000904294BFC2F58060801AA882284884F384
:10E530001088441801F06EF82648A98AC26820465F
:10E54000BDE8B040104700BFB0B5EFF31080EFF367
:10E55000108172B626498C78022C03D10024002247
:10E560008C7004E00A8A8B8A1A446FF39F224B8ACC
:10E570000A829A4211D0CD8A012D0ED1ACB1012C64
:10E580001BD10D8802248C700024AD1A0C808D8262
:10E590002D0412D10C828C7008E080F3108801F0F9
:10E5A00035F8BDE8B04000F017B81446A34294BF58
:10E5B000C4F580621A1B8A82224680F310880448C0
:10E5C000898A1044034AD268BDE8B040104700BFB2
:10E5D000B0030020502A0108EFF31080EFF3108100
:10E5E00072B60349CA8A013ACA8280F3108870471A
:10E5F000B0070020F8B50120F2F754F90520F3F731
:10E60000F4FB2D492D4A2E4B2E4C2F4D2F4E002022
:10E610000027B7F5006F07D0C851D051D851E0514D
:10E62000E851F0510437F4E7294C2046F3F786FE11
:10E630002046F3F780FE202802D026A3FAF70FF831
:10E64000F2F77AF8E52806D000902AA302200021EC
:10E65000012200F06FFF2F4C2046F5F755FA2046B7
:10E66000F5F774FA10B12CA3F9F7F9FF2068314CD3
:10E6700000250026016841F0010101602580B0B24B
:10E68000B5EB502F07D121880029FCD0F5F7C8FF42
:10E6900025800136F3E70020F2F704F91D48F5F76D
:10E6A0007BFA40B124A301200021012201B0BDE882
:10E6B000F04000F03FBFF8BD6C2100206C19002035
:10E6C0006C29002078310020783900207841002022
:10E6D0003C4A00200D0A202E2E2E2E2049324320A7
:10E6E0004E6F74205265616479202E2E2E2E200DDF
:10E6F0000A0000003D204572726F723A2049324391
:10E7000020534C415645204944203D253032780D58
:10E710000A000000CC4A00203D2054696D6572203B
:10E7200032205374617274204572726F72203D0DF5
:10E730000A000000481900203D2054696D657220D0
:10E74000322053746F70204572726F72203D0D0A33
:10E7500000000000124A116819B101F1140281424F
:10E76000F9D1002918BF0121084670470C4A1168E9
:10E7700009B100230B721060416100F013B800BFB3
:10E7800010B5074909680A46496921B10B68046850
:10E790009C42F8D800E000215061416110BD00BFEB
:10E7A0004C1900202DE9F041DFF830800446D8F8FC
:10E7B0002000D8F81870804705460120266820728E
:10E7C000B8472844864203D2B8472844206000E076
:10E7D0002068D8F80810BDE8F0410847242A01084D
:10E7E000BFB5054602A80C46FFF71CFCBDF90C009E
:10E7F000029B0090284602F053FE2846F1F792FD56
:10E800002080BFBDB0B5416E91B102680C4B0D4D7B
:10E8100091689268C1F34261520F5C5C695C9B5CD9
:10E82000AA5CC900D200B1FBF4F1B2FBF3F201E043
:10E8300001220121A0F86810A0F86A20B0BD00BF35
:10E84000E07F0108D87F010810B5816ACA0706D0A9
:10E850000268C36A546824F40034234353608A076F
:10E8600006D50268036B546824F480342343536054
:10E870004A0706D50268436B546824F48024234376
:10E8800053600A0706D50268836B546824F4004479
:10E8900023435360CA0606D50268C36B946824F408
:10E8A0008054234393608A0606D50268036C9468FB
:10E8B00024F40054234393604A060FD50268436C46
:10E8C000546824F480141C43B3F5801F546005D1B0
:10E8D000836C546824F4C00423435360090606D5AE
:10E8E0000168C06C4A6822F400221043486010BDE1
:10E8F000BCB504460020C4F88C00F3F7C5FC0546FF
:10E900002068016809070BD56FF07E404FF40011B5
:10E9100000222B460090204600F0B0FB70B9206822
:10E92000006840070CD56FF07E404FF48001002254
:10E930002B460090204600F0A1FB08B10320BCBD8F
:10E940002020C4F88400C4F88800002084F88000E7
:10E95000E066BCBD806A0021A0F85E10A0F85610E9
:10E96000F5F7D5BAB0B5846A2068D4F88420D4F815
:10E9700088508168212A09D111F0800106D0002039
:10E98000A4F85600204600F053F820688068222D35
:10E9900008D110F0400005D00020A4F85E00204609
:10E9A00000F02AF8D4F88C0040F01000C4F88C0075
:10E9B0002046BDE8B040F5F7AABA0168806A096848
:10E9C000890648BFF5F728BD0021A0F85610016858
:10E9D00051E8021F026821F0800142E80213002B77
:10E9E000F5D14DF808EDF9F760FE5DF808EBF8D1C8
:10E9F0007047806AF5F71EBD10B50168F9F794FC01
:10EA0000FBD1E549026852E8022F03680A4043E857
:10EA10000224002CF6D1C16E012902D1F9F7B2FF10
:10EA2000FCD12021C0F8881000210167C16610BD0B
:10EA3000016851E8001F026821F0C00142E800139C
:10EA4000002BF5D14DF808EDF9F71BFC5DF808EB4C
:10EA5000F8D12021C0F8841070470168D0F88820D0
:10EA6000222A39D1B0F860204B6A1A40836D23F80E
:10EA7000022BB0F85E20013AA0F85E208365B0F862
:10EA80005E200AB1704701684DF808EDF9F74CFCBB
:10EA90005DF808EBF7D14DF808EDF9F727FF5DF8C1
:10EAA00008EBF8D12021C0F8881000210167C26E60
:10EAB000012A18BFF5F748BCC1664DF808EDF9F713
:10EAC00061FF5DF808EBF8D10168CA69D20601D58B
:10EAD00010220A62F9F7D4BCF9F704BD2DE9F84F0A
:10EAE000F9F703FC63D1B4F86870AB4EF9F78CFD0D
:10EAF000002F61D01AF020005ED02068A16D426A1C
:10EB00002A4021F8022BB4F85E20013AA4F85E20D6
:10EB1000A165D0F81CA05FEA4A711ED05FEACA72F4
:10EB200018BFB8F1000F01D0F9F7A1FC5FEA8A72B3
:10EB300004D5B9F1000F01D0F9F739FC002904D54B
:10EB4000B9F1000F01D0F9F71CFCD4F88C0020B10A
:10EB50002046F5F7DCF9C4F88CB0B4F85E00002864
:10EB6000C6D1206850E8000F216820F48070F9F7C2
:10EB700022FEF6D1206850E8020F21683040F9F7F4
:10EB8000FAFCF7D1F9F783FC0DD1C4F86CB0F9F7B2
:10EB90008EFAFCD12068C169C90601D51021016235
:10EBA000F9F7CEFCA4E72046F5F7CEFBA0E7816994
:10EBB00041F0080181611AE0B4F85E00B8B1B4F820
:10EBC0006810884213D2206850E8020F216820F0B4
:10EBD0008050F9F7D0FCF6D106482067206850E84D
:10EBE000000F216840F02000F9F7E5FDF6D1BDE8FF
:10EBF000F88F00BF5BEA00080168D0F88820222A5D
:10EC00003AD1B0F86020496A1140826D1170B0F8B5
:10EC10005E100139A0F85E10816D01318165B0F898
:10EC20005E1001B1704701684DF808EDF9F77CFB03
:10EC30005DF808EBF7D14DF808EDF9F757FE5DF8F0
:10EC400008EBF8D12021C0F8881000210167C26EBE
:10EC5000012A18BFF5F778BBC1664DF808EDF9F742
:10EC600091FE5DF808EBF8D10168CA69D20601D5BA
:10EC700010220A62F9F704BCF9F734BC2DE9F84F09
:10EC8000F9F733FB65D1B4F86870434EF9F7BCFC73
:10EC9000002F63D01AF0200060D02068A16D406A78
:10ECA00028400870B4F85E000138A4F85E00A16D39
:10ECB00020680131A165D0F81CA05FEA4A711ED01E
:10ECC0005FEACA7218BFB8F1000F01D0F9F7CFFBA5
:10ECD0005FEA8A7204D5B9F1000F01D0F9F767FB3A
:10ECE000002904D5B9F1000F01D0F9F74AFBD4F897
:10ECF0008C0020B12046F5F70AF9C4F88CB0B4F8BE
:10ED00005E000028C4D1206850E8000F216820F47C
:10ED10008070F9F750FDF6D1206850E8020F2168A5
:10ED20003040F9F728FCF7D1F9F7B1FB0DD1C4F861
:10ED30006CB0F9F7BCF9FCD12068C169C90601D5EE
:10ED400010210162F9F7FCFBA2E72046F5F7FCFA77
:10ED50009EE7816941F0080181611AE0B4F85E0024
:10ED6000B8B1B4F86810884213D2206850E8020F96
:10ED7000216820F08050F9F7FEFBF6D1BE482067ED
:10ED8000206850E8000F216840F02000F9F713FDDB
:10ED9000F6D1BDE8F88F00BFFEFFFFEF70B5016848
:10EDA00004468068674ED4E903230D681843E3697D
:10EDB000354066693043654E18432843624D08600C
:10EDC000486820F4405010434860A942A0691CBF25
:10EDD000226A10438A68324010438860626AC86AB7
:10EDE00020F00F001043C8625948814208D0A94260
:10EDF0000AD05848814210D1574859A6006807E008
:10EE000055480068800802E053480068800A534E65
:10EE100000F0030056F8206000E010265448A94294
:10EE200010D00121B3F5004F1AD1082E00F28180D5
:10EE3000DFE806F00546507F497F7F7F4E00F3F7FD
:10EE400045FF42E00121082E00F27380DFE806F062
:10EE500005711C71147171711A00F3F737FF0DE021
:10EE6000082E66D8DFE806F0054953654C656565F0
:10EE70005100F3F72BFF45E0F3F744FF002855D08E
:10EE8000626A01E04FF400403A4931F812106268BA
:10EE9000B0FBF1F002EB4201884249D3B0EB023FF4
:10EEA00046D8010E000210EB520041F10001002390
:10EEB000F1F7C0F9304AA0F54071914234D937E0FA
:10EEC000F3F710FF01E0F3F71DFF78B3626A01E08A
:10EED0004FF40040274931F81210B0FBF1F061689F
:10EEE0004A0802EB4000B0FBF1F04FF6F071014030
:10EEF0001ED0C0F34200084316E0F3F7F3FE01E032
:10EF0000F3F700FF90B1626A01E04FF40040194945
:10EF100031F81210B0FBF1F0616800EB5100B0FB6A
:10EF2000F1F080B2102803D32168C860002100E00E
:10EF300001210020C4E91C004FF00110A066084622
:10EF400070BD00BFF369FFCF00800040FFF4FF11E8
:10EF5000004400400038014088000058C87F010884
:10EF60000100000004000000020000000800000092
:10EF70000024F400E0290108FFFC0F0010B5A0F800
:10EF80005E2081650021A0F85C200167816851B195
:10EF9000B1F1805F0BD0B1F5805F0CD1016921B96F
:10EFA00040F2FF110AE0016939B9FF2106E0016969
:10EFB00019B13F2102E0002100E07F21A0F860109C
:10EFC0000021C0F88C102221C0F88810016851E897
:10EFD000021F036841F0010143E80214002CF5D13F
:10EFE000416EB1F1005F03D1B0F86810914221D9B0
:10EFF00082680021204BF9F71FFB1E4A08BF134609
:10F00000036718BF00290AD1016851E8001F026890
:10F0100041F0200142E80013002BF5D124E0016803
:10F0200051E8001F026841F4907142E80013002B80
:10F03000F5D119E0826800210D4BF9F7FDFA0B4A72
:10F0400008BF1346036718BF002903D00168F9F70A
:10F05000B6FAFBD1016851E8021F026841F0805105
:10F0600042E80213002BF5D1002010BDDDEA0008B4
:10F070007DEC00085BEA0008F9EB00082DE9F84395
:10F08000DDF8209004460068984616460F4609F1C0
:10F090000105C1693940C91BB1FA81F14909B14281
:10F0A0001ED1002DF5D0F3F7EFF8A0EB080048458E
:10F0B00019D8B9F1000F16D0206801684907E8D5C2
:10F0C000C1690905E5D54FF40061016250E8000F00
:10F0D000216820F4D070F9F76EFB1CD02068F5E7AA
:10F0E0000020BDE8F883206850E8000F216820F474
:10F0F000D070F9F760FBF6D1206850E8020F216864
:10F1000020F00100F9F737FAF6D12020C4F8840086
:10F1100004F188000FE0206850E8020F216820F019
:10F120000100F9F728FAF6D12020C4F88400C4F8C9
:10F13000880004F18C00002184F8801020210160F7
:10F140000320BDE8F88300000148F4F7E1BE00BFEA
:10F15000184B0020F0B599B009AD0E460446402189
:10F160002846F1F79FF92078052E2AD8592828D16A
:10F170006078442800F09780462800F0C080482836
:10F1800000F0C5804F2800F0CA80562800F0DA80D1
:10F190005A2840F0D480A078432800F01D815328DD
:10F1A00000F02D81482840F02881DCA201201421A4
:10F1B000FDF7CCFB41F28830F2F717FEF9F7F6FFC6
:10F1C0001BE1042EC0F0BB80502840F0B880A0782E
:10F1D000A0F13001022962D26078312840F0C1806C
:10F1E000092E2BD1E078202521796279A37900EBD3
:10F1F000800005EB4006B04806700678314430398F
:10F20000017002EB8201AD4A05EB410111701178EA
:10F210001944AB4B30391170E17901EB810105EBF9
:10F2200041011970217A1C78214430391970017814
:10F230001278914202D8017802310170FDF7AAF8E4
:10F24000DFF874C29D4A9E4C9E4E002703209CF816
:10F2500000101378257886F820705A2786F82170D8
:10F26000012786F8227086F8237086F827009CF81C
:10F27000000086F82800107886F82900207886F8A3
:10F280002A0091488DF828708DF829108DF82A30C1
:10F290008DF82B500990F9F731FF0821AAE03228A8
:10F2A00000F0AB804BE0A078A0F13001092946D8EE
:10F2B000E178A1F13002092A41D82579A5F1480267
:10F2C0000B2A3CD8012303FA02F240F621031A422A
:10F2D00035D000EB80007D4E482D01EB4000A0F5BD
:10F2E0000470706000F08E80532D00F090804D2DE2
:10F2F00040F092807068C0EB001080008BE0A07836
:10F3000039281CD83038C0B2FDF704FB0EE0A078D5
:10F31000392814D83038C0B2FDF7F4FA06E0A078E6
:10F3200039280CD83038C0B2FDF7FCFA2078032118
:10F330008DF82400B4F80100ADF825005AE0FDF77F
:10F34000FBFA5AE0A078432813D0482855D16F48DB
:10F3500008212A460A906E480990F9F77DF96D4B0D
:10F3600038E0FDF7E9FA4AA30120F8F737FE032158
:10F3700040E001AC2021F9F7EBF82046F9F78CFDCD
:10F380009DF8041043209DF808208DF824009DF876
:10F390000B008DF82510BDF805108DF828200122EE
:10F3A0008DF82B00ADF82610BDF80910ADF8291026
:10F3B0000821D3B2834207D854FA82F3CEB2013285
:10F3C0000131DB79AB55F4E7C9B201202A46FDF7DC
:10F3D000BDFA4D4B009557E000208DF8040001A8C0
:10F3E000F5F7D2FB4C48052109909DF80400413007
:10F3F0008DF8280009AAF9F72FF919B0F0BDFDF72B
:10F400000DFAFAE770684FF46161484303E07068F1
:10F41000092801D80A20706070684FF47A71484357
:10F42000F9F78AFF2078052101278DF82400D4F808
:10F430000100CDF8250009AAF9F70EF921480021AD
:10F4400080F820105A2180F8211080F8227080F86E
:10F450002370A178303980F82410E178303980F8B1
:10F4600025102179532908D171680A2905D1012174
:10F4700080F82410002180F8251080F82650F9F734
:10F480003DFE706812A300900120F8F7A7FDB4E7D5
:10F49000232323232323204D544D20564552204916
:10F4A0006E76616C6964206F72204D69736D617452
:10F4B00063680D0A000000004200002043000020A5
:10F4C000440000200000002050005A0148030020A2
:10F4D0002323232323232059554E484F524E205097
:10F4E0006572696F646963697479204368616E67E6
:10F4F000656420746F205B202564205D2053656364
:10F500006F6E64730D0A00008983010803170A0EE9
:10F5100056005A01B98301084C005A012159756EF1
:10F52000486F726E20535453205265766976652178
:10F530000000000070B586B01C460023ADF8023014
:10F540003A4B1D7A854201D2FB2042E0D868084040
:10F5500088422AD132B15A6822B10DF105000DF16D
:10F56000020190471C480AAB4FF4007122460593F4
:10F5700001F0AAFF0546FEF79DFFBDF802006946AF
:10F58000284480B2FEF758FF01301FD0BDF802209A
:10F59000BDF800101A4B0DF1050042B110F8015BE7
:10F5A0008EB2013A01319D55F7E7FA2011E013FAC6
:10F5B00081F0059BADF800104FF40071224601F078
:10F5C00083FFFFF709F8FEF781FF02E0FFF704F879
:10F5D000FD2040B206B070BDD44B002080B513486A
:10F5E0000021182200F07DF8054800214FF48062C8
:10F5F00000F077F8034801680348BDE880400847F9
:10F60000B0030020502A010849E50008022000212B
:10F6100000F046B80220012100F042B803494860DA
:10F62000704700BF01490872704700BFB007002053
:10F63000B0B5EFF31084EFF3108072B62348016881
:10F6400019B10848D0E9001507E0406800280548CE
:10F650000CBFD0E90415D0E902158847A84784F308
:10F660001088B0BDF829010818480021C0E9001130
:10F67000704700BFEFF31082EFF3108372B629B129
:10F68000012909D111494968084303E00F49496834
:10F6900021EA00000D49486082F31088704700BFDE
:10F6A000EFF31082EFF3108372B629B1012909D16B
:10F6B00006490968084303E00449096821EA000093
:10F6C0000249086082F31088704700BFB80200202A
:10F6D000130408BF704711F8013B013A00F8013BE1
:10F6E000F6E7130408BF704700F8011B013AF8E77A
:10F6F000FFF79EBF70477047B0B5EFF31085144613
:10F70000EFF3108172B6FCF727FE424901EB80004F
:10F71000846185F31088B0BD2DE9F047DFF8CCA0F7
:10F720003C4E4FF0FF390125DAF8048006F1080459
:10F7300000EA0800CAF8040033687168DAF80020AB
:10F740001040B268184230D011402ED1274657F8E9
:10F75000081F0842FBD0396808407968084208BF92
:10F76000C7F8049079680840FCF7F6FDF06005FAE8
:10F7700000F0796821EA00007860EFF31080EFF381
:10F78000108172B63168F26805FA02F29143316075
:10F7900031699143316180F31088F06806EB800095
:10F7A00080698047DAF80400C6E74FF0FF30F06068
:10F7B000FFF7A1FFEFF31084EFF3108072B631680A
:10F7C0007068DAF800201140DAF80420114204D100
:10F7D000B168014208BFFFF78BFF84F31088FFF781
:10F7E00089FFCAF80480BDE8F08700BFA0000020B0
:10F7F00010B5EFF31082EFF3108372B6054B1C685F
:10F8000003EBC10104431C600B691843086182F3D8
:10F81000108810BDC00200202DE9F041012490B1F4
:10F820001F4683B1002406461546DDF818800460A3
:10F830007648426A08469047B47234817060C6E9DF
:10F8400003787461F5722046BDE8F08110B56F4809
:10F85000C169846A88472146BDE81040084700BF57
:10F86000F8B504466948C169D0E909678847054683
:10F870002046B047281A3946BDE8F840084700BF7F
:10F880002DE9F843614EEFF31088EFF3108072B664
:10F89000D6E9044080470546A0475B4F3C6854B119
:10F8A000401B21460A684B69121A38BF00220A60C1
:10F8B000002B1946F6D1B5694FF00009E4B126686E
:10F8C0001EB1A8473C68864210D2A4F8089062692D
:10F8D000D4E903103A608847E07A012804D1A07A7D
:10F8E00010B9204600F02AF83C68E7E724B1207AF6
:10F8F00010B92046FEF756FF88F31088BDE8F8835C
:10F9000041480021016041480068004710B588B1B6
:10F9100004463E48426A0846904760602046FEF72B
:10F9200019FF48B1204600F03FF82046BDE81040DE
:10F9300000F004B8012010BD002010BDF8B528B1BA
:10F940000446FEF707FF08B9607A08B10120F8BD48
:10F950002E4EEFF31085EFF3108072B66768306AB1
:10F9600080470021A1724FF480718742218138BF06
:10F9700007462760244F386860B1B0698047216826
:10F980000844396820600968884205D32046FEF79C
:10F99000F7FE04E0306980472046FEF7E7FE85F376
:10F9A00010880020F8BD00BF012158B3B0B5164D36
:10F9B000EFF31084EFF3108272B681722968E1B11F
:10F9C00000228142427207D00A46B2B182420AD076
:10F9D000536911461A46F8E70272406940B128603F
:10F9E000FEF7E0FE09E0406900B90020486104E04C
:10F9F0000648C06880470020286084F310880021F2
:10FA0000BDE8B040084670474C190020242A010880
:10FA1000FEE7000010B504460748016A2046884703
:10FA200028B10648844202D30548844201D9002007
:10FA300010BD012010BD00BF4C290108C0CA893685
:10FA40000028503710B5074C00F00F03B0F1FF3F0E
:10FA5000034A2344C8BF83180801187010BD00BFB3
:10FA600000E400E014ED00E00648BFF34F8F064AC3
:10FA7000016801F4E06111430160BFF34F8F00BFE3
:10FA8000FDE700BF0CED00E00400FA05F0B500232F
:10FA90008B4228BFF0BD02EB430632F8134002331D
:10FAA000768824F0030426F0030605598759075188
:10FAB0008551044406446568776867607560E7E7C8
:10FAC0002DE9F0410588984616460C460746012A5E
:10FAD00009D1201D294631B10268013982F0004266
:10FAE00040F8082BF7E7102D14D0202D1ED0402D04
:10FAF00015D0802D0ED0B5F5807F17D0B5F5007FDD
:10FB00000DD0B5F5805F0AD0B5F5006F0ED0B5F514
:10FB1000806F0FD13846214600F078F80AE07A6805
:10FB200020462946012300F077FC03E038462146B1
:10FB300000F086F9B8F1000F04D0BA68B989204600
:10FB4000FFF7A4FF012E16D1284602F0E3FB014681
:10FB50004FF07E5002F094FA064665B1D4E90017E2
:10FB6000F8F7C0FB206087F00041F8F7BBFB60604E
:10FB70000834013DF1E7BDE8F0810000002201807A
:10FB80001029426016D0202916D0402916D080298D
:10FB900016D0B1F5807F15D0B1F5007F14D0B1F546
:10FBA000806F13D0B1F5805F12D0B1F5006F18D11E
:10FBB000154B0EE00D4B0CE00D4B0AE00D4B08E031
:10FBC0000D4B06E00D4B04E00D4B02E00D4B00E049
:10FBD000054B4DF808EDF8F789FD5DF808EB40B2EC
:10FBE0007047FF20FBE700BF987F0108587F01089E
:10FBF000887F0108B87F0108487F0108787F0108E5
:10FC0000A87F0108387F0108687F01082DE9F04FBF
:10FC10009DB00388059101EB83024FEA830B0292AA
:10FC20005A08019203904068970007EB8302049002
:10FC3000D8080023002800F0F1801590059800EB0B
:10FC40000B0500EB0308C4198618049829681844AA
:10FC50000B90D8F8000009900891CDE9172714936C
:10FC600002F076F97168D6F80CA0D4F80890E7682D
:10FC70006A681A91B1681C916168CDF848A00C9629
:10FC80001B912946CDF8449013970A950692AD68CA
:10FC90003268C9680E95109107922268C8F8000072
:10FCA000D8F80C001992CDF858B0D8E901B60D96E5
:10FCB0000F9002F04DF9C8F80C003046F8F740FB01
:10FCC000069DC8F808005846F8F73AFBC8F8040043
:10FCD0003846F8F73AFC1C99E060484602F038F9DB
:10FCE000A060DDE91A1002F033F9DDF81C806060D5
:10FCF0001998F8F790FC2060DDE9081002F0DAFCB2
:10FD000007465846F8F7CAFADDF82CA00546DAE9A6
:10FD10000094F8F7E4FB06463846F8F70EFCF8F7CF
:10FD2000CDFBDDF828B04946CBF80400F8F76EFDAE
:10FD300006462846F8F701FCF8F751FC1999CBF86C
:10FD40000000F8F705FD0546DDE91A0102F0B2FCF6
:10FD50002146064602F05AFB07462846F8F7BFFB45
:10FD6000F8F782FB0C9F21467860F8F725FC0446E3
:10FD70003046F8F7B4FBF8F7F6F93860B946DDE934
:10FD80000D0102F097FC0646DDE90F0102F092FC3E
:10FD9000DAE902850746F8F707FB04463046F8F72C
:10FDA000B2FBF8F7E0F9CBF80C003046F8F7FCFAB4
:10FDB00004463846F8F7A7FBF8F7F3FBCBF8080042
:10FDC0001C98119902F076FC0446DDE9120102F05C
:10FDD00071FC2946064602F019FB07462046F8F753
:10FDE000E3FAF8F741FBC9F80C0020462946DDF894
:10FDF00058B002F00BFB04463046F8F7D5FAF8F796
:10FE0000B2F9DDE91727149BC9F8080015980BF122
:10FE1000100B10371032103301380BE7019C059896
:10FE2000049A0223214600F0F7FA039821460223A0
:10FE3000426802981DB0BDE8F04F00F0EDBA000036
:10FE40002DE9F04FA9B00490008889464FEA500B85
:10FE5000279001EB8B0858F82B102291D9E9005616
:10FE60002846219602F074F859F82B102890259115
:10FE700002F06EF808EB8B0454F82B10239102F07B
:10FE800067F8D4F804A0C9F800003046F8F75DFB25
:10FE9000D8F804602690F8F7DCFB04EB8B014F6880
:10FEA0000391F8F7E1FA2299C9F80400F8F766FA25
:10FEB0003146229002F04CF8F8F7E5FCCDF890902E
:10FEC00049F82B005146219802F0F4FBDDF894909C
:10FED0000546F8F74EFCDDF88CA0F8F736FBC8F8BD
:10FEE00004002898F8F745FCF8F7B0FBCDF8088037
:10FEF00048F82B003146269802F0DCFBF8F7C3FCEB
:10FF000060602298F8F77DFBF8F7AEFA44F82B0012
:10FF100028464946019402F01BF8F8F797FB03992D
:10FF20004FEA8B0648606FF0030000EB8B0100EB9B
:10FF3000CB0020911F906FF0070000EB0B11269172
:10FF40000BEB4B0100EB81008F0028906FF001005C
:10FF5000279A00EB9200400823900498406805908F
:10FF600090084FEACB0200900020279000202290BA
:10FF700000202190249D27982C18A818D4E9029AD3
:10FF80001392D0F808801A90C06819904846F8F784
:10FF900042FB05EB060B25901296DBF80810DBF808
:10FFA0000C201E911C9201F0D3FFEE191197B1683D
:10FFB000F7681D9101F0CCFF199DA0605046F8F73D
:10FFC000BFF9DBF80C10CDF85CB0834601F0C0FF40
:10FFD000F1681B9601F0BCFFE0604846F8F70EFCA4
:10FFE0001C9C8146F8F797FCF8F74DFC169050469C
:10FFF000F8F754F9DDF878A00646F8F727FB1D9DC1
:020000040801F1
:10000000F8F79EF915905146259802F053FBF8F742
:1000100045F919905846F8F742FAF8F734FC80464B
:100020004846F8F73CFAF8F71FFA18903046F8F708
:100030008CFAF8F733F90546059821994418229966
:1000400001441491279900EB010B2398002800F03C
:100050003881CDF82C802499CDE90E451F9889462A
:100060000F18099720980E1828980A1805460D921F
:10007000289026980C188246306851681094089091
:10008000079101F065FF39680C901E9101F060FF47
:1000900061681D9101F05CFF59F80A2059F80510BC
:1000A00056F8045CCDF898A04C461C9257F8042CE6
:1000B000306028462592069101F04AFF57F8041C4B
:1000C0000A9001F045FF59F80A1001F041FF46F887
:1000D000040CDDF85490DBF808604846F8F71BFA8A
:1000E000DBF80CA0169F80463846F8F71AF901464F
:1000F000F8F72EFB179C3146E060F8F787FB0746C0
:100100004846F8F70EF90146F8F783FB0699A06018
:10011000F8F734F916900446DDE9071002F0CAFA40
:1001200017900546DDE91D1002F0C4FA014615904E
:10013000204601F00DFF25990446F8F71FF9DDF878
:1001400070B0594601F004FF05462046F8F7E9F87B
:1001500007462846F8F7DFF9F8F786F9099F514670
:1001600047F8040CF8F728FA05462046F8F7D3F9C3
:10017000F8F7A4F8149D38600B9FD5F81090384616
:10018000F8F7ADF9D5F81480199E04463046F8F713
:100190000BF9F7F7E8FF1A9D4946E860F8F7A2F86F
:1001A00004463846F8F700F9F8F7FBF9A8600A9812
:1001B000259902F07FFAF8F7C8FA04460C981E99C0
:1001C00002F078FA1D9902F075FA05462046F8F714
:1001D00086F906462846F8F7E7F8F8F712FADDF848
:1001E00090B028994BF8010085F00041484602F094
:1001F0000DF905462046F8F7D7F8F8F75FF80D999E
:100200000E9C0F9F48603846D4F81880F8F7CCF859
:10021000D4F81CA0189D06462846F8F782F8F8F78F
:100220004DF91B9C4146E060F8F7C6F90646384692
:10023000F8F777F8F8F7D3F9A060DDE9150102F0D7
:1002400039FA81461C98259902F034FA179902F080
:1002500031FA07464846F8F764F804463846F8F796
:10026000A3F8F8F758FB269E51464BF80600F8F71E
:10027000CDFA04464846F8F797F8F7F774FF109957
:1002800048602098083820901F9808381F902898B8
:10029000083828903046A6F10800269027980830A4
:1002A000279022981030229021981830219023987E
:1002B000119F139A129E013808370832083623908E
:1002C00058E6DBE902A7DDF854904846F8F729F82C
:1002D000169E83463946F8F705F80146584602F05F
:1002E000E9F9DDF85CB05146CBF80C00F7F7FAFFFE
:1002F00006464846F8F7C8F8F8F771F9CBF8080051
:1003000014984746D0E904A94046F8F70AF8199E20
:1003100080464946F7F7E6FF0146F8F719FADDF897
:1003200068805146C8F80C00F7F7DCFF06463846EF
:10033000F8F7D5F8F8F753F9C8F808002846D4E9D3
:100340000679F8F7A1F8189C06464946F8F7EAF945
:10035000F8F7B4F81B9E3946F060F8F7E3F9044665
:100360002846F8F7BCF8F8F71CF9009DB0600D4E70
:100370002498059A04232946B047049C02982946EC
:1003800004236268B0476268019829460423B04795
:100390006268039829460423B44629B0BDE8F04FAB
:1003A000604700BF190401082DE9F0411446884652
:1003B000064674B1F8F710FAF8F793F901462846A3
:1003C00001F0C6FD01F0C0FA48F8040B0836013C04
:1003D000EFE7BDE8F0812DE9F84FF8F7E6F8009275
:1003E0005BF8047BC24513D05BF8045B38462946B2
:1003F00001F033FE06463846294601F02EFE00285D
:1004000018BF444608F10108002E18BF2F46E9E73F
:100410000098F8F78DB800002DE9F04FC1B00E46F6
:1004200000F10C01CDE90232043033460091019015
:100430000B96D908DA00DDF804A0C8004FEA0119CC
:100440000591CDE90C238046A0EBD300C0003A9083
:1004500048013E9001EB8100C50001EB4100C10065
:100460004FEA001B40913BA80021CDF8FCB080E88A
:100470002003399129465AF808004F46DDF8F890D4
:1004800045465AF801102F902E9101F061FD044667
:10049000329040985AF800203A985AF800101046C6
:1004A00027922B9101F054FD01463190204601F036
:1004B0004FFD04465AF80910DAF800002D912C90EF
:1004C00001F046FD06465AF807005AF80B10369020
:1004D000359101F03DFD01463090304601F038FD88
:1004E0002146074601F034FDCAF800003846F7F708
:1004F000D6FF4AF809000AEB0800349050F8048C43
:100500003B98504450F804BC38904046594601F09E
:100510001FFD0546269040985044379050F8044CF3
:100520003A98504450F8047C33902046F7F79CFFEB
:1005300001462590F7F722FF30998146304602F0B8
:10054000B9F84946054602F0B5F83D994AF8010068
:100550004846F7F7F5FE3F994AF801004046F8F79C
:10056000F4F805462A902046F8F78DF901462990BF
:10057000F8F7DBF870490D4601F048FF044630906B
:10058000DDE92E1002F096F80646289027982B9960
:1005900002F090F801462790304602F08BF8F7F70A
:1005A000B2FF07462E903D980AEB000B3F985BF890
:1005B000045C504450F8046C24902846F8F721F865
:1005C00021462F9001F0C4FC04462B90DDE92C015C
:1005D00002F070F839462D9001F0BAFC21462C90BB
:1005E00002F068F83C994AF80100DDE9251001F0B5
:1005F000AFFC07463E985AF8049C0AEB00084846B0
:1006000058F8041C269101F0A3FC04462846F8F78C
:1006100020F805462046F7F793FE3946064601F0D6
:1006200097FC4AF8040C3046F8F72DF948F8040C0A
:10063000DDE9311002F03EF806462046F7F72EFEBF
:100640003146044601F084FC4BF8040C2046F7F7D1
:10065000D8FF249941F8040CDDE9291002F02AF8AA
:10066000354CF7F76AFF0546DDE9271001F070FC0D
:10067000F7F763FF269983464846DDF8F08002F0DD
:1006800019F82946044601F063FC0746DDE93510F8
:1006900002F010F85946814601F05AFC06463846E9
:1006A000F7F7D7FF349941F8040C314638460B9ED2
:1006B00002F000F8339941F8040C2046F7F7EEFDFC
:1006C000044648463B9DDDF8F490F8F73EF80746AF
:1006D0002046F7F7C9FE389941F8040C2046F8F790
:1006E000D2F8379941F8040CDDE92B0101F030FC18
:1006F0003A994AF80100DDE92F0101F0DBFF0446D9
:10070000DDE92D0101F0D6FF2146074601F0D2FFB9
:100710004AF8050020463946DDF8FCB001F018FC27
:100720004099DDE90C234AF80100399992441944B3
:10073000B142FFF49EAE01E0F304353F402BC0F020
:100740006A820298DDF800900023012480B20490B0
:100750000598C0EBC0004FEAC008CDF8B8800498F7
:100760000399034451F83300C3EBC30603EB830C36
:100770005D0103EB430E08933A9051F8360039902F
:1007800051F83C0038904859379051F83E000A9093
:1007900018010A5836922A1D8A583592021D885827
:1007A000DA000432349088584FEA0E123390885899
:1007B0003290F000043008583190101D08583090E5
:1007C0004FEACC00043008582F904FEACE00043096
:1007D0000858CDE9069409903C993B9A2D9459F814
:1007E00001000C4659F8021017461990189101F0B3
:1007F000AFFB05462190409859F8081059F80000C1
:100800001691179001F0A4FB01462090F7F78DFF99
:10081000054625903E9859F80010D9F800001D9122
:100820001C9001F095FBDDF8F4A059F80B1006467A
:100830001F9059F80A001A911B9001F089FB01469C
:100840001E90304601F084FB2946834601F080FB70
:10085000C9F8000009EB040009EB0701299050F8E2
:10086000040C2B9151F8041C1190109101F070FBB5
:100870000546409809EB08012A9151F8041C4844A8
:100880002C9050F8040C0E910F9001F061FB804603
:100890002846F7F7C0FE074624903E98484450F893
:1008A000041C269059F8040C1391129001F050FB8F
:1008B000064609EB0A0050F8042C27903F9848445C
:1008C000159250F8041C28901046149101F040FB3A
:1008D00082463046F7F739FE3946239001F0EAFEAA
:1008E000259907462290584601F0E4FE01462590DE
:1008F000379801F08BFD04463598F7F7C5FDF7F7FB
:1009000032FC3E9949F801002846F7F777FF804608
:10091000DDE9201001F0CEFE83463046F7F796FE63
:100920005946064601F014FB05462090DDE91E10ED
:1009300001F0C0FE4146074601F0BCFE0146219091
:10094000369801F063FD04463498F7F7DCFDF7F7BD
:100950000AFC3D9949F801003046F7F7F6FE0546D6
:100960001E904046F7F780FD01461F90329801F037
:100970004DFD04463098F7F7C6FDF7F7F4FB3F99B5
:1009800049F80100DDE9101001F094FE8246DDE92E
:100990000E1001F08FFE80465046F7F72FFF9F495B
:1009A0000E4601F033FD05461190DDE9181001F007
:1009B00081FE0746DDE9161001F07CFE044638464C
:1009C000F7F7A9FFF7F7A7FD06461890DDE9120132
:1009D00001F070FE2946199001F0BAFA054612900E
:1009E000DDE91A1001F066FE3146179001F0B0FA09
:1009F00001461A90F7F799FE83461B905046F7F789
:100A00000AFE864EF7F787FD054616903846F7F73B
:100A100046FDF7F780FD04461390DDE9141001F060
:100A200049FE2946159001F093FA0646DDE91C01BE
:100A300001F040FE2146824601F08AFA314607461F
:100A400001F038FE01461D903A9801F0DFFC0546A2
:100A50003398F7F790FCF7F731FC3C9949F801001F
:100A600012981A9901F026FE04461A903046F7F7BC
:100A7000FBFC01461C90399801F0C8FC05463198F2
:100A8000F7F75BFDF7F71AFC2E9949F80100199862
:100A9000119901F00FFE8346DDE9170101F00AFE0E
:100AA00080465846F7F7B7FD07461890DDE915016F
:100AB00001F000FE13990546504601F0FBFD294662
:100AC000044601F0F7FD01461990389801F09EFCAC
:100AD00006462F98F7F7D8FCF7F7F0FC3B9949F852
:100AE00001005846F7F78AFE07462846F7F713FF36
:100AF0000A9E82465146F7F7F5FB099D04463946A2
:100B0000F7F75AFDF7F72FFB409949F80100DDE9A7
:100B1000230101F01DFA49F8040C3798229901F0DD
:100B200075FC04463598259901F070FCF7F739FDFE
:100B3000269941F8040C3698209901F067FC044688
:100B40003498219901F062FCF7F7E5FE279941F806
:100B5000040C32981E9901F059FC044630981F99F4
:100B600001F054FCF7F7D7FE289941F8040C3A98A5
:100B70001B9901F04BFC044633981D9901F046FC8B
:100B8000F7F70FFD299941F8040C39981A9901F0EB
:100B90003DFC044631981C9901F038FCF7F701FD43
:100BA0002A99DDF8B88041F8040C3898189901F0BA
:100BB0002DFC04462F98199901F028FCF7F7F1FC59
:100BC0002B99DDF8FCB041F8040C3046F7F75CFCDB
:100BD0000446284651460B9E01F018FCF7F7E1FC4D
:100BE000DDE92C1441F8040C0C9881440D98044460
:100BF000B442FFF4F1AD079CDDF818900598089B0E
:100C0000013409F108098442FFF4A9AD0298059B5B
:100C1000C00002900DE441B0BDE8F08FF304353F11
:100C200010B558B14FF40071F7F77FFC38B905489B
:100C300060614FF480602082002000E0FF2040B21D
:100C400010BD00BF4486020810B548B14021F7F737
:100C50006CFC30B90448606180202082002000E0F4
:100C6000FF2040B210BD00BF4496020810B558B135
:100C70004FF48061F7F759FC38B9054860614FF4CB
:100C800000602082002000E0FF2040B210BD00BFC5
:100C90004498020810B550B18021F7F746FC38B9E6
:100CA000044860614FF480702082002000E0FF2043
:100CB00040B210BD44B8020810B548B11021F7F792
:100CC00034FC30B90448606120202082002000E01C
:100CD000FF2040B210BD00BF44BC020810B558B19F
:100CE0004FF40061F7F721FC38B9054860614FF413
:100CF00080502082002000E0FF2040B210BD00BFE5
:100D0000C4BC020810B558B14FF48071F7F70DFC60
:100D100038B9054860614FF400702082002000E07F
:100D2000FF2040B210BD00BFC4FC020810B548B19E
:100D30002021F7F7FAFB30B9044860614020208297
:100D4000002000E0FF2040B210BD00BFC404030833
:100D5000F8B514460E46054673B12846314622467C
:100D60001F4600F095FA284621463A46012301B075
:100D7000BDE8F040FEF7A4BE28463146002201231C
:100D8000FEF79EFE284631462246BDE8F84000F0B8
:100D90000FBB0000202917D0402917D0802917D079
:100DA000B1F5807F16D0B1F5007F15D0B1F5806F19
:100DB00014D0B1F5805F13D0B1F5006F1CBF4FF0B8
:100DC000FF3070470E490847074908470749084759
:100DD0000749084707490847074908470749084797
:100DE00000490847DD0C0108B90C01082D0D010868
:100DF000490C0108950C0108050D0108210C01089A
:100E00006D0C010810B50B781478634003704B78B3
:100E10005478634043708B78947863408370CB78C8
:100E2000D4786340C3700B791479634003714B79B4
:100E30005479634043718B79947963408371CB79A2
:100E4000D4796340C3710B7A147A634003724B7A8E
:100E5000547A634043728B7A947A63408372CB7A7C
:100E6000D47A6340C3720B7B147B634003734B7B68
:100E7000547B634043738B7B947B63408373C97B58
:100E8000D27B5140C17310BD2DE9F04F8DB0164695
:100E9000024696F8F000002800F04A8101911146C0
:100EA00009A83246FFF7AEFFDFF88CB2A34DDFF89A
:100EB000888306F110040120029696F8F0109DF840
:100EC0002420884280F0DE809DF8273008949DF829
:100ED0002A409DF825A09DF830C007909DF832E08B
:100EE0009DF8319006929DF8262004939DF82830B5
:100EF00018F8041018F80A7003931BF80C3087EAEE
:100F0000010058409DF82F30EE5C46409DF83300BC
:100F10008DF8336018F80C600590285D1BF80440CC
:100F2000774078401BF8037078408DF8320018F84D
:100F3000030086EA000315F80A60734063401BF85B
:100F40000A408DF8313015F80C309DF82EC0634002
:100F500018F8024059409DF82C3048408DF8300078
:100F600018F809001BF8036080EA040171409DF83D
:100F70002B60AF5D794018F80370EB5C8DF82F1093
:100F8000A95C1BF80220784048401BF80610484036
:100F900003998DF82E0018F8060087EA000615F868
:100FA00009707E40049F56409DF82D208DF82D60DD
:100FB0001BF8096073401BF801606340584018F843
:100FC00002308DF82C0018F80E0083EA00047440FB
:100FD000EE5D744015F80E608DF82B4018F8014056
:100FE000634073401BF80760734018F80760069F62
:100FF0008DF82A3084EA0603AC5C1BF802206340BB
:101000001BF80E405C409DF829308DF829406C5C3F
:1010100005996240504018F8032070401BF80760A3
:101020008DF8280018F80C0082EA000474406E5C09
:10103000744015F80C608DF8274018F8074062409E
:1010400072401BF801607240EE5C1BF803308DF8B3
:10105000262018F801201BF80C1054407440029E02
:101060006140089C8DF82510E95D594048402146B3
:1010700050408DF8240009A800F0E6FB07981034D2
:1010800001301AE76C4D9DF829309DF82610A85CB8
:101090009DF82820AA5C8DF824009DF825008DF885
:1010A00028209DF82C20285CAA5C8DF82C209DF827
:1010B0003020AA5C8DF830209DF82D20AA5C8DF898
:1010C0002920EA5C8DF825209DF831208DF831002B
:1010D000685C9DF82E108DF82E00685C9DF832102B
:1010E000AA5C8DF826009DF82A008DF82D20224656
:1010F000285C8DF83200685C9DF833108DF82A006A
:101100009DF82F00285C8DF833009DF82B00285C9B
:101110008DF82F00685C9DF827108DF82700685C1B
:101120008DF82B0009A90198FFF76CFE002000E064
:10113000FF200DB0BDE8F08F00810108008001089C
:101140002DE9F84FA1F11003102B6DD8012404FAFA
:1011500003F3384C234267D013460C46250605D0CE
:1011600010F8015B013C03F8015BF7E77020DFF842
:10117000C88002EB010A4FF00109002500EB810055
:10118000C3B24FF0FF3000EB1310009382F8F00071
:10119000009B4819984244D2C0B20AEB0507B0FB45
:1011A000F1F317F8024C17F801BC03FB110617F80E
:1011B000040C17F8033C6EB119291DD3F6B2102E9A
:1011C0001AD118F80BE018F804C018F8036018F8E2
:1011D000000014E018F800E018F8030018F80460A4
:1011E0004FFA89F31B2418F80BC004EAD31380EAE2
:1011F000090083EA490902E01E46A446DE46535D23
:1012000058400AF8050050190435437873407B7044
:10121000837883EA0C03BB70C07880EA0E00F87014
:10122000B6E70020BDE8F88F002082F8F000FF202C
:10123000BDE8F88F0101010000820108F1F7E4FA2E
:10124000FCF798FFF6F77CFCF6F7DCFCF6F754FDAC
:10125000F6F7FEFCF6F703FDFCE7130408BF704742
:1012600011F8013B013A00F8013BF6E71044013860
:10127000130408BF704711F8013B013A00F8013927
:10128000F6E7130408BF704700F8011B013AF8E7BE
:101290002DE9F04F87B0D1E900750E46804614461F
:1012A0003846F6F7FBFFF7F79CFA60603846F7F729
:1012B00047F8F7F796FA2060B8F8000006F108033F
:1012C000451E06EBC50004F10806021DD8F81400FF
:1012D00000F10804012D47DB18680692CDE90106EC
:1012E00052F8041C5E68CDE90335009101F0E2F983
:1012F0008246069831460768F7F78BFA05948346CD
:101300002568059844685046F7F717F9804628463F
:10131000F7F731F881463046029EF7F7B4FAF7F74F
:101320007AF9F7F726FAF7F75CFA70605046F7F7A4
:10133000EAF805465846F7F700F90446DDE90001EA
:1013400000F006FEF6F7AAFF2146059C01F0B2F96F
:10135000F7F747FADDE90335069A306008340836B6
:101360000833083A013DB5E707B0BDE8F08F00004B
:10137000B0B50E4A0A4D43F23904091A0131136817
:1013800003FB054313606FF00042B3FBF2F2C2EBC4
:10139000C2729A1A92FBF1F303FB11210844B0BD0B
:1013A0006D4EC64101490860704700BF48010020EA
:1013B0002DE9F04F87B08146D1E900070D4616466A
:1013C000014600F0C5FD04463846F7F74DF80746DC
:1013D0002046F7F758FAF7F704FA70602046F7F757
:1013E00043F8F7F7FEF9B9F80010306006F1080A83
:1013F00005F1080805EBC100021FD9F8140000F13F
:101400000809CDE9051252F8040CD8F80010D8F8F4
:1014100004600490039101F04DF904460190069890
:1014200031460768F7F7F5F9009005462046D9E9F7
:1014300000B1029100F0EAFF04465846F7F763F85E
:1014400005463046F7F71FFAF7F765FAF6F726FF75
:10145000F7F7C7F9CAF804000198F6F78CFF0746BA
:101460000098029900F0D2FF0646DDE9031000F073
:101470006FFDF6F7F9FFF7F7ECF8F7F7B2F9DDE9EA
:101480000512CAF800000AF1080A08F1080809F173
:1014900008090139083A0129B3DC07B0BDE8F08F2B
:1014A00081B0C0B5039303AB04A21021009300F0F8
:1014B0000BF8BDE8884001B0704700BF2564732574
:1014C0003033643A000000002DE9F04F97B0064633
:1014D00000200129C0F227810DF11A00A1F1010BB2
:1014E00015464FF0200AB14603960138CDF804B0F6
:1014F00002902978A9EB0600002900F011815845D7
:1015000080F20E81252919D12F4617F8012FA2F15B
:101510003004B4FA84F14909092C12D802354FF08D
:101520000008A2F13004092C0FD808EB880402EB64
:101530004402A2F1300815F8012BF2E709F8011B6B
:10154000ECE04FF0FF383D4600E0013D252A35D064
:10155000582A1AD0782A19D0642A13D0692A11D0AF
:10156000732A16D0752A46D0632A22D109F10109BF
:10157000B8F1020F2BDB09F801AC09F10109A8F160
:101580000108F5E70495023136E040310495102258
:1015900033E01C46654880CC002F08BF074638461C
:1015A000EEF7C0FE404516DA09F801ABA8F10108D4
:1015B000F8E7252009F8010BA9EB060058451ADACF
:1015C0002A78A2B109F8012BA9EB060010E001CBA3
:1015D00009F8010CA2E0039E0021814204DA7A5C42
:1015E00009F801200131F8E78944234696E0013DDE
:1015F0005845C0F2938004950A22480656A5A6EBEA
:10160000090A4BA058BF054653F804BB00200593B8
:1016100001F00203BBF1000F48BF012000EA530EA6
:10162000BEF1000F18BFCBF1000B7346A8EB0E08FC
:1016300011F0010C4FF0300108BF2021BEF1000F66
:1016400018BF2D23BBF1000F0ED00020BBF1000FFF
:101650000ED0BBFBF2F70DF11A0607FB12B4BB4626
:101660002C5D34540130F1E730208DF81A00012050
:10167000DDF804B0A8EB0005BCF1000F0AEB0B028B
:1016800013D1DDF808C0002600244FF0200A2F19DE
:10169000012F11DB013C09F806A001361719F6D11C
:1016A000059B039EA9EB040937E01E46059BDDF868
:1016B00008C04FF0200A05E01E46059BA9EB04096F
:1016C00022447D1EBEF1000F05D009F8016B039E78
:1016D000013A01D121E0039E6F1E002D05DD09F8BE
:1016E000011B013A3D46F7D117E0002100280ADD31
:1016F000441E1CF8000009F80100013120468A420E
:10170000F4D1894409E08944501A012F05DB09F816
:1017100001AB0138A7F10107F7D1049D0135E8E6D7
:10172000002189F8001017B0BDE8F08FBD860108D0
:101730003031323334353637383961626364656647
:101740006768696A6B6C6D6E6F70717273747576B1
:101750007778797A0000000030313233343536370B
:1017600038394142434445464748494A4B4C4D4E1F
:101770004F505152535455565758595A0000000073
:1017800080B50848016841F400310160016821F426
:10179000003101602B48F2F737FD0F20F1F74AF8CE
:1017A000002080BD3800005880B506490860F6F773
:1017B000B5F9F6F7D9FA0448016841F00061016013
:1017C000002080BD501900208008005810B50F4936
:1017D0001C4C486020464FF40011F2F758FB20687B
:1017E000C169C903FCD4C1694902FCD58168154CA3
:1017F00041F4800181602046F2F713FB0349204643
:101800000122F2F77FFD002010BD00BFB0010020D3
:1018100080B50C48F2F7DAFC08B1EFF771FB044829
:10182000F0F742FA18B1BDE88040EFF769BB80BD20
:10183000DC49002080B50A4601460248F2F79EFDC9
:10184000002080BD184B002070B50A7803784478DA
:101850008578C6785A4002704A78624042708A7829
:101860006A408270CA787240C27002790B795A401D
:10187000437902714A795A40837942718A795A4090
:10188000C3798271CA795A40037AC2710A7A5A407E
:10189000437A02724A7A5A40837A42728A7A5A406A
:1018A000C37A8272CA7A5A40037BC2720A7B5A4058
:1018B000437B02734A7B5A40837B42738A7B5A4044
:1018C0008273C27BC97B5140C17370BD2DE9F04169
:1018D000C0F3C751A1F17F050446172DA8BFBDE88D
:1018E000F0814FF07F471549002D0FDA00F030FBF3
:1018F000B7EB400F1FD300281DDD002CA8BF00242C
:1019000019DAB4F1004F18BF0D4C14E00D4A22FA59
:1019100005F6344208BFBDE8F08100F019FBB7EBD3
:10192000400F08D3002806DD002C03DA4FF4000036
:10193000E8400444B4432046BDE8F081CAF249714E
:10194000000080BFFFFF7F0070B5054600F02AFE53
:10195000044620F00040C0F1FF40C00F08D025F041
:101960000040C0F1FF40C00F04BF0120EEF7C9FDE9
:10197000204670BD21F0004201F00043A2F1605208
:10198000B2F5801F28BFD2F17F6C0BD95FEA001C33
:1019900043EAC20242EB507018BF704728BF20F0E4
:1019A00001007047B2F5801FBCBF184670474FEA70
:1019B000410C1CF5001F02D2084600F0EEBD70B5C8
:1019C00000F05CF900000089FFF7F6BF4FF000401F
:1019D000A0F580007047000010B591EA030F48BFE2
:1019E00083F0004300F1A681841A71EB030C05D249
:1019F000121943EB0C03001B61EB0C014FEA11546D
:101A0000A4EB135CDFF81CE11EEA430F18BF9EEA4B
:101A1000445F73D021EA045123EA0E0343F4801398
:101A2000DCF1200E32D322FA0CFE10EB0E0023FA6A
:101A30000CFE41EB0E01CCF1200E03FA0EFE10EB72
:101A40000E00CCF1200E51F10001B1F5801F32D211
:101A500001EB045112FA0EF2BDE8104058BF704776
:101A6000401C38BF5FEA420218BF7047002814BF0D
:101A700020F0010041F100014FEA410313F5001F7E
:101A800038BF7047A1F1C04100F046B9012A43EBCD
:101A90000302ACF1200CDCF11F0E32BF4FF0000E40
:101AA00023FA0CF310EB030041EB0451B4EB115F8C
:101AB000D0D0A1EB045101F58011490801EB04518C
:101AC0005FEA30000ED350F1000038BF12FA0EFE6C
:101AD00008D1BDE81040C9E7401C38BF5FEA4202A8
:101AE000CAD1C3E7BDE810404FEA410313F5001F18
:101AF00038BF7047A1F1C04100F00EB99EEA445FC3
:101B000008D011EA5E0FBDE8104004BF01F00041AB
:101B100000207047BDE8104070B500F0AFF800BF7E
:101B200064FBBE3E0000E0FF70B5DFF848C11CEA70
:101B3000111E1EBF1CEA13159EEA0C0F95EA0C0F2E
:101B400000F06F8081EA03044EEAD47EAE4421EABD
:101B50004C1123EA4C1341F4801143F48013AEF18D
:101B60007F7EA1FB024CA0FB0365361955EB0C05EB
:101B7000A1FB034C4CF10003A0FB021C16EB0C066E
:101B8000654153F10003094218BF46F0010613F402
:101B9000007F0BD14FEA03314FEA053041EA15517E
:101BA00040EA165034036FF003020AE04FEAC32103
:101BB0004FEAC52041EA555140EA5650F4026FF011
:101BC000020202EB2E4201EB025585EACE710AD0E9
:101BD0005FEA440C18BF24F0004450F1000041F1CA
:101BE000000120EAD47040F2FE7C624500D270BD54
:101BF000A84214BF4FF080444FF04044002E08BF6D
